:100000000C949A2F0C94CB2F0C94CB2F0C94CB2FB9
:100010000C94CB2F0C94CB2F0C94CB2F0C94CB2F78
:100020000C9482910C94CB2F0C94CB2F0C945FBD2D
:100030000C94CB2F0D94EAA20C94CB2F0C94CB2FC5
:100040000C94CB2F0D940E0D0C94CB2F0C94CB2F26
:100050000C94CB2F0C94CB2F0D9432220D94119B2A
:100060000C94CB2F0C943D3C0C94CB2F0C94CB2FA9
:100070000C94CB2F0C94CB2F0C94CB2F0C94CB2F18
:100080000C94CB2F0C94CB2F0C94CB2F0C94CB2F08
:100090000C94813C0C94CB2F0C94CB2F0C94CB2F35
:1000A0000C94CB2F0C94CB2F0C94CB2F0C94CB2FE8
:1000B0000C94CB2F0C94CB2F0C94CB2F0C94CB2FD8
:1000C0000C94CB2F0C94CB2F0C94CB2F0C94CB2FC8
:1000D0000C94CB2F0C94CB2F0C94CB2F0C94CB2FB8
:1000E0000C94CB2F2C3B303B353B3D3B523B6B3B89
:1000F000903BBA3B2E013401840160017801C001BC
:10010000C2018C013E016401BA0156012A0180013D
:100110009001B601AA01DC01A2018601BE014201E3
:1001200082016801CA01740174017401B401B4014F
:10013000B40194016601B401EA01C401D401400193
:100140003A01DE014A013C019201A401AE015E01C7
:10015000A601AC01D2014A015A01E8019C01280123
:10016000CC01E201D001E001BC014C019A017E0109
:100170007201B801700144015201BC01B0013001AB
:100180005C01084AD73B3BCE016E84BCBFFDC12F4A
:100190003D6C74319ABD56833DDA3D00C77F11BE78
:1001A000D9E4BB4C3E916BAAAABE000000803F057B
:1001B000A84CCDB2D44EB93836A9020C50B99186AC
:1001C00088083CA6AAAA2ABE000000803F07634216
:1001D00036B79BD8A71A39685618AEBAAB558C1DDE
:1001E0003CB7CC5763BD6DEDFD753EF6177231BF60
:1001F000000000803F08000000BE922449123EAB80
:10020000AAAA2ABECDCCCC4C3E00000080BEABAA30
:10021000AAAA3E00000000BF000000803F000000CE
:100220000000084178D3BB4387D1133D190E3CC36E
:10023000BD4282AD2B3E68EC8276BED98FE1A93EED
:100240004C80EFFFBE01C4FF7F3F000000000000B4
:100250000D940B9D0D94B6560D9487250D942E4646
:100260000D943C9D0D9494290D9443460D9466285D
:100270000D943C650D94669C0D947A9C0D94C54636
:100280000D945C9C0D945B580D942E9D0D94903FA5
:100290000D941C7B0D94E99C0D94129D0D949A294C
:1002A0000D94A68C0D94329D0D94D87D0D949E5680
:1002B0000D942B410D94CB9C0D94409D0D949E9CD0
:1002C0000D9462460D94B2420D94DF460D94EE58A3
:1002D0000D94A8580D9414850D9497420D94854C57
:1002E0000D942A9D0D94209D0D94B8580D94A9420B
:1002F0000D9487460D94A0420D94183A0D941C9DC0
:100300000D94CD560D947E580D9448460D942D585D
:100310000D94A9490D9443370D94B0460D9488442B
:100320000D94E3560D94829C0D94C0580D947676EE
:100330000D94DC9D0D94169D0D94DF9C0D94532B14
:100340000D94E9260D940A580D948A9C0D94A89C4E
:100350000D9459280D9425570D94B79C0D94949C99
:100360000D94389D0D9485290D94DE580D94F75603
:100370000D94249D0D9407470D94459D0D943E5872
:100380000D948C460D9496460D94529C0D945C43AE
:100390000D943C6D0D94B0580D940E9D0D94BB457D
:1003A0000D94019D0D94C19C0D94579C0D943D742A
:1003B0000D94BC310D942A320D9442570D94709CCB
:1003C0000D94079D0D94FD9C0D9481320D94206C2D
:1003D0000D94D59C0D94CA580D945A91486172643D
:1003E000636F6465642044656661756C7420536551
:1003F0007474696E6773204C6F6164656400537434
:100400006F7265642073657474696E6773207265BA
:10041000747269657665640046696C616D656E74B9
:100420002073657474696E67733A204469736162FE
:100430006C6564002020204D323030204400466935
:100440006C616D656E742073657474696E67733A60
:10045000002020204D3230392053004175746F2D1B
:10046000526574726163743A20533D3020746F207A
:1004700064697361626C652C203120746F20696E31
:100480007465727072657420657874727564652D18
:100490006F6E6C79206D6F76657320617320726565
:1004A000747261637473206F72207265636F766516
:1004B00072696573002046002020204D32303820BC
:1004C00053005265636F7665723A20533D457874E8
:1004D0007261206C656E67746820286D6D292046F6
:1004E0003A537065656420286D6D2F6D2900205A80
:1004F000002046002020204D323037205300526526
:1005000074726163743A20533D4C656E6774682061
:10051000286D6D2920463A537065656420286D6DFD
:100520002F6D29205A3A205A4C69667420286D6D27
:1005300029002044002049002020204D3330342061
:100540005000504944206865617462656420736599
:100550007474696E67733A002044002049002020BB
:10056000204D33303120500050494420736574745D
:10057000696E67733A00205A0020590020204D32DE
:100580003036205800486F6D65206F66667365745D
:1005900020286D6D293A00204500205A002059007E
:1005A00020580020420020540020204D32303520B9
:1005B0005300416476616E6365642076617269619F
:1005C000626C65733A20533D4D696E2066656564C3
:1005D0007261746520286D6D2F73292C20543D4D58
:1005E000696E2074726176656C20666565647261FF
:1005F000746520286D6D2F73292C20423D6D696E26
:10060000696D756D207365676D656E742074696DB5
:100610006520286D73292C20583D6D6178696D75B2
:100620006D205859206A65726B20286D6D2F7329D3
:100630002C20205A3D6D6178696D756D205A206AB5
:1006400065726B20286D6D2F73292C2020453D6D20
:100650006178696D756D2045206A65726B20286D23
:100660006D2F73290020540020204D323034205348
:1006700000416363656C65726174696F6E3A205303
:100680003D616363656C65726174696F6E2C2054A3
:100690003D7265747261637420616363656C657239
:1006A0006174696F6E00204500205A0020590020B7
:1006B000204D3230312058004D6178696D756D20C4
:1006C000416363656C65726174696F6E20286D6D3E
:1006D0002F7332293A00204500205A00205900206B
:1006E000204D3230332058004D6178696D756D2092
:1006F00066656564726174657320286D6D2F73295A
:100700003A00204500205A0020590020204D39325F
:1007100020580053746570732070657220756E697F
:10072000743A0053657474696E67732053746F7202
:10073000656400454550524F4D204572726F7200FE
:100740006F6B0A002046002045004731205A0020E8
:10075000423A0020453A00543A005A206C697665C6
:100760002061646A757374206F7574206F662072DF
:10077000616E67652E2053657474696E6720746FAF
:1007800020302E20436C69636B20746F20636F6E82
:1007900074696E75652E005A206C697665206164F7
:1007A0006A757374206F7574206F662072616E674E
:1007B000652E2053657474696E6720746F20300055
:1007C00020573A0020453A00543A004B494C4C3AE5
:1007D00020004D3730310022283229005400496E64
:1007E00076616C6964205420636F64652E00556ED9
:1007F0006B6E6F776E204D20636F64653A202573B2
:10080000200A004D3232302053256900203A200062
:10081000004C414E472053454C20464F52434544DF
:1008200000222831290020453A00205A3A00205958
:100830003A0020453A00205A3A0020593A00583AE6
:10084000004D31313320530020002E0020423A0069
:1008500020453A00543A0020503A002042403A00E5
:1008600020403A00202F003A00205400202F002082
:10087000423A00202F006F6B20543A002569206D0A
:10088000696E2C2025692073656300496E76616C62
:100890006964204D20636F64653A202573200A0047
:1008A000556E6B6E6F776E204720636F64653A20DC
:1008B0002573200A004D65736820626564206C65AD
:1008C00076656C696E67206E6F74206163746976FB
:1008D000652E000A002020000A4D6561737572655F
:1008E0006420706F696E74733A000A5A20736561F0
:1008F000726368206865696768743A20002C004E4E
:10090000756D20582C593A2000206D6963726F6E06
:10091000730045786365737369766520626564204A
:100920006C6576656C696E6720636F72726563745F
:10093000696F6E3A2000473238205730003A200065
:1009400054656D70657261747572652063616C6960
:1009500062726174696F6E20646F6E652E20436FE2
:100960006E74696E7565207769746820707265733E
:1009700073696E6720746865206B6E6F622E00006D
:10098000205A20736869667420286D6D293A0050DA
:10099000494E44412074656D70657261747572656D
:1009A0003A2000002F3600537465703A2000002072
:1009B0005A20736869667420286D6D293A00504981
:1009C0004E44412074656D70657261747572653A4C
:1009D00020002F362028736B6970706564290053DE
:1009E0007465703A2000005A45524F3A2000007357
:1009F000746172742074656D70657261747572656E
:100A00003A200050494E44412070726F6265206365
:100A1000616C6962726174696F6E20737461727463
:100A200000473238205730000A00205A3A20002070
:100A3000593A200020583A200043616C6962726183
:100A400074696F6E206661696C6564212043686516
:100A5000636B20746865206178657320616E642023
:100A600072756E20616761696E2E004D32390062C9
:100A70007573793A2070617573656420666F7220B2
:100A8000696E70757400627573793A207061757360
:100A9000656420666F722075736572006275737984
:100AA0003A2070726F63657373696E6700205570CA
:100AB0006C6F616420696E2070726F67726573730A
:100AC0000044495341424C45440A00454E41424C82
:100AD00045440A004653656E736F722000504154BE
:100AE000393132355F696E69743A25640A004665AA
:100AF00062202031203230313800436F6D70696CD4
:100B000065643A2000286E6F6E652C20646566610E
:100B1000756C7420636F6E66696729004665622094
:100B2000203120323031382032303A31323A3234CA
:100B30000020332E312E312D5243352D3135310ADF
:100B400000737461727400466163746F727920522D
:100B500045534554001B5B324A1B5B313B31484FC8
:100B6000726967696E616C205072757361206933B8
:100B70001B5B323B3348507275736120526573655D
:100B800061726368002500202020202020002020A2
:100B9000202020200045524153494E4720616C6C73
:100BA000206461746100466163746F7279205245FC
:100BB00053455400FFFFFF0000A0400000A040008C
:100BC00000004000007F43000056439AD951430083
:100BD000000000000080C09A99193E00007F430089
:100BE0000052430000524300000000000080C09A01
:100BF00099193E6563686F3A004572726F723A00E8
:100C000000002110422063308440A550C660E77088
:100C1000088129914AA16BB18CC1ADD1CEE1EFF130
:100C20003112100273325222B5529442F772D662D8
:100C3000399318837BB35AA3BDD39CC3FFF3DEE380
:100C40006224433420040114E664C774A444855428
:100C50006AA54BB528850995EEE5CFF5ACC58DD5D0
:100C60005336722611163006D776F6669556B44678
:100C70005BB77AA719973887DFF7FEE79DD7BCC720
:100C8000C448E5588668A7784008611802282338C8
:100C9000CCC9EDD98EE9AFF9488969990AA92BB970
:100CA000F55AD44AB77A966A711A500A333A122A18
:100CB000FDDBDCCBBFFB9EEB799B588B3BBB1AABC0
:100CC000A66C877CE44CC55C222C033C600C411C68
:100CD000AEED8FFDECCDCDDD2AAD0BBD688D499D10
:100CE000977EB66ED55EF44E133E322E511E700EB8
:100CF0009FFFBEEFDDDFFCCF1BBF3AAF599F788F60
:100D00008891A981CAB1EBA10CD12DC14EF16FE13F
:100D10008010A100C230E320045025404670676077
:100D2000B9839893FBA3DAB33DC31CD37FE35EF38F
:100D3000B1029012F322D2323542145277625672C7
:100D4000EAB5CBA5A89589856EF54FE52CD50DC5DF
:100D5000E234C324A0148104667447642454054417
:100D6000DBA7FAB79987B8975FE77EF71DC73CD72F
:100D7000D326F2369106B016576676761546345667
:100D80004CD96DC90EF92FE9C899E9898AB9ABA97F
:100D90004458654806782768C018E1088238A328B7
:100DA0007DCB5CDB3FEB1EFBF98BD89BBBAB9ABBCF
:100DB000754A545A376A167AF10AD01AB32A923A07
:100DC0002EFD0FED6CDD4DCDAABD8BADE89DC98D1F
:100DD000267C076C645C454CA23C832CE01CC10C57
:100DE0001FEF3EFF5DCF7CDF9BAFBABFD98FF89F6F
:100DF000176E367E554E745E932EB23ED10EF01EA7
:100E00007C3C3E5E2B3D3F2F5B5D3B2C2A225C00F1
:100E10004D3234004D3233202573006175746F25D7
:100E2000692E67000A002F000A002E0044656C65D9
:100E300074696F6E206661696C65642C2046696C0C
:100E4000653A200046696C652064656C657465646C
:100E50003A002E002E002E002E004E6F7720667274
:100E60006573682066696C653A20004E6F77206470
:100E70006F696E672066696C653A20002220706F8A
:100E800073002220706172656E743A2200535542DD
:100E9000524F5554494E452043414C4C2074617289
:100EA0006765743A2200747279696E6720746F20E6
:100EB00063616C6C207375622D67636F6465206677
:100EC000696C6573207769746820746F6F206D6139
:100ED0006E79206C6576656C732E204D4158206CC0
:100EE0006576656C2069733A00256920686F7572B4
:100EF00073202569206D696E757465730054494DC2
:100F0000454F55543A004D3131300046756C6C20D8
:100F10005258204275666665720022206661696CCF
:100F200065643A204275666665722066756C6C2150
:100F300000456E717565696E6720746F2074686511
:100F40002066726F6E743A2022002200456E717521
:100F500065696E6720746F207468652066726F6EB5
:100F6000743A20220022206661696C65643A20424E
:100F700075666665722066756C6C210022004D36C0
:100F80003030004731204533204632303000473181
:100F900020452D3320463230300050727573612069
:100FA0006933204D4B322E35206F6B0050727573B4
:100FB00061206933204D4B322E3520726561647992
:100FC0002E007A5F6D696E3A20007A5F6D61783A23
:100FD00020005A204F666673657400795F6D696EF4
:100FE0003A2000795F6D61783A20005920767A6462
:100FF000616C656E6F7374206F64206D696E3A006A
:10100000592064697374616E63652066726F6D2028
:101010006D696E3A00416E6F0059657300785F6DBF
:10102000696E3A2000785F6D61783A2000446574FB
:1010300061696C792058595A206B616C2E0058599F
:101040005A2063616C2E2064657461696C73004E74
:10105000796E692070726F76656475207A206B6195
:101060006C6962726163692E00492077696C6C203B
:1010700072756E207A2063616C6962726174696F47
:101080006E206E6F772E004E796E692070726F76CB
:101090006564752078797A206B616C69627261632E
:1010A000692E205A616265726520746F20707269C2
:1010B000626C697A6E65203132206D696E2E00494E
:1010C0002077696C6C2072756E2078797A20636164
:1010D0006C6962726174696F6E206E6F772E204941
:1010E000742077696C6C2074616B6520617070721C
:1010F0006F782E203132206D696E732E004E796E1E
:10110000692070726564656872656A6920747279B5
:10111000736B752070726F20504C412E004E6F77AC
:1011200020492077696C6C20707265686561742055
:101130006E6F7A7A6C6520666F7220504C412E007B
:10114000446F6272792064656E2C206A73656D202D
:1011500076617365207469736B61726E61204F7282
:101160006967696E616C2050727573612069332EF6
:101170002043686365746520616279636820566105
:10118000732070726F7665646C61206B616C69624C
:101190007261636E696D2070726F636573656D3F18
:1011A0000048692C204920616D20796F7572204FAD
:1011B000726967696E616C20507275736120693362
:1011C000207072696E7465722E20576F756C642082
:1011D000796F75206C696B65206D6520746F206771
:1011E0007569646520796F75207468726F756768BA
:1011F000207468652073657475702070726F636504
:1012000073733F005A61636E75207469736B6E6F00
:101210007574206C696E6B7520612056792062753B
:101220006465746520706F737475706E6520736E7D
:10123000697A6F76617420747279736B75206F743C
:101240006163656E696D20746C616369746B6120A4
:10125000646F6B7564206E65646F7361686E65742E
:1012600065206F7074696D616C6E69207679736B3F
:10127000792E2050726F686C65646E65746520739A
:1012800069206F6272617A6B792076206E61736972
:101290002070726972756363652076206B61706976
:1012A000746F6C65204B616C6962726163650049A3
:1012B0002077696C6C20737461727420746F207075
:1012C00072696E74206C696E6520616E6420796F3E
:1012D000752077696C6C206772616475616C6C79DC
:1012E000206C6F77657220746865206E6F7A7A6CF7
:1012F0006520627920726F746174696E672074680A
:1013000065206B6E6F622C20756E74696C20796F2E
:1013100075207265616368206F7074696D616C20FF
:101320006865696768742E20436865636B2074681C
:101330006520706963747572657320696E206F75BE
:10134000722068616E64626F6F6B20696E206368E3
:1013500061707465722043616C6962726174696F57
:101360006E2E004E796E69207A6B616C69627275BF
:101370006A6920767A64616C656E6F7374206D653E
:101380007A69206B6F6E63656D20747279736B7907
:10139000206120706F76726368656D206865617486
:1013A000626564752E004E6F7720492077696C6CFA
:1013B0002063616C69627261746520646973746131
:1013C0006E6365206265747765656E207469702050
:1013D0006F6620746865206E6F7A7A6C6520616E26
:1013E0006420686561746265642073757266616308
:1013F000652E004E656A6472697620706F6D6F634A
:10140000692073656C667465737475207A6B6F6E92
:10141000746F6C756A69206E656A63617374656A5E
:10142000736920636879627920767A6E696B616A84
:101430006963692070726920736573746176656E83
:1014400069207469736B61726E792E0046697273DC
:10145000742C20492077696C6C2072756E2074683A
:10146000652073656C667465737420746F2063689F
:1014700065636B206D6F737420636F6D6D6F6E208D
:10148000617373656D626C792070726F626C656DEB
:10149000732E005370757374656E692057697A6195
:1014A0007264612076796D617A6520756C6F7A65FA
:1014B0006E65207679736C65646B792076736563ED
:1014C00068206B616C69627261636920612073706E
:1014D00075737469206B616C69627261636E6920F7
:1014E00070726F636573206F64207A616361746BDF
:1014F000752E20506F6B7261636F7661743F00527E
:10150000756E6E696E672057697A617264207769BB
:101510006C6C2064656C6574652063757272656EB1
:10152000742063616C6962726174696F6E207265A8
:1015300073756C747320616E6420737461727420AF
:1015400066726F6D2074686520626567696E6E698A
:101550006E672E20436F6E74696E75653F00436839
:1015600063657465206F70616B6F76617420706F56
:10157000736C65646E69206B726F6B206120706F95
:101580007A6D656E697420767A64616C656E6F73CE
:1015900074206D657A6920747279736B6F75206140
:1015A00020686561746265643F00446F20796F75DF
:1015B0002077616E7420746F20726570656174208D
:1015C0006C617374207374657020746F2072656130
:1015D000646A7573742064697374616E63652062F4
:1015E00065747765656E206E6F7A7A6C6520616EC2
:1015F0006420686561746265643F0057697A61724E
:101600006461206D757A657465206B64796B6F6CAD
:101610006976207A6E6F767520737075737469744D
:10162000207A206D656E752043616C696272617409
:10163000696F6E202D3E2057697A61726400596F80
:10164000752063616E20616C7761797320726573B8
:10165000756D65207468652057697A6172642066CB
:10166000726F6D2043616C6962726174696F6E2084
:101670002D3E2057697A6172642E004A6520746F8E
:1016800020504C412066696C616D656E743F004965
:101690007320697420504C412066696C616D656EE1
:1016A000743F0050726F73696D20766C6F7A746549
:1016B00020504C412066696C616D656E7420646FCA
:1016C000206578747275646572752C20706F207453
:1016D0006520737469736B6E65746520746C6163E7
:1016E00069746B6F2070726F207A61766564656EC5
:1016F000692066696C616D656E74752E00506C654D
:1017000061736520696E7365727420504C41206668
:10171000696C616D656E7420746F207468652065F6
:10172000787472756465722C207468656E207072AE
:10173000657373206B6E6F6220746F206C6F6164D1
:101740002069742E0050726F73696D207A6176651E
:1017500064746520504C412066696C616D656E74DF
:10176000206120706F207465206F626E6F767465E3
:101770002057697A6172646120737469736B6E7546
:1017800074696D20726573657420746C616369742B
:101790006B612E00506C65617365206C6F61642015
:1017A000504C412066696C616D656E7420616E6499
:1017B000207468656E20726573756D652057697A4F
:1017C000617264206279207265626F6F74696E67FE
:1017D00020746865207072696E7465722E00507294
:1017E00065646568726976616D20747279736B7572
:1017F0002E2050726F73696D2063656B656A746526
:101800002E0050726568656174696E67206E6F7A2C
:101810007A6C652E20506C65617365207761697400
:101820002E004A652066696C616D656E74207A6170
:10183000766564656E3F0049732066696C616D650D
:101840006E74206C6F616465643F00567365206A36
:101850006520686F746F766F2E00416C6C20697321
:1018600020646F6E652E20486170707920707269F7
:101870006E74696E67210050726F73696D206F63BB
:10188000697374657465206865617462656420615C
:1018900020737469736B6E65746520746C61636921
:1018A000746B6F2E00506C6561736520636C6561AD
:1018B0006E206865617462656420616E642074687E
:1018C000656E20707265737320746865206B6E6F2F
:1018D000622E0050726F73696D206E61686C656472
:1018E0006E65746520646F206D616E75616C752026
:1018F00061206F7072617674652070726F626C65C2
:101900006D2E20506F207465206F626E6F76746547
:101910002057697A61726461207265626F6F746FBB
:1019200076616E696D207469736B61726E792E00D9
:10193000506C6561736520636865636B206F7572B9
:101940002068616E64626F6F6B20616E64206669EF
:1019500078207468652070726F626C656D2E2054FB
:1019600068656E20726573756D65207468652057B3
:10197000697A617264206279207265626F6F74693E
:101980006E6720746865207072696E7465722E00CF
:1019900057697A61726400205761746368646F6785
:1019A00020526573657400496E666F726D61636580
:1019B00000496E666F2073637265656E0043656BE8
:1019C000616E69206E61207A63686C61646E757403
:1019D0006920747279736B79206120706F646C6F09
:1019E0007A6B792E0057616974696E6720666F7231
:1019F000206E6F7A7A6C6520616E64206265642067
:101A0000636F6F6C696E67004B616C2E207072762D
:101A10006E692076727374767900466972737420E9
:101A20006C617965722063616C2E00576169742066
:101A3000666F7220757365722E2E2E00506F757A48
:101A400069746520626568656D207469736B7500E3
:101A50005573656420647572696E67207072696E73
:101A6000740042796C6F20767973756E7574692095
:101A700066696C616D656E74752075737065736EE3
:101A8000653F005761732066696C616D656E7420F7
:101A9000756E6C6F616420737563636573736675CF
:101AA0006C3F0056796A6D6F75742066696C616D64
:101AB000656E7400556E6C6F61642066696C616D53
:101AC000656E74005679736F7576616D2066696C0A
:101AD000616D656E7400556E6C6F6164696E672030
:101AE00066696C616D656E7400556E6B6E6F776EB6
:101AF00020636F6D6D616E643A2022004C616469F1
:101B0000740054756E650053442063617264205BF9
:101B1000466C73684169725D00534420636172646E
:101B200020205B6E6F726D616C5D00537461626C3E
:101B30006520616D6269656E742074656D70657293
:101B400061747572652032312D32364320697320FD
:101B50006E656564656420612072696769642073DD
:101B600074616E6420697320726571756972656451
:101B70002E005465706C2E206B616C2E20205B7AD9
:101B800061705D0054656D702E2063616C2E2020A5
:101B9000205B6F6E5D005465706C2E206B616C2E47
:101BA00020205B7679705D0054656D702E20636136
:101BB0006C2E20205B6F66665D005465706C6F74E0
:101BC0006E69206B616C69627261636520646F6B22
:101BD0006F6E63656E612E20506F6B726163756A04
:101BE000746520737469736B656D20746C616369CF
:101BF000746B612E0054656D7065726174757265E9
:101C00002063616C6962726174696F6E2069732010
:101C100066696E69736865642E20436C69636B2026
:101C2000746F20636F6E74696E75652E00546570F5
:101C30006C2E206B616C2E20202020202020202064
:101C4000200054656D702E2063616C2E20202020B2
:101C5000202020202020005465706C6F7461005497
:101C6000656D706572617475726500506F64706F38
:101C7000726100537570706F7274005A6173746191
:101C8000766974207469736B0053746F702070727E
:101C9000696E740053544F505045442E20005374C5
:101CA00065707261746520746F6F20686967683A47
:101CB00020004A65207469736B6F767920706C61BF
:101CC00074206E6120686561746265643F004973C9
:101CD00020737465656C207368656574206F6E2071
:101CE000686561746265643F0043656C6B6F76790B
:101CF00020636173203A00546F74616C20707269C4
:101D00006E742074696D65203A0046696C616D657A
:101D10006E742063656C6B656D203A00546F74615E
:101D20006C2066696C616D656E74203A0043617366
:101D3000207469736B75203A2020005072696E74AC
:101D40002074696D653A20200046696C616D656E8E
:101D500074203A20200046696C616D656E742075B0
:101D60007365643A20200053746174697374696BFD
:101D70006120200053746174697374696373202057
:101D8000004368796261202D20446F736C6F206B73
:101D90002070726570697375207374617469636B08
:101DA000652070616D65746921004572726F7220E3
:101DB0002D20737461746963206D656D6F72792075
:101DC000686173206265656E206F766572777269EF
:101DD0007474656E00527963686C6F73740053702D
:101DE0006565640054726964656E69202020202056
:101DF0005B4361735D00536F72743A202020202092
:101E0000205B54696D655D0054726964656E69207C
:101E100020205B5A61646E655D00536F72743A20D6
:101E200020202020205B4E6F6E655D005472696437
:101E3000656E69205B416265636564615D00536F37
:101E400072743A20205B416C7068616265745D0059
:101E500054726964656E6920736F75626F72750084
:101E6000536F7274696E672066696C6573002053E6
:101E70006F667477617265205265736574004C6596
:101E8000686B65207A6B6F73656E693A00536C6995
:101E900067687420736B65773A0053746176206BC2
:101EA0006F6E632E207370696E2E0053686F7720FB
:101EB000656E642073746F70730054657A6B65206F
:101EC0007A6B6F73656E693A00536576657265204B
:101ED000736B65773A004E61737461767465207434
:101EE00065706C6F74753A005365742074656D701D
:101EF000657261747572653A004E617374617665DE
:101F00006E690053657474696E6773004368796223
:101F100061207A61706F6A656E6900576972696ED7
:101F200067206572726F720050726F686F7A656EAB
:101F30006500537761707065640053656C6620744A
:101F40006573742073746172742020005469736B1C
:101F50006F76792076656E742E3A005072696E74D1
:101F60002066616E3A005A6B6F6E74726F6C756AA0
:101F70007465203A00506C65617365206368656321
:101F80006B203A0053656C662074657374204F4B68
:101F9000004E657A61706F6A656E6F2020202000A8
:101FA0004E6F7420636F6E6E6563746564004D6F71
:101FB000746F72004865617465722F546865726D44
:101FC0006973746F720053656E7A6F722066696C04
:101FD000616D656E74753A0046696C616D656E740D
:101FE0002073656E736F723A00546F636920736576
:101FF000005370696E6E696E67004E65746F636939
:10200000207365004E6F74207370696E6E696E6721
:1020100000507265646E692F6C6576792076656E06
:10202000742E0046726F6E742F6C65667420666144
:102030006E7300546573742076656E74696C617498
:102040006F72750046616E20746573740053656C21
:1020500066746573742073656C68616C202000532E
:10206000656C6674657374206661696C65642020B4
:10207000004C6576792076656E742E3A004578744A
:1020800072756465722066616E3A004C65767920DF
:1020900076656E74206E61207472797363653F009B
:1020A0004C65667420686F74656E642066616E3F6F
:1020B0000053656C6674657374206572726F72206C
:1020C0002100456E6473746F70206E6F74206869B0
:1020D0007400456E6473746F707300456E6473743E
:1020E0006F7000507265646E69207469736B6F76EF
:1020F000792076656E743F0046726F6E7420707240
:10210000696E742066616E3F004B6F6E74726F6C07
:1021100061205A2061786973202000436865636BF1
:10212000696E67205A20617869732020004B6F6EBA
:1021300074726F6C612059206178697320200043AC
:102140006865636B696E6720592061786973202028
:10215000004B6F6E74726F6C6120582061786973E8
:10216000202000436865636B696E672058206178A2
:1021700069732020004B6F6E74726F6C6120686F02
:1021800074656E64202000436865636B696E672028
:10219000686F74656E642020004B6F6E74726F6C94
:1021A000612073656E7A6F727500436865636B6951
:1021B0006E672073656E736F727320004B6F6E7461
:1021C000726F6C6120656E6473746F707300436826
:1021D00065636B696E6720656E6473746F707300FE
:1021E0004B6F6E74726F6C612062656420202020DA
:1021F0002000436865636B696E6720626564202018
:1022000020202000567365204F4B202020202020C6
:10221000202020202000416C6C20636F7272656367
:102220007420202020202000426564202F20486553
:10223000617465720044656C6B61206F7379004155
:10224000786973206C656E677468004F7361004134
:102250007869730053656C66746573742020202060
:1022600020202020200052506920706F727420209E
:1022700020205B7A61705D0052506920706F72742B
:1022800020202020205B6F6E5D0052506920706F0F
:102290007274202020205B7679705D005250692096
:1022A000706F7274202020205B6F66665D0057722D
:1022B0006974696E6720746F2066696C653A2000E6
:1022C000766F6C756D652E696E6974206661696CD8
:1022D0006564002053697A653A20004B617274612D
:1022E0002076796A6D75746100436172642072654D
:1022F0006D6F766564005344207072696E74696E08
:1023000067206279746520006F70656E2066616970
:102310006C65642C2046696C653A20006F70656EB0
:10232000526F6F74206661696C6564004B617274F2
:102330006120766C6F7A656E61004361726420691A
:102340006E73657274656400534420696E6974200D
:102350006661696C0046696C652073656C656374C1
:1023600065640046696C65206F70656E65643A202F
:10237000006572726F722077726974696E6720747B
:102380006F2066696C650053442063617264206F3E
:102390006B0043616E6E6F7420656E74657220739E
:1023A00075626469723A200050726176793A00521F
:1023B000696768743A004F626E6F766F76616E6916
:1023C000207469736B7500526573756D696E672053
:1023D0007072696E74004F626E6F76656E692074FC
:1023E00069736B7500526573756D696E67207072E5
:1023F000696E7400506F6B7261636F766174005226
:102400006573756D65207072696E740052657365D1
:102410006E643A20004F64737472616E7465207448
:1024200069736B6F767920706C6174207A206865AF
:1024300061746265642070726F73696D2E00506CF8
:10244000656173652072656D6F766520737465656F
:102450006C2073686565742066726F6D20686561B5
:10246000746265642E0050726F73696D2076796AAC
:102470006D6574652075727963686C656E6520663C
:10248000696C616D656E7400506C65617365207078
:10249000756C6C206F75742066696C616D656E7407
:1024A00020696D6D6564696174656C7900686F772A
:1024B000746F2E707275736133642E637A00686F67
:1024C00077746F2E707275736133642E636F6D0055
:1024D000666F72756D2E707275736133642E637AD8
:1024E00000666F72756D2E707275736133642E6342
:1024F0006F6D00707275736133642E637A00707251
:1025000075736133642E636F6D005469736B207053
:102510006F7A6173746176656E005072696E7420B3
:10252000706175736564005469736B2070726572B5
:102530007573656E005072696E742061626F72749B
:102540006564005072696E74657220646973636FAC
:102550006E6E65637465640050726F207679737572
:102560006E7574692066696C616D656E7475207333
:102570007469736B6E6574652070726F73696D201A
:10258000746C616369746B6F00506C656173652076
:10259000707265737320746865206B6E6F6220744F
:1025A0006F20756E6C6F61642066696C616D656E1D
:1025B000740050726F206E61687261746920747269
:1025C00079736B79206120706F6B7261636F7661D4
:1025D0006E6920737469736B6E65746520746C61C9
:1025E0006369746B6F2E005072657373206B6E6F2E
:1025F0006220746F2070726568656174206E6F7AF6
:102600007A6C6520616E6420636F6E74696E7565A7
:102610002E006120737469736B6E65746520746C31
:10262000616369746B6F00616E64207072657373AF
:1026300020746865206B6E6F620050726564656817
:1026400072656A746520747279736B7521005072BB
:10265000656865617420746865206E6F7A7A6C6550
:102660002100507265646568726576005072656815
:1026700065617400506F77657255700050726F73AA
:10268000696D2063656B656A746500506C65617384
:10269000652077616974004E656A647269766520A9
:1026A0007A61766564746520504C412066696C617E
:1026B0006D656E742070726F73696D2E00506C655D
:1026C000617365206C6F616420504C412066696CB9
:1026D000616D656E742066697273742E004A6520A0
:1026E000504C412066696C616D656E74207A61762C
:1026F0006564656E3F00497320504C412066696CEB
:10270000616D656E74206C6F616465643F002020AC
:10271000506C616E6E657242756666657242797460
:1027200065733A2000556D69737465746520707225
:102730006F73696D207469736B6F767920706C614B
:1027400074206E61206865617462656400506C6518
:1027500061736520706C61636520737465656C20BE
:102760007368656574206F6E206865617462656466
:102770002E004E6168726976616E692050494E4440
:10278000410050494E44412048656174696E6700BC
:10279000504944206B616C2E2020202020202020D6
:1027A000202020005049442063616C2E20202020EE
:1027B0002020202020202000504944206B616C2ED6
:1027C00020756B6F6E63656E6100504944206361D4
:1027D0006C2E2066696E69736865640050494420F8
:1027E0006B616C696272616365005049442063618A
:1027F0006C6962726174696F6E00506F7A61737494
:1028000061766974207469736B005061757365201B
:102810007072696E7400556D697374657465206CAF
:1028200069737420706170697275206E6120706FB9
:10283000646C6F7A6B752061207564727A756A7446
:1028400065206A656A20706F6420747279736B6F9B
:102850007520626568656D206D6572656E692070B2
:1028600072766E696368203420626F64752E205022
:102870006F6B756420747279736B61207A61636821
:102880007974692070617069722C207679706E6538
:102890007465207469736B61726E752E00506C6183
:1028A00063652061207368656574206F66207061C0
:1028B00070657220756E64657220746865206E6F35
:1028C0007A7A6C6520647572696E67207468652019
:1028D00063616C6962726174696F6E206F662066F5
:1028E00069727374203420706F696E74732E20497E
:1028F0006620746865206E6F7A7A6C6520636174F7
:1029000063686573207468652070617065722C203F
:10291000706F776572206F666620746865207072CC
:10292000696E74657220696D6D6564696174656C4A
:10293000792E006F6B004F6666004E6F206D6F76CC
:10294000652E005A61646E61205344206B6172747D
:1029500061004E6F205344206361726400547279A9
:10296000736B61004E6F7A7A6C650046696C616DBD
:10297000656E74206E657A61766564656E00466981
:102980006C616D656E74206E6F74206C6F61646530
:1029900064004261727661206E656E6920636973BE
:1029A000746100436F6C6F72206E6F7420636F727E
:1029B00072656374004E65004E6F0050726F7369EC
:1029C0006D20616B7475616C697A756A74652E002F
:1029D000506C6561736520757067726164652E0067
:1029E0005679736C61206E6F7661207665727A65B8
:1029F000206669726D776172653A004E6577206670
:102A000069726D776172652076657273696F6E2089
:102A1000617661696C61626C653A00506F73756EC6
:102A20006F7574205A004D6F7665205A00506F7391
:102A3000756E6F75742059004D6F76652059005082
:102A40006F73756E6F75742058004D6F76652058E2
:102A5000004578747275646572004B616C696272CE
:102A6000616365205A2E204F746163656E696D2025
:102A7000746C616369746B6120706F73756E7465DB
:102A8000205A206F737520617A206B7E686F726E9A
:102A9000696D7520646F72617A752E20506F74763F
:102AA0007264746520746C616369746B656D2E006B
:102AB00043616C6962726174696E67205A2E20529C
:102AC0006F7461746520746865206B6E6F6220742A
:102AD0006F206D6F766520746865205A206361727F
:102AE000726961676520757020746F207468652055
:102AF000656E642073746F70706572732E20436C02
:102B000069636B207768656E20646F6E652E004B7D
:102B1000616C6962726163652058595A2E204F7446
:102B20006163656E696D20746C616369746B6120AB
:102B3000706F73756E7465205A206F737520617A9B
:102B4000206B7E686F726E696D7520646F72617A3A
:102B5000752E20506F74767264746520746C616396
:102B600069746B656D2E0043616C69627261746992
:102B70006E672058595A2E20526F74617465207404
:102B80006865206B6E6F6220746F206D6F766520B4
:102B9000746865205A206361727269616765207587
:102BA0007020746F2074686520656E642073746F84
:102BB00070706572732E20436C69636B2077686553
:102BC0006E20646F6E652E00506F73756E6F757436
:102BD000206F7375004D6F76652061786973004DC5
:102BE00065736820426564204C6576656C696E6724
:102BF000004E617065746900566F6C74616765732F
:102C0000005465706C6F74790054656D7065726105
:102C10007475726573004B616C6962726163650003
:102C200043616C6962726174696F6E00537461769E
:102C30002072656D656E750042656C7420737461F9
:102C400074757300207A203900206F662039004D9A
:102C50006572696D207265666572656E636E692066
:102C60007679736B75206B616C69627261636E69F2
:102C7000686F20626F6475004D6561737572696E6F
:102C800067207265666572656E6365206865696751
:102C90006874206F662063616C6962726174696F29
:102CA0006E20706F696E74004D6572656E65207A76
:102CB0006B6F73656E693A004D656173757265641B
:102CC00020736B65773A00486C61766E69206E619F
:102CD0006269646B61004D61696E004D3232312072
:102CE000496E76616C69642065787472756465728A
:102CF00020004D32313820496E76616C6964206560
:102D00007874727564657220004D32303020496EDF
:102D100076616C69642065787472756465722000F0
:102D20005265706F7274696E6720656E6473746F3C
:102D30007020737461747573004D313137204B61AD
:102D40006C2E207072766E692076727374767900BC
:102D50004D313137204669727374206C6179657228
:102D60002063616C2E004649524D574152455F4EDB
:102D7000414D453A4D61726C696E2056312E302EB0
:102D8000323B20537072696E7465722F6772626C89
:102D9000206D617368757020666F722067656E368E
:102DA000204649524D574152455F55524C3A68743E
:102DB0007470733A2F2F6769746875622E636F6D34
:102DC0002F707275736133642F50727573612D6942
:102DD000332D506C75732F2050524F544F434F4C2E
:102DE0005F56455253494F4E3A312E30204D4143A4
:102DF00048494E455F545950453A507275736120A9
:102E00006933204D4B322E35204558545255444598
:102E1000525F434F554E543A3120555549443A304C
:102E2000303030303030302D303030302D303030A8
:102E3000302D303030302D30303030303030303098
:102E40003030300A004D31303920496E76616C697E
:102E50006420657874727564657220004D31303578
:102E600020496E76616C696420657874727564655A
:102E70007220004D31303420496E76616C696420D7
:102E80006578747275646572200055766F6C6E6536
:102E90006E612072656D656E69636B61004C6F6F6A
:102EA00073652070756C6C6579005A617665737412
:102EB0002066696C616D656E74004C6F616420669C
:102EC000696C616D656E74005A61766164656E69E6
:102ED0002066696C616D656E7475004C6F61646924
:102EE0006E672066696C616D656E7400436973740A
:102EF000656E69206261727679004C6F6164696EFB
:102F00006720636F6C6F72004C6576793A004C6590
:102F100066743A005679626572206A617A796B61EB
:102F20000053656C656374206C616E6775616765DD
:102F30000043657374696E6100456E676C69736800
:102F4000004B494C4C45442E2000496E76616C691B
:102F50006420657874727564657200566C6F7A745B
:102F6000652066696C616D656E7400496E7365728B
:102F7000742066696C616D656E74005469736B2EA4
:102F80002076656E743A005072696E742046414E28
:102F90003A2000547279736B2E2076656E743A0075
:102FA0004E6F7A7A6C652046414E3A0045787472CD
:102FB0007564657220696E666F00207A2034002087
:102FC0006F662034005A6C657073756A6920707280
:102FD00065736E6F7374206B616C69627261636E8E
:102FE00069686F20626F647500496D70726F7669F1
:102FF0006E67206265642063616C696272617469E6
:103000006F6E20706F696E74004B616C69627275CF
:103010006A69205A0043616C6962726174696E6703
:10302000205A004B616C696272616365204F4B00EE
:1030300043616C6962726174696F6E20646F6E6562
:10304000004B616C6962726F766174205A00436153
:103050006C696272617465205A005A61687269769F
:10306000616E69204F4B2E0048656174696E672060
:10307000646F6E652E005A6168726976616E6900D0
:1030800048656174696E67005641524F56414E491A
:103090003A204E657A6E616D612C206E65706F64AA
:1030A000706F726F76616E61207665727A652066E8
:1030B00069726D776172652E20506F757A697469D7
:1030C000206E6120766C6173746E69206E65626536
:1030D0007A7065636921005741524E494E473A2044
:1030E0005468697320697320616E20756E6F66661F
:1030F000696369616C2C20756E737570706F727482
:103100006564206275696C642E2055736520617456
:1031100020796F7572206F776E207269736B210052
:1031200043485942413A2046696C616D656E74208E
:1031300073656E7A6F72206E6572656167756A6518
:103140002C207A6B6F6E74726F6C756A7465207A5E
:1031500061706F6A656E692E004552524F523A2077
:1031600046696C616D656E742073656E736F722055
:103170006973206E6F7420726573706F6E64696E10
:10318000672C20706C6561736520636865636B20D4
:10319000636F6E6E656374696F6E2E00462E2061DC
:1031A00075746F7A61762E205B7A61705D00462EB1
:1031B000206175746F6C6F616420205B6F6E5D00C1
:1031C000462E206175746F7A61762E205B76797059
:1031D0005D00462E206175746F6C6F6164205B6FBB
:1031E00066665D00462E206175746F7A61762E20CA
:1031F0005B4E2F415D00462E206175746F6C6F61D0
:1032000064205B4E2F415D0046696C2E2073656E15
:103210007A6F72205B7A61705D0046696C2E207354
:10322000656E736F7220205B6F6E5D0046696C2E59
:103230002073656E7A6F72205B7679705D004669E7
:103240006C2E2073656E736F72205B6F66665D0017
:1032500046696C2E2073656E7A6F72205B4E2F412B
:103260005D0046696C2E2073656E736F72205B4E35
:103270002F415D002046726565204D656D6F727946
:103280003A20005469736B61726E61206E656279D9
:103290006C61206A65737465207A6B616C69627217
:1032A0006F76616E612E20506F73747570756A74DD
:1032B000652070726F73696D20706F646C65206D2E
:1032C000616E75616C752C206B617069746F6C61D7
:1032D000205A6163696E616D652C206F647374613F
:1032E00076656320506F73747570206B616C6962D2
:1032F000726163652E005072696E74657220686138
:1033000073206E6F74206265656E2063616C696204
:103310007261746564207965742E20506C656173E8
:103320006520666F6C6C6F7720746865206D616EC8
:1033300075616C2C206368617074657220466972D7
:1033400073742073746570732C2073656374696F74
:103350006E2043616C6962726174696F6E20666C85
:103360006F772E00507275746F6B00466C6F77002C
:10337000446F6B6F6E636F76616E6920706F6879F2
:1033800062750046696E697368696E67206D6F7655
:10339000656D656E747300207A203400206F66209E
:1033A0003400486C6564616D206B616C69627261A8
:1033B000636E6920626F6420706F646C6F7A6B79E2
:1033C00000536561726368696E672062656420639B
:1033D000616C6962726174696F6E20706F696E747E
:1033E0000049746572616365200049746572617497
:1033F000696F6E2000446F6E6520736176696E6739
:103400002066696C652E00446F6E65207072696E6F
:1034100074696E672066696C6500536F75626F72C0
:10342000206E656B6F6D706C65746E692E20506FC9
:103430006B7261636F7661743F0046696C652069E9
:103440006E636F6D706C6574652E20436F6E74696A
:103450006E756520616E797761793F004E656B749A
:1034600065726520736F75626F7279206E65627523
:10347000646F7520736574726964656E792E204D72
:103480006178696D616C6E6920706F63657420731B
:103490006F75626F72752070726F207365747269D8
:1034A00064656E69206A65203130302E00536F6D7F
:1034B000652066696C65732077696C6C206E6F742B
:1034C00020626520736F727465642E204D61782EC2
:1034D000204E6F2E206F662066696C657320696EC2
:1034E000203120666F6C64657220666F7220736F86
:1034F0007274696E67206973203130302E00536515
:103500006E7A6F722066696C616D656E74750046C7
:10351000696C616D656E742073656E736F720046C1
:10352000696C616D656E74207679746C6163656E2B
:1035300020612073707261766E65206261727679A7
:103540003F0046696C616D656E74206578747275B4
:1035500064696E672026207769746820636F7272D1
:1035600065637420636F6C6F723F0056796D656E92
:1035700069742066696C616D656E74004368616E84
:1035800067652066696C616D656E74005279636869
:103590006C6F73742076656E742E0046616E2073B6
:1035A00070656564004B6F6E74722E2076656E7464
:1035B0002E5B7A61705D0046616E7320636865639F
:1035C0006B2020205B6F6E5D004B6F6E74722E203F
:1035D00076656E742E5B7679705D0046616E732041
:1035E000636865636B20205B6F66665D00656E7166
:1035F0007565696E6720220045787472756465721E
:10360000002045787465726E616C20526573657434
:10361000005072696E7465722073746F70706564A7
:103620002064756520746F206572726F72732E202E
:1036300046697820746865206572726F7220616EC9
:103640006420757365204D39393920746F20726597
:1036500073746172742E202854656D706572617484
:103660007572652069732072657365742E205365C9
:103670007420697420616674657220726573746168
:103680007274696E6729004E6F204C696E65204E1A
:10369000756D626572207769746820636865636B15
:1036A00073756D2C204C617374204C696E653A20E3
:1036B000004E6F20436865636B73756D2077697486
:1036C00068206C696E65206E756D6265722C204C89
:1036D000617374204C696E653A200020746F6F200E
:1036E0006C6F6E6720657874727573696F6E207089
:1036F000726576656E746564004C696E65204E7502
:103700006D626572206973206E6F74204C617374F2
:10371000204C696E65204E756D6265722B312C20D0
:103720004C617374204C696E653A20005072696E6A
:103730007465722068616C7465642E206B696C6CB2
:1037400028292063616C6C6564210020636F6C64C0
:1037500020657874727573696F6E20707265766516
:103760006E74656400636865636B73756D206D6965
:10377000736D617463682C204C617374204C696EA6
:10378000653A200043485942413A004552524F524F
:103790003A00456E642066696C65206C697374003C
:1037A0006F70656E00545249474745524544006565
:1037B0006E6473746F7073206869743A2000536C80
:1037C0006565702E2E2E005679706E6F7574206DA3
:1037D0006F746F72790044697361626C65207374F1
:1037E000657070657273004E616872616E6F2076ED
:1037F0007963686F7A69206E6173746176656E694A
:103800000044656661756C742073657474696E67D5
:1038100073206C6F6164656400446174756D3A0077
:10382000446174653A00506F757A6520616B7475F8
:10383000616C6E690043757272656E740020436F2F
:10384000756E7420583A200056796D656E61206F50
:103850006B3F004368616E67656420636F727265D9
:1038600063746C793F005A63686C616469740043E7
:103870006F6F6C646F776E0050726F207573706538
:10388000736E6F75206B616C696272616369206F22
:10389000636973746574652070726F73696D2074E9
:1038A00069736B6F766F7520747279736B752E20E8
:1038B000506F74767264746520746C616369746BA4
:1038C000656D2E00506C6561736520636C65616E7B
:1038D00020746865206E6F7A7A6C6520666F72203E
:1038E00063616C6962726174696F6E2E20436C69EA
:1038F000636B207768656E20646F6E652E00446F81
:103900006A656C79206F6261205A20766F7A696BE4
:1039100079206B7E686F726E696D7520646F72615D
:103920007A753F00417265206C65667420616E6433
:10393000207269676874205A7E6361727269616778
:10394000657320616C6C2075703F00204C6173744E
:1039500020557064617465643A200056796265721E
:1039600074652065787472756465723A0043686F97
:103970006F73652065787472756465723A00507271
:103980006F73696D206F7465767265746520696404
:103990006C65722061206D616E75616C6E65206F63
:1039A00064737472616E74652066696C616D656EB6
:1039B000742E00506C65617365206F70656E2069B0
:1039C000646C657220616E642072656D6F7665202F
:1039D00066696C616D656E74206D616E75616C6C8D
:1039E000792E005A6D656E612075737065736E6116
:1039F00021004368616E6765207375636365737347
:103A000021005469736B207A205344005072696E10
:103A1000742066726F6D205344005465706C6F742F
:103A20002E206B616C6962726163650054656D7014
:103A30002E2063616C6962726174696F6E005A6BEB
:103A4000616C6962726F7661740043616C69627265
:103A50006174650052657365742058595A206B6112
:103A60006C6962722E0052657365742058595A2031
:103A700063616C6962722E004B616C696272616392
:103A8000652058595A0043616C69627261746520FF
:103A900058595A002042726F776E206F7574205209
:103AA0006573657400426567696E2066696C6520A0
:103AB0006C697374004B616C696272616365205854
:103AC000595A206E65707265736E612E204C657652
:103AD0007920707265646E6920626F64206D6F6317
:103AE000207670726564752E0058595A2063616C97
:103AF0006962726174696F6E20636F6D70726F6D51
:103B0000697365642E204C6566742066726F6E74EE
:103B10002063616C6962726174696F6E20706F6995
:103B20006E74206E6F7420726561636861626C658B
:103B30002E004B616C6962726163652058595A208E
:103B40006E65707265736E612E20507265646E6969
:103B5000206B616C69627261636E6920626F647967
:103B6000206D6F63207670726564752E0058595A07
:103B70002063616C6962726174696F6E20636F6D3E
:103B800070726F6D697365642E2046726F6E74205B
:103B900063616C6962726174696F6E20706F696EC7
:103BA0007473206E6F7420726561636861626C6506
:103BB0002E004B616C6962726163652058595A200E
:103BC0007620706F7261646B752E20582F59206FAC
:103BD0007379206D69726E65207A6B6F73656E659F
:103BE0002E20446F627261207072616365210058FB
:103BF000595A2063616C6962726174696F6E2061E9
:103C00006C6C2072696768742E20582F5920617877
:103C100065732061726520736C696768746C7920C4
:103C2000736B657765642E20476F6F64206A6F62DF
:103C300021004B616C6962726163652058595A209A
:103C40007620706F7261646B752E205A6B6F73658E
:103C50006E692062756465206175746F6D61746949
:103C6000636B79207679726F766E616E6F207072F9
:103C700069207469736B752E0058595A2063616C02
:103C80006962726174696F6E20616C6C2072696721
:103C900068742E20536B65772077696C6C206265A1
:103CA00020636F72726563746564206175746F6DF3
:103CB00061746963616C6C792E004B616C6962722E
:103CC0006163652058595A2073656C68616C612E78
:103CD000204B616C69627261636E6920626F64205F
:103CE000706F646C6F7A6B79206E656E616C657A4B
:103CF000656E2E0058595A2063616C696272617456
:103D0000696F6E206661696C65642E20426564206F
:103D100063616C6962726174696F6E20706F696E45
:103D20007420776173206E6F7420666F756E642ED9
:103D3000004B616C6962726163652058595A207644
:103D400020706F7261646B752E20582F59206F732D
:103D500079206A736F75206B6F6C6D652E204772CA
:103D60006174756C756A69210058595A2063616CD9
:103D70006962726174696F6E206F6B2E20582F59C3
:103D80002061786573206172652070657270656E60
:103D9000646963756C61722E20436F6E6772617423
:103DA000756C6174696F6E7321004B616C6962722E
:103DB0006163652058595A2073656C68616C612E87
:103DC000204E61686C65646E65746520646F206D5B
:103DD000616E75616C752E0058595A2063616C696B
:103DE00062726174696F6E206661696C65642E2011
:103DF000506C6561736520636F6E73756C742074AD
:103E00006865206D616E75616C2E004B616C696236
:103E1000726163652058595A2073656C68616C61E2
:103E20002E204C65767920707265646E6920626F11
:103E300064206D6F63207670726564752E205372F6
:103E40006F766E656A7465207469736B61726E75E6
:103E50002E0058595A2063616C6962726174696FEF
:103E60006E206661696C65642E204C656674206600
:103E7000726F6E742063616C6962726174696F6ED7
:103E800020706F696E74206E6F7420726561636854
:103E900061626C652E004B616C69627261636520C2
:103EA00058595A2073656C68616C612E2050726598
:103EB000646E69206B616C69627261636E69206215
:103EC0006F6479206D6F63207670726564752E2043
:103ED00053726F766E656A7465207469736B617274
:103EE0006E752E0058595A2063616C696272617454
:103EF000696F6E206661696C65642E2046726F6E14
:103F0000742063616C6962726174696F6E20706F96
:103F1000696E7473206E6F7420726561636861628C
:103F20006C652E004B616C696272616365205A207A
:103F300073656C68616C612E2053656E736F7220BF
:103F40006A65206F64706F6A656E79206E65626F56
:103F500020707265727573656E79206B6162656C35
:103F60002E2043656B616D206E61207265736574F0
:103F70002E00426564206C6576656C696E6720660C
:103F800061696C65642E2053656E736F722064697D
:103F900073636F6E6E6563746564206F7220636116
:103FA000626C652062726F6B656E2E20576169745A
:103FB000696E6720666F722072657365742E004BA0
:103FC000616C696272616365205A2073656C686117
:103FD0006C612E2053656E736F72206E6573657011
:103FE0006E756C2E205A6E6563697374656E612000
:103FF000747279736B613F2043656B616D206E61F4
:104000002072657365742E00426564206C65766568
:104010006C696E67206661696C65642E2053656EFD
:10402000736F72206469646E742074726967676567
:10403000722E20446562726973206F6E206E6F7AF3
:104040007A6C653F2057616974696E6720666F728C
:104050002072657365742E004B616C6962726163D6
:1040600065205A2073656C68616C612E2053656E03
:10407000736F72207365706E756C207072696C69F5
:1040800073207679736F6B6F2E2043656B616D20A3
:104090006E612072657365742E00426564206C65E4
:1040A00076656C696E67206661696C65642E205365
:1040B000656E736F722074726967676572656420DC
:1040C000746F6F20686967682E2057616974696E24
:1040D0006720666F722072657365742E005A61687E
:1040E000726976616E692062656400426564204889
:1040F000656174696E6700426564204F4B2E004213
:10410000656420646F6E650056707261766F205B27
:10411000756D5D00526967687420736964655B75CD
:104120006D5D00526573657400567A616475202078
:104130005B756D5D00526561722073696465205B1B
:10414000756D5D004B6F72656B636520706F646C9D
:104150006F7A6B7900426564206C6576656C2063CC
:104160006F727265637400566C65766F20205B75A4
:104170006D5D004C6566742073696465205B756DC8
:104180005D00567072656475205B756D5D004672EA
:104190006F6E7420736964655B756D5D0042656464
:1041A000004E656E69207A6B616C6962726F766130
:1041B0006E6120767A64616C656E6F7374207472C0
:1041C00079736B79206F64207469736B6F766520E7
:1041D000706F646C6F7A6B792E20506F737475708A
:1041E000756A74652070726F73696D20706F646C8E
:1041F00065206D616E75616C752C206B61706974E2
:104200006F6C61205A6163696E616D652C206F640B
:10421000737461766563204E6173746176656E694F
:10422000207072766E69207672737476792E0044EF
:10423000697374616E6365206265747765656E206D
:10424000746970206F6620746865206E6F7A7A6C6E
:104250006520616E642074686520626564207375F2
:10426000726661636520686173206E6F7420626599
:10427000656E20736574207965742E20506C6561BD
:10428000736520666F6C6C6F7720746865206D6154
:104290006E75616C2C20636861707465722046696C
:1042A0007273742073746570732C20736563746902
:1042B0006F6E204669727374206C61796572206339
:1042C000616C6962726174696F6E2E00446F6C611B
:1042D00064656E69206F7379205A004C6976652099
:1042E00061646A757374205A0041646A75737469F5
:1042F0006E67205A004175746F20686F6D650041CC
:1043000075746F5A61766564656E692066696C2E96
:10431000004175746F4C6F61642066696C616D65F6
:104320006E74004175746F6D617469636B65207A9A
:1043300061766164656E692066696C616D656E7435
:104340007520646F737475706E6520706F757A6513
:1043500020707269207A61706E7574656D2066696F
:104360006C616D656E742073656E7A6F72752E2E3A
:104370002E004175746F6C6F6164696E67206669A9
:104380006C616D656E7420617661696C61626C65EB
:10439000206F6E6C79207768656E2066696C616D40
:1043A000656E742073656E736F7220697320747507
:1043B000726E6564206F6E2E2E2E004175746F6DC7
:1043C000617469636B65207A61766164656E6920EA
:1043D00066696C616D656E747520616B7469766E6B
:1043E000692C20737469736B6E65746520746C61DD
:1043F0006369746B6F206120766C6F7A74652066D8
:10440000696C616D656E742E2E2E004175746F6C33
:104410006F6164696E672066696C616D656E74209A
:104420006973206163746976652C206A75737420E2
:10443000707265737320746865206B6E6F622061A3
:104440006E6420696E736572742066696C616D6557
:104450006E742E2E2E00207C20417574686F723A87
:10446000200056736500416C6C0041637469766589
:104470002045787472756465723A2000AC0F9A0F0B
:10448000C20FCA0FD20FDB0FE30F0010EB0F191092
:1044900015101D1025103E102D1069104F10BF1063
:1044A00087101D11FD10A1114011AF120412A613A7
:1044B00063134C14F313FF149314AA155E153E16E0
:1044C000FB158F167B16FD16A316941745170218B9
:1044D000DE17371822185A184B18A51877183019F4
:1044E000D31890199719B119A719E519BD191A1AF6
:1044F000081A2B1A501A3C1A831A621AB41AA31AF1
:10450000D61AC41AE91A021BFC1A071B191B2B1B0B
:10451000841B721BA81B961BF51BBA1B421C2D1C6F
:104520005F1C571C731C6B1C891C7B1C941C9E1CE1
:10453000CE1CB21CF71CE91C1C1D0A1D3B1D2D1DA9
:10454000561D491D741D671DAA1D811DDE1DD51D2B
:10455000F61DE41D1A1E081E3E1E2C1E601E501E57
:104560006E1E8D1E7E1EAB1E9A1EC91EBA1EE81E32
:10457000D61E031FF91E1B1F0C1F321F281F3A1FB8
:104580005B1F4C1F751F661F841FA01F911FAE1F4E
:10459000B41FD81FC61FF11FE91F0420FA1F2320D4
:1045A0001120442033205F204D207D207120A02049
:1045B0008B20B120C220D220DB20F820E3201B2159
:1045C00009213F212D216321512187217521AA2114
:1045D0009921CE21BC21F221E02116220422282299
:1045E0003F2235224F224B225422782266229C22DF
:1045F0008A22AE22C022D322E922DB22F62208231D
:104600001C233A232C234823552363237123872318
:104610009223AF23A823C723B623E523D623FF2362
:10462000F4230C243E24152488246624BE24AD24BF
:10463000E124D024FE24F3241A250A253525272534
:10464000432589255825E725B225272612264E26FB
:104650003A266C26622674268B267C26BD26972653
:10466000F626DD260E274D27252782277227A42729
:104670009027CA27B827EA27DC270A28FA279D2887
:104680001628332936293A295229432964295D29D4
:104690007E296B29A3299229B829B529D029BB29BC
:1046A000FB29E029262A1B2A382A2D2A4A2A3F2AB2
:1046B000512AB02A5A2A672B0F2BD52BC82BDF2B58
:1046C000F82BF12B092C012C202C162C382C2C2CFF
:1046D000492C442C782C4F2CB82CA82CD62CC72C29
:1046E000DB2CF22C092D202D502D392D662D452E39
:1046F0005C2E732E9D2E8A2EBA2EAA2EDB2EC82E4D
:10470000FA2EEC2E0E2F082F212F142F392F312F98
:10471000412F4A2F6B2F5B2F872F7B2FA02F932F9B
:10472000AC2FBF2FBA2FE92FC52F153009303030ED
:1047300023304E30413068305A3080307630D730B8
:10474000883059312031AE319C31D231C031F6310F
:10475000E4311A3208323E322C3262325032743234
:10476000F63283326B336433833370339C33973345
:10477000C133A233EA33E133F53307343A341A3420
:10478000AD345C340F35FE3442351F357C356B3526
:104790009B358C35B735A535DB35C935ED35F83565
:1047A000013611368736B136DB36F9362C374B37C2
:1047B00065378B3784379237A037A537AF37BE3789
:1047C000D637C7370138E737203819383538263813
:1047D0003D38533848386F386638C438783824390B
:1047E000FE384B396D395B39B3397E39F239E339EB
:1047F0000C3A023A2C3A1A3A4A3A3E3A663A543A53
:10480000863A783A943AA53AE93AB53A6D3B323B62
:10481000EF3BB23B793C323CF43CBA3C693D313D24
:10482000D83DAA3D523E0B3EE43E963E723F243FA9
:104830000840BF3F9A405840EB40DD40FF40F74002
:1048400014410841234135412941554144417341B7
:1048500067418E4182419D412F42A141DB42CC42C2
:10486000E942F5421143FF42724323430B44BB43E9
:104870005644664462446A44457872656D652073A7
:1048800070616E206F6620746865205A2076616CB6
:10489000756573210043616C63756C6174696F6E3B
:1048A000206F6620746865206D616368696E65209D
:1048B000736B657720616E64206F66667365742024
:1048C0006661696C65642E00203C20005741524EA1
:1048D000494E473A2046726F6E7420706F696E744D
:1048E000206E6F7420726561636861626C652E2052
:1048F0005920636F6F7264696E6174653A00004994
:104900007465726174696F6E3A200000004041FF67
:10491000FFBF4000005C43FFFFBF4000005C43005E
:10492000004643000040410000464300004041FF74
:10493000FFBF400000E442FFFFBF4000005743FFBD
:10494000FFBF40000057430000CC420000E442009B
:1049500000CC42000040410000CC42000040410039
:104960000046430000E44200004643000057430075
:10497000004643062833D036C23E013F154132423D
:104980003B43F2443B45F24622473B48F2493B4A0F
:10499000F05898590C5A085B0C5C086110679B6EC4
:1049A0002271077208FF095A0D000EFF19045E08F4
:1049B00020642B6D322FFF45303A20005A3A2000F8
:1049C000593A2000583A20004D53312C4D53322093
:1049D00050696E730A005A00205A3A005900205953
:1049E0003A00580020583A0024F4D43050C38E20A6
:1049F000C2A24017828B7011127A910D816CD90A74
:104A0000A861E108C7586607615143061E4B5D0562
:104A1000C145A7041A411104093D980371393103B6
:104A20004036DB0265339102D4305402802E1D02E1
:104A3000632CEE01752AC501B028A0011027810161
:104A40008F2564012B244B01E0223401AC211F018E
:104A50008D200D01801FFC00841EED00971DDF00DE
:104A6000B81CD200E61BC600201BBC00641AB200B2
:104A7000B219A8000A19A0006A189900D11791006C
:104A800040178B00B516840031167E00B3157900EF
:104A90003A157300C7146F0058146A00EE136600CD
:104AA0008813630025135E00C7125B006C12570069
:104AB00015125400C111510070114F0021114B000B
:104AC000D61049008D1047004610440002104200E5
:104AD000C00F4000800F3E00420F3C00060F3B001D
:104AE000CB0E3800930E37005C0E3500270E3400D5
:104AF000F30D3200C10D3100900D3000600D2E001D
:104B0000320D2D00050D2C00D90C2B00AE0C290008
:104B1000850C29005C0C2700350C27000E0C2600A4
:104B2000E80B2400C40B2400A00B23007D0B230002
:104B30005A0B2100390B2100180B2000F80A1F0026
:104B4000D90A1E00BB0A1E009D0A1D00800A1D0016
:104B5000630A1C00470A1B002C0A1B00110A1A00DA
:104B6000F7091A00DD091900C4091900AB09190079
:104B7000920917007B091800630917004C091600F9
:104B800036091600200916000A091500F508150057
:104B9000E0081400CC081400B8081400A40814009D
:104BA000900813007D0812006B08130058081200CB
:104BB00046081200340811002308110012081100E1
:104BC00001081100F0071000E0071000D0071000E6
:104BD000C0071000B0070F00A107100091070E00DA
:104BE00083070F0074070F0065070E0057070E00BC
:104BF00049070E003B070D002E070E0020070D0091
:104C000013070D0006070D00F9060C00ED060D0058
:104C1000E0060C00D4060C00C8060C00BC060C0014
:104C2000B0060C00A4060B0099060C008D060B00C4
:104C300082060B0077060B006C060B0061060A006B
:104C400057060B004C060A0042060A0038060A0006
:104C50002E060A0024060A001A060A001006090099
:104C600007060A00FD050900F4050900EB05090027
:104C7000E2050900D9050900D0050900C7050900AA
:104C8000BE050900B5050800AD050800A505090029
:104C90009C050800940508008C05080084050800A0
:104CA0007C050800740508006C0507006505080010
:104CB0005D050700560508004E050700470507007B
:104CC0004005080038050700310507002A050700E0
:104CD000230507001C050600160507000F05070041
:104CE0000805060002050700FB040600F50407009E
:104CF000EE040600E8040600E2040700DB040600F8
:104D0000D5040600CF040600C9040600C30406004B
:104D1000BD040600B7040600B1040500AC0406009B
:104D2000A6040600A00405009B04060095040500E7
:104D3000900406008A04050085040500800406002E
:104D40007A04050075040500700405006B04050075
:104D500066040500610405005C04050057040500B5
:104D6000520405004D0405004804050043040500F5
:104D70003E0404003A040500350405003004040034
:104D80002C04050027040400230405001E0404006D
:104D90001A04040016040500110404000D040400A4
:104DA000090405000404040000040400FC030400DA
:104DB000F8030400F4030400F0030400EC0304000F
:104DC000E8030400E4030400E0030400DC0304003F
:104DD000D8030400D4030400D0030400CC0304006F
:104DE000C8030300C503030024F404D9201BC40C2A
:104DF0005C0E9804C4095F0265077101F405F900AF
:104E0000FB04B30048048700C10369005803550040
:104E100003034500BE023A008402310053022A0017
:104E20002902250004022000E4011C00C801190029
:104E3000AF011700980114008401130071011000E4
:104E40006101100051010E0043010D0036010B00FD
:104E50002B010B0020010B00150109000C010900BA
:104E600003010800FB000800F3000800EB00070046
:104E7000E4000600DE000600D8000600D2000600AE
:104E8000CC000500C7000500C2000500BD000400FD
:104E9000B9000400B5000400B1000400AD00040036
:104EA000A9000400A5000300A20003009F00040065
:104EB0009B0003009800030095000200930003008C
:104EC000900003008D0002008B00030088000200A8
:104ED0008600020084000300810002007F000200BF
:104EE0007D0002007B0002007900020077000100D3
:104EF00076000200740002007200010071000200DE
:104F00006F0002006D0001006C0002006A000100E9
:104F100069000200670001006600010065000100F1
:104F200064000200620001006100010060000100F5
:104F30005F0002005D0001005C0001005B000100F9
:104F40005A000100590001005800010057000100FB
:104F500056000100550001005400010053000000FC
:104F600053000100520001005100010050000100F7
:104F70004F0001004E0000004E0001004D000100F6
:104F80004C0001004B0000004B0001004A000100F2
:104F900049000100480000004800010047000100EE
:104FA00046000000460001004500000045000100E9
:104FB00044000100430000004300010042000000E3
:104FC00042000100410000004100010040000100DA
:104FD0003F0000003F0001003E0000003E000100D5
:104FE0003D0000003D0001003C0000003C000000CE
:104FF0003C0001003B0000003B0001003A000000C3
:105000003A000100390000003900010038000000BA
:1050100038000000380001003700000037000100B0
:1050200036000000360000003600010035000000A8
:10503000350000003500010034000000340000009D
:105040003400010033000000330000003300010091
:105050003200000032000000320001003100000088
:10506000310000003100010030000000300000007D
:10507000300001002F0000002F0000002F00000072
:105080002F0001002E0000002E0000002E00010065
:105090002D0000002D0000002D0000002D0001005B
:1050A0002C0000002C0000002C0000002C0001004F
:1050B0002B0000002B0000002B0000002B00010043
:1050C0002A0000002A0000002A0000002A00010037
:1050D000290000002900000029000000290000002C
:1050E000290001002800000028000000280000001E
:1050F0002800000028000100270000002700000011
:105100002700000027000000270001002600000003
:1051100026000000260000002600000026000100F6
:1051200025000000250000002500000025000000EB
:1051300025000000250001002400000024000000DC
:1051400024000000240000002400010023000000CF
:1051500023000000230000002300000023000000C3
:1051600023000000230001002200000022000000B4
:1051700022000000220000002200000022000100A6
:10518000210000002100000021000000210000009B
:10519000210000002100000021000100200000008B
:1051A000200000002000000020000000200000007F
:1051B0002000000020000000200001001F0000006F
:1051C0001F0000001F0000001F0000001F00000063
:1051D0001F0000001F0001001E0000001E00000054
:1051E0001E0000001E0000004572723A204D494E1C
:1051F00054454D50204245440054656D70657261C0
:1052000074757265206865617465642062656420E8
:105210007377697463686564206F66662E204D49F4
:105220004E54454D502074726967676572656420FD
:1052300021004572723A204D415854454D5020424C
:1052400045440054656D70657261747572652068BF
:10525000656174656420626564207377697463684E
:105260006564206F66662E204D415854454D502090
:105270007472696767657265642021004572723ACD
:10528000204D494E54454D50003A20457874727572
:10529000646572207377697463686564206F6666FD
:1052A0002E204D494E54454D5020747269676765F4
:1052B0007265642021004572723A204D4158544570
:1052C0004D50003A2045787472756465722073778A
:1052D000697463686564206F66662E204D4158547A
:1052E000454D5020747269676765726564202100BE
:1052F00020484F54454E4420544845524D414C207F
:1053000052554E4157415900204845415442454469
:1053100020544845524D414C2052554E4157415919
:1053200000544845524D414C2052554E4157415929
:105330000042454420544845524D414C2052554E60
:10534000415741590020544845524D414C20525537
:105350004E4157415920282050524548454154203C
:10536000484F54454E44290020544845524D414C25
:105370002052554E4157415920282050524548450A
:105380004154204845415442454429005052454823
:10539000454154204552524F5200424544205052FC
:1053A0004548454154204552524F520050494420EF
:1053B0004175746F74756E652066696E6973686592
:1053C00064212050757420746865206C61737420AA
:1053D0004B702C204B6920616E64204B6420636FFE
:1053E0006E7374616E74732066726F6D2061626F8C
:1053F000766520696E746F20436F6E66696775729B
:105400006174696F6E2E6800504944204175746F55
:1054100074756E65206661696C6564212074696DC0
:10542000656F75740020403A00543A00423A0050CB
:105430004944204175746F74756E65206661696CAE
:105440006564212054656D706572617475726520A4
:10545000746F6F206869676800204B643A200020F1
:105460004B693A2000204B703A200020436C617356
:105470007369632050494420002054753A2000206D
:105480004B753A2000206D61783A2000206D696EDE
:105490003A200020643A200020626961733A2000BB
:1054A0001000C90210012C014001220170011801F5
:1054B000B0010E01F00104015002FA00B002F00048
:1054C0003003E600D003DC009004D2007005C80071
:1054D000A006BE000008B400B009AA00D00BA000CE
:1054E000600E960060118C00001582002019780073
:1054F000C01D6E00A0226400B0275A00902C5000FE
:1055000000314600E0343C0010383200903A280068
:10551000603C1E00A03D1400803E0A00203F0000B9
:1055200070012C0190012701B0012201C0011D0171
:10553000F00118011002130130020E01600209018E
:1055400090020401C002FF000003FA004003F500CE
:105550008003F000D003EB002004E6007004E100BB
:10556000E004DC004005D700C005D2004006CD00B5
:10557000D006C8008007C3003008BE00F008B9009C
:10558000C009B400B00AAF00B00BAA00D00CA5004F
:10559000000EA000500F9B00C0109600501291000A
:1055A00000148C00C0158700B0178200B0197D0070
:1055B000D01B7800001E730040206E00902269000E
:1055C000F024640040275F0090295A00E02B55002A
:1055D000102E500020304B0010324600E0334100C6
:1055E00090353C001037370070383200A0392D005C
:1055F000B03A2800A03B2300603C1E00103D19007B
:10560000903D1400103E0F00703E0A00C03E0500A1
:10561000003F0000436F6E74696E75652077697492
:105620006820616E6F7468657220626F7764656E62
:105630003F0053746174653A2000473736004D349B
:1056400035205A004D3435004738300020003E00E8
:105650003E0020003E003E003E003E0020003E0096
:105660003E00200000002D2D2D2D2D2D2D2D2D2D1A
:105670002D2D2D2D2D2D2D2D2D2D004E2F41004E5C
:105680002F41006D6D00004D373031004D37303205
:1056900000496E76616C6964205049442063616CF6
:1056A0002E20726573756C74732E204E6F74207388
:1056B000746F72656420746F20454550524F4D2EB3
:1056C000004D353030004731205A313520463135D4
:1056D00030300047393100473120583530205931BA
:1056E00039302045302046373030300047393000DF
:1056F0004D373032004D3730322043004D37303295
:105700002055004D373032004731205A3135204680
:10571000313530300047393100473120583530209D
:1057200059313930204530204637303030004D383F
:105730003300473930004D3834004D313034205378
:1057400030004D383400473120583130205931383D
:1057500030204634303030004731205A3130204636
:10576000313330302E303030004D31343020533032
:10577000004D313034205330004D31303700473147
:1057800020452D302E303735303020463231303004
:105790002E303030303000473120583530205935E8
:1057A000352045332E3632373733004731205832D3
:1057B0003030205935352045302E343933383600D5
:1057C00047312058323030205937352045332E3676
:1057D000323737330047312058353020593735209C
:1057E00045302E3439333836004731205835302093
:1057F0005939352045332E3632373733004731207B
:1058000058323030205939352045302E343933382C
:10581000360047312058323030205931313520455B
:10582000332E363237373300473120583530205940
:105830003131352045302E34393338360047312068
:1058400058353020593133352045332E36323737ED
:10585000330047312058323030205931333520451C
:10586000302E363631373400473120583230302030
:10587000593135352045322E3632373733004731EE
:1058800020583130302059313535204532004731EC
:105890002058373520593135352045322E350047CF
:1058A00031204631303830004731205835302059CA
:1058B000313535004731204634303030004D3230FC
:1058C00034205331303030004731205A302E3135BA
:1058D000302046373230302E3030300047312045CE
:1058E0002D312E35303030302046323130302E30B0
:1058F00030303030004D38330047393000473231D6
:10590000004739322045302E3000473120583130A1
:10591000302E30204531322E352046313030302E79
:1059200030004731205836302E302045392E302077
:1059300046313030302E30004739322045302E305D
:105940000047323800473837004D31303920533264
:105950003135004D31393020533630004D3134303F
:1059600020533630004D3130342053323135004D24
:1059700031303700473930004731204531004D384C
:1059800032004731204531004D3833004D3130363B
:1059900020532564004D32323020532564003A20D4
:1059A0000020202020202020202020202020202017
:1059B0002020202000203A2000202020202020200D
:1059C00020202020202020202020202020002020F7
:1059D00020202020202020202020200025730020AF
:1059E00020002D2D3A2D2D002000200020004C00FD
:1059F0002020002046002D2D2D003E5553420053FF
:105A000044002D2D002520202020200020200020D3
:105A100020000120002020202D2D2D200020205AA4
:105A2000002020000120004D36303000464C455803
:105A3000202D20203234302F3530005050202020AF
:105A40002D20203235342F3130300048495053203A
:105A50002D20203232302F3130300041425320206F
:105A60002D20203235352F31303000504554202044
:105A70002D20203233302F383500504C4120202D3E
:105A800020203231352F3630006661726D20202D96
:105A900020203235302F3430004D3234004D323337
:105AA00020257300052E2E00580059005A00457815
:105AB00074727564657200473939004469736162B4
:105AC0006C65206661726D206D6F64653F0044698E
:105AD0007361626C65206661726D206D6F64650034
:105AE0004661726D206E756D626572004D383400CE
:105AF00063757272656E745F706F733A006375726E
:105B000072656E745F706F735F696E69743A004D91
:105B10003834004731205A31350047323820570099
:105B20005A30005A3100593000593100583000586D
:105B30003100456E642073746F707320646961670F
:105B4000004D3434004732382057001B5B303B3166
:105B50004842656C74207374617475731B5B313BD0
:105B60003248582025641B5B323B3248592025645B
:105B7000001B5B323B314850494E44413A202020C3
:105B80002025642563001B5B303B31484E6F7A7AD9
:105B90006C653A202020256425631B5B313B31482E
:105BA0004265643A20202020202025642563001BC4
:105BB0005B313B31485057523A202020202020258D
:105BC000642E2530316456002D2D2D2D2D2D2D2D9B
:105BD0002D2D2D2D00466C6173684169722049504E
:105BE00020416464723A002D2D2D2D2D2D2D2D2D4B
:105BF0002D2D2D00466562202031203230313800B5
:105C00002D2D2D2D2D2D2D2D2D2D2D2D00453344BC
:105C1000763666756C6C0052414D426F31336100CF
:105C2000315F37356D6D5F4D4B3235002D2D2D2D8C
:105C30002D2D2D2D2D2D2D2D00207265706F2050B6
:105C40007275736133442F4D4B330020332E312E48
:105C5000312D5243352D313531004669726D7761F2
:105C600072653A0025642E25642E25642E25640075
:105C70004661726D206E756D626572000072630020
:105C80006265746100616C706861006465760050E3
:105C9000525553413344465700332E312E312D5245
:105CA00043350000000A0B02090C0D0E080703041F
:105CB00001000000000000000000000000000000E3
:105CC00000000000000000000000000000000012C2
:105CD00011100000000000000000000000000000A3
:105CE00000000000000000000000000000000000B4
:105CF0000000000000000000000102102020080841
:105D0000102040102040800201020108040201011D
:105D10000204081020408080402010080402018006
:105D2000040201804020100804020108040201015D
:105D30000204081020408001020408102040801056
:105D40000804088010204004408010204004800592
:105D5000050505070508080808020202020A0A08E4
:105D6000080404040401010101010101010303030A
:105D70000303030303040707070C0C0C0C0C0C0CA7
:105D80000C0202020206060606060606060B0B0BAE
:105D90000B0B0B0B0B07070A0A0A0A0A0A05050573
:105DA0000404040808000020002300260029002C19
:105DB000002F00320000010000030106010901006C
:105DC000002200250028002B002E003100340002A4
:105DD000010000050108010B01000021002400273B
:105DE000002A002D003000330001010000040107EB
:105DF000010A01024E414E494E495459494E46CD81
:105E0000CCCC3D0AD7233C17B7D13877CC2B329571
:105E100095E6241FB14F0A000020410000C842004F
:105E2000401C4620BCBE4CCA1B0E5AAEC59D740019
:105E3000407A10F35A00A0724E18090010A5D4E859
:105E40000000E87648170000E40B54020000CA9AEC
:105E50003B000000E1F5050000809698000000403E
:105E6000420F000000A08601000000102700000083
:105E700000E803000000006400000000000A0000C9
:105E80000000000100000000002C76D888DC674F7D
:105E90000823DFC1DFAE59E1B1B796E5E3E453C6AD
:105EA0003AE651997696E8E6C28426EB898C9B62A5
:105EB000ED407C6FFCEFBC9C9F40F2BAA56FA5F44F
:105EC00090055A2AF75C936B6CF9676DC11BFCE077
:105ED000E40D47FEF520E6B500D0ED902E030094CA
:105EE0003577050080841E080000204E0A0000005F
:105EF000C80C333333330F986E12831141EF8D2169
:105F000014893BE65516CFFEE6DB18D1844B381BCF
:105F1000F77C1D901DA4BBE424203284725E228194
:105F200000C9F124ECA1E53D2700349425BCC3ED64
:105F30005801659411241FBECFEFD1E2DEBFCDBF63
:105F400000E00CBF17E0A0E0B2E0ECE7F7E603E00A
:105F50000BBF02C007900D92AC31B107D9F729E110
:105F6000ACE1B7E001C01D92A635B207E1F71FE52D
:105F7000C2E3DFE500E006C022970109FE010BBF86
:105F80000F9472A9CA32D10780E00807A9F70F94CD
:105F90004AA30D94ACB30C940000109249191092CE
:105FA00038194091391950913A19EBE3F9E180E041
:105FB00090E061E070E09B01082E02C0220F331FC9
:105FC0000A94E2F724233523232B11F41182108243
:105FD000019632968730910571F7089581E593E037
:105FE0000F94B7AD10923A1910923919EAE7F0E020
:105FF000808187608083ACE7B0E08C9180648C9373
:106000008081806880838FE580937E0082E080932A
:106010007D00C3CF282F2F7090917B0083FF02C09B
:10602000986001C0977F90937B0090917C00822FB5
:106030008770987F892B80937C000895982F21E0AA
:1060400030E080E0A9014F755270452B29F04FEFE9
:10605000490F911102C00895492F220F331F8F5FFE
:10606000803111F0942FEECF0895CF93C09149194C
:10607000C7FF36C0CF70EC2FF0E021E030E00C2EEF
:1060800002C0220F331F0A94E2F740913919509150
:106090003A1924233523232B71F440917800509131
:1060A0007900EE0FFF1FE55CF64E20813181240F51
:1060B000351F31832083C73010F4CF5F0BC0809130
:1060C00038198F5F80933819803118F00F94CB21E5
:1060D00064DFC0E08C2FB2DF9DDFC09349190AC096
:1060E00080917A00806480937A0080914919806859
:1060F00080934919CF9108959091A107911107C0FC
:106100009091C00095FFFCCF8093C6000895913018
:1061100031F49091C80095FFFCCF8093CE00089594
:10612000CF92DF92EF92FF920F931F93CF93DF9363
:106130008C01D42EC62FD72FD60EDC1671F1F801A4
:10614000E080F180C990C7010F945DB0C816F1F0EE
:106150006C2DC7010F948DB0C7010F945DB08C15E5
:10616000A9F0E3E3F7E08491EF01882329F0C4DF8D
:106170002196FE018491F9CF8AE0DF91CF911F91A2
:106180000F91FF90EF90DF90CF90B6CFF801808114
:106190009181019691838083D0CFDF91CF911F9120
:1061A0000F91FF90EF90DF90CF900895EF92FF92C4
:1061B0000F931F93CF93DF931F92CDB7DEB78C0160
:1061C0007B01460FF8018081918149830F945DB076
:1061D000F70181937F01F80180819181019691837C
:1061E000808349814E11EECF0F90DF91CF911F91A7
:1061F0000F91FF90EF9008950F931F93CF93DF932C
:10620000CDB7DEB72C970FB6F894DEBF0FBECDBF6B
:106210008C0140E350E360E370E04D835E836F8365
:1062200078879C878B8744E0BE016B5F7F4FCE01F0
:106230000B9676DF40E160EF76E1CE010B9670DFE2
:1062400040E160E077E1CE010B966ADF40E160EE6D
:1062500076E1CE010B9664DF44E068ED76E1CE0195
:106260000B965EDF44E064ED76E1CE010B9658DFDD
:1062700044E06CED76E1CE010B9652DF44E060EC39
:1062800076E1CE010B964CDF44E060E177E1CE0190
:106290000B9646DF44E064EC76E1CE010B9640DFDE
:1062A00044E068EC76E1CE010B963ADF44E06CEC1A
:1062B00076E1CE010B9634DF44E060ED76E1CE016D
:1062C0000B962EDF4CE062E778E0CE010B9628DFDC
:1062D00044E06BE678E0CE010B9622DF44E06AEA08
:1062E00072E0CE010B961CDF44E066EA72E0CE015C
:1062F0000B9616DF44E062EA72E0CE010B9610DFE7
:1063000044E06AE972E0CE010B960ADF44E066E9F8
:1063100072E0CE010B9604DF44E062E972E0CE0148
:106320000B96FEDE80E290E09A87898742E0BE010C
:10633000675F7F4FCE010B96F3DE41E067E678E0C2
:10634000CE010B96EDDE44E066E272E0CE010B96E4
:10635000E7DE44E06EE172E0CE010B96E1DE44E060
:1063600062E678E0CE010B96DBDE44E06EE578E095
:10637000CE010B96D5DE44E06AE172E0CE010B96C9
:10638000CFDE41E06EE878E0CE010B96C9DE44E056
:1063900066E472E0CE010B96C3DE46E552E360E0B0
:1063A00070E049835A836B837C831C870B8744E0AE
:1063B000BE016F5F7F4FCE010B96B2DEE3EFFBE0D5
:1063C00084918F01882331F097DE0F5F1F4FF80112
:1063D0008491F8CFE3E2F7E084918F01882331F0D4
:1063E0008BDE0F5F1F4FF8018491F8CF8AE084DEC7
:1063F0002C960FB6F894DEBF0FBECDBFDF91CF91C4
:106400001F910F9108950F931F93CF93DF93C3EFC5
:10641000DBE0FE0184918E01882331F06DDE0F5F99
:106420001F4FF8018491F8CFE3E1F7E084918F01E9
:10643000882331F061DE0F5F1F4FF8018491F8CFA0
:106440008AE05ADEFE01849103EF1BE0882331F0DD
:1064500053DE0F5F1F4FF8018491F8CF4091F01683
:106460005091F1166091F2167091F3168BE097E05F
:106470000E94E0434091F4165091F5166091F61693
:106480007091F71688E097E00E94E0434091F8167B
:106490005091F9166091FA167091FB1685E097E01D
:1064A0000E94E0434091FC165091FD166091FE164B
:1064B0007091FF1682E097E00E94E0438AE01CDEC4
:1064C000FE01849103EF1BE0882331F015DE0F5F9E
:1064D0001F4FF8018491F8CFE8EEF6E084918F0128
:1064E000882331F009DE0F5F1F4FF8018491F8CF48
:1064F0008AE002DEFE01849103EF1BE0882331F085
:10650000FBDD0F5F1F4FF8018491F8CF409100171A
:106510005091011760910217709103178FED96E06B
:106520000E94E043409104175091051760910617AF
:10653000709107178CED96E00E94E0434091081798
:106540005091091760910A1770910B1789ED96E029
:106550000E94E04340910C1750910D1760910E1767
:1065600070910F1786ED96E00E94E0438AE0C4DD4B
:10657000FE01849103EF1BE0882331F0BDDD0F5F46
:106580001F4FF8018491F8CFE8EBF6E084918F017A
:10659000882331F0B1DD0F5F1F4FF8018491F8CFF0
:1065A0008AE0AADDFE01849103EF1BE0882331F02D
:1065B000A3DD0F5F1F4FF8018491F8CF4091E016E3
:1065C0005091E1166091E2167091E3168FEA96E021
:1065D0000E9408444091E4165091E5166091E61639
:1065E0007091E7168CEA96E00E9408444091E81604
:1065F0005091E9166091EA167091EB1689EA96E0DF
:106600000E9408444091EC165091ED166091EE16F0
:106610007091EF1686EA96E00E9408448AE06CDDED
:10662000FE01849103EF1BE0882331F065DD0F5FED
:106630001F4FF8018491F8CFE1E7F6E084918F01D4
:10664000882331F059DD0F5F1F4FF8018491F8CF97
:106650008AE052DDFE01849103EF1BE0882331F0D4
:106660004BDD0F5F1F4FF8018491F8CF4091D81692
:106670005091D9166091DA167091DB1688E696E093
:106680000E94E0434091D4165091D5166091D616E1
:106690007091D71685E696E00E94E0438AE02CDDF3
:1066A000FE01849103EF1BE0882331F025DD0F5FAD
:1066B0001F4FF8018491F8CFE2EBF5E084918F0150
:1066C000882331F019DD0F5F1F4FF8018491F8CF57
:1066D0008AE012DDFE01849103EF1BE0882331F094
:1066E0000BDD0F5F1F4FF8018491F8CF4091DC164E
:1066F0005091DD166091DE167091DF1689EA95E003
:106700000E94E0434091C0165091C1166091C2169C
:106710007091C31686EA95E00E94E04340911017FD
:1067200050911117609112177091131783EA95E039
:106730000E9408444091C4165091C5166091C61637
:106740007091C71680EA95E00E94E0434091C81618
:106750005091C9166091CA167091CB168DE995E0DB
:106760000E94E0434091CC165091CD166091CE1618
:106770007091CF168AE995E00E94E0434091D016CF
:106780005091D1166091D2167091D31687E995E099
:106790000E94E0438AE0B0DCFE01849103EF1BE03D
:1067A000882331F0A9DC0F5F1F4FF8018491F8CFE7
:1067B000E5E8F5E084918F01882331F09DDC0F5FDF
:1067C0001F4FF8018491F8CF8AE096DCFE01849196
:1067D00003EF1BE0882331F08FDC0F5F1F4FF801C0
:1067E0008491F8CF409172085091730860917408B9
:1067F000709175088CE795E00E94E043409176081F
:1068000050917708609178087091790889E795E050
:106810000E94E04340917A0850917B0860917C0887
:1068200070917D0886E795E00E94E0438AE064DC91
:10683000FE01849103EF1BE0882331F05DDC0F5FE4
:106840001F4FF8018491F8CFE8E6F5E084918F01BD
:10685000882331F051DC0F5F1F4FF8018491F8CF8E
:106860008AE04ADCFE01849103EF1BE0882331F0CB
:1068700043DC0F5F1F4FF8018491F8CF4091AA02CB
:106880005091AB026091AC027091AD028EE595E043
:106890000E94E0436091A6027091A7028091A80235
:1068A0009091A9020F94D222AB01BC018BE595E037
:1068B0000E94E0436091A2027091A3028091A40221
:1068C0009091A5020F94DE22AB01BC0188E595E012
:1068D0000E94E0438AE010DCFE01849103EF1BE09C
:1068E000882331F009DC0F5F1F4FF8018491F8CF46
:1068F000E2E4F5E084918F01882331F0FDDB0F5F46
:106900001F4FF8018491F8CF8AE0F6DBFE018491F5
:1069100003EF1BE0882331F0EFDB0F5F1F4FF8011F
:106920008491F8CF40919A0250919B0260919C0211
:1069300070919D0288E395E00E94E0436091960289
:106940007091970280919802909199020F94D222AF
:10695000AB01BC0185E395E00E94E04360919202A7
:106960007091930280919402909195020F94DE228F
:10697000AB01BC0182E395E00E94E0438AE0BCDB0E
:10698000FE01849103EF1BE0882331F0B5DB0F5F3C
:106990001F4FF8018491F8CFEEEFF4E084918F015E
:1069A000882331F0A9DB0F5F1F4FF8018491F8CFE6
:1069B0008AE0A2DBFE01849103EF1BE0882331F023
:1069C0009BDB0F5F1F4FF8018491F8CF40912602A7
:1069D00050912702609128027091290284EF94E07F
:1069E0000E94E04320E030E040E752E460911E0264
:1069F00070911F0280912002909121020F9407A7AD
:106A0000AB01BC0181EF94E00E94E0434091620839
:106A10005091630860916408709165088EEE94E06F
:106A20000E94E0438AE068DBFE01849103EF1BE0F3
:106A3000882331F061DB0F5F1F4FF8018491F8CF9D
:106A4000E2ECF4E084918F01882331F055DB0F5F95
:106A50001F4FF8018491F8CF8AE04EDBFE0184914C
:106A600003EF1BE0882331F047DB0F5F1F4FF80176
:106A70008491F8CF40915E0850915F086091600862
:106A80007091610888EB94E00E94E04320E030E0E0
:106A900040E752E460911A0270911B0280911C023F
:106AA00090911D020F9407A7AB01BC0185EB94E008
:106AB0000E94E0438AE020DBFE01849103EF1BE0AB
:106AC000882331F019DB0F5F1F4FF8018491F8CF55
:106AD000EBE5F4E084918F01882331F00DDB0F5F4B
:106AE0001F4FF8018491F8CF8AE006DBFE01849104
:106AF00003EF1BE0882331F0FFDA0F5F1F4FF8012F
:106B00008491F8CF4091670850E060E070E081E543
:106B100094E00E9408448AE0EFDAFE01849103EFDA
:106B20001BE0882331F0E8DA0F5F1F4FF8018491F2
:106B3000F8CF80918E08882339F1EEE3F4E0849158
:106B40008F01882331F0D8DA0F5F1F4FF80184914D
:106B5000F8CF8AE0D1DAFE01849103EF1BE08823AD
:106B600031F0CADA0F5F1F4FF8018491F8CF4091DE
:106B7000460250914702609148027091490284E3B5
:106B800094E00E94E0430BC0E8E1F4E08491EF015F
:106B9000882329F0B1DA2196FE018491F9CF8AE0A9
:106BA000DF91CF911F910F91A7CAAF92BF92CF9261
:106BB000DF92EF92FF920F931F93CF93DF93CDB7A6
:106BC000DEB7E0970FB6F894DEBF0FBECDBF80E111
:106BD000ECEBF2E0DE01919601900D928A95E1F7DF
:106BE00080E1ECECF2E0DE01519601900D928A9585
:106BF000E1F780E1ECEDF2E0DE01119601900D92FB
:106C00008A95E1F76E0181E2C80ED11C80EFE82E73
:106C100086E1F82E8E010F5E1F4F60E077E1AE0136
:106C20004F5F5F4F90EEA92E96E1B92E20E030E045
:106C3000F60181919191A191B1916F01F701819339
:106C40009193A193B1937F01F80181919191A191C9
:106C5000B1918F01FB0181939193A193B193BF01F6
:106C6000FA0181919191A191B191AF01F5018193C7
:106C70009193A193B1935F012F5F3F4F2430310572
:106C8000B9F60F94F30380E090E4ACE9B4E48093A8
:106C9000D8169093D916A093DA16B093DB1680938A
:106CA000D4169093D516A093D616B093D7161092FB
:106CB000DC161092DD161092DE161092DF1680E2BE
:106CC0009EE4A0E0B0E08093101790931117A0937A
:106CD0001217B09313171092C0161092C11610928B
:106CE000C2161092C31680E090E0A0E2B1E4809357
:106CF000C4169093C516A093C616B093C71680937A
:106D0000C8169093C916A093CA16B093CB168DECF3
:106D10009CECACECBEE38093CC169093CD16A09384
:106D2000CE16B093CF1680E090E0A0E2B0E480935E
:106D3000D0169093D116A093D216B093D31610927A
:106D40007A0810927B0810927C0810927D081092AD
:106D500076081092770810927808109279081092AD
:106D600072081092730810927408109275088DE3DF
:106D70009AE0A1E8B1E48093AA029093AB02A093B9
:106D8000AC02B093AD026DEC7CEC84E99FE30F9410
:106D9000CC226093A6027093A7028093A8029093DE
:106DA000A90265E87BEE80E692E40F94D822609316
:106DB000A2027093A3028093A4029093A5020F9461
:106DC000A71480E090E0A0E8BFE380939E02909338
:106DD0009F02A093A002B093A1021092670880E0E6
:106DE00090E0A0E4B0E48093260290932702A09361
:106DF0002802B093290240E050E064E372E440933B
:106E00001E0250931F026093200270932102109281
:106E1000620810926308109264081092650810923C
:106E20005E0810925F08109260081092610840E0BE
:106E300050E060E071E440931A0250931B026093AB
:106E40001C0270931D0210928E088093460290934C
:106E50004702A0934802B09349020E94F756E3EF1D
:106E6000FBE084918F01882331F046D90F5F1F4FDB
:106E7000F8018491F8CFECEDF3E084918F01882341
:106E800031F03AD90F5F1F4FF8018491F8CF8AE0B3
:106E9000E0960FB6F894DEBF0FBECDBFDF91CF9165
:106EA0001F910F91FF90EF90DF90CF90BF90AF9028
:106EB00023C90F931F93CF93DF93CDB7DEB72C97E2
:106EC0000FB6F894DEBF0FBECDBF8C019C878B87B9
:106ED00046E552E360E070E049835A836B837C832C
:106EE00044E0BE016B5F7F4FCE010B965FD943E05C
:106EF00050E0BE016B5F7F4FCE0101960F9414AD41
:106F0000892B09F009C140E160EF76E1CE010B96D3
:106F10004DD940E160E077E1CE010B9647D940E1E1
:106F200060EE76E1CE010B9641D90F94F30344E075
:106F300068ED76E1CE010B9639D944E064ED76E157
:106F4000CE010B9633D944E06CED76E1CE010B9681
:106F50002DD944E060EC76E1CE010B9627D944E0D0
:106F600060E177E1CE010B9621D944E064EC76E153
:106F7000CE010B961BD944E068EC76E1CE010B966E
:106F800015D944E06CEC76E1CE010B960FD944E0C4
:106F900060ED76E1CE010B9609D920E030E040E2C9
:106FA00051E46091C4167091C5168091C6169091F7
:106FB000C7160F9435A6181664F480E090E0A0E29E
:106FC000B1E48093C4169093C516A093C616B093EF
:106FD000C71620E030E040E251E46091C81670919D
:106FE000C9168091CA169091CB160F9435A6181623
:106FF00064F480E090E0A0E2B1E48093C81690933E
:10700000C916A093CA16B093CB164CE062E778E09D
:10701000CE010B96CBD844E06BE678E0CE010B9620
:10702000C5D844E06AEA72E0CE010B96BFD844E0CE
:1070300066EA72E0CE010B96B9D844E062EA72E0EB
:10704000CE010B96B3D844E06AE972E0CE010B960C
:10705000ADD844E066E972E0CE010B96A7D844E0D3
:1070600062E972E0CE010B96A1D842E0BE01675FF3
:107070007F4FCE010B969AD841E067E678E0CE01CB
:107080000B9694D844E066E272E0CE010B968ED85F
:1070900044E06EE172E0CE010B9688D844E062E6EF
:1070A00078E0CE010B9682D844E06EE578E0CE0120
:1070B0000B967CD844E06AE172E0CE010B9676D85C
:1070C00041E06EE878E0CE010B9670D844E066E4CB
:1070D00072E0CE010B966AD80F94A714E3EFFBE0A1
:1070E00084918F01882331F007D80F5F1F4FF8017B
:1070F0008491F8CFEEEFF3E084918F01882339F08B
:107100000E947C300F5F1F4FF8018491F7CF8AE017
:107110000E947C3091E014C048DDC8010F945DB03E
:107120008F3F69F4C80101960F945DB08F3F39F429
:10713000C80102960F945DB091E08F3F09F090E096
:10714000892F2C960FB6F894DEBF0FBECDBFDF910E
:10715000CF911F910F910895CF93DF93EC0160E0E1
:107160008E810F947F9D81E090E00F94C19B61E040
:107170008E810F947F9D81E090E00F94C19B60E031
:107180008E810F947F9D84E690E0DF91CF910D94E6
:10719000C19BCF92DF92EF92FF920F931F93CF93F9
:1071A000DF937C01C0E0D0E0C62ED12C87010C0F0C
:1071B0001D1F61E0F80187810F94469DB6010C2EDA
:1071C00002C0759567950A94E2F76170F8018781AE
:1071D0000F947F9D2196C430D10541F7C701DF91FF
:1071E000CF911F910F91FF90EF90DF90CF90B4CF90
:1071F000CF92DF92EF92FF920F931F93CF93DF9383
:107200007C01C0E0D0E0C62ED12C87010C0F1D1FE1
:1072100061E0F80187810F94469DB6010C2E02C0F3
:10722000759567950A94E2F76170F80187810F946C
:107230007F9D2196C830D10541F7C701DF91CF91DD
:107240001F910F91FF90EF90DF90CF9085CF1F930C
:10725000CF93DF93EC01162F642F8C810F947F9DC9
:107260008D818F3F19F060E00F947F9D8F85612F96
:1072700084FF05C0CE01DF91CF911F91B9CF70E09F
:1072800084E0759567958A95E1F7CE0182DF612FDD
:10729000CE01DF91CF911F917CCF40E0D8CF61E04C
:1072A000FCDF80E496E00D94C19B62E0F6DF80E4B1
:1072B00096E00D94C19BCF93DF93CDB7DEB72897AF
:1072C0000FB6F894DEBF0FBECDBF28E0ECEEF2E0C3
:1072D000DE01119601900D922A95E1F7FC012389B8
:1072E000421710F04FEF420FFE013196E40FF11DEF
:1072F000E40FF11D2081260F2068622F28960FB61B
:10730000F894DEBF0FBECDBFDF91CF91C6CFFC0199
:107310006089262F2460208B6C60BFCFCF93DF93D2
:10732000EC01423018F08F8588608F874B8B1C8A68
:10733000222329F0413019F48F8584608F8780E5FE
:1073400093EC0F94C19B60E08C810F947F9D60E073
:107350008E810F947F9D8D818F3F19F060E00F9497
:107360007F9D6F8564FD19C063E0CE0112DF84E963
:1073700091E10F94C19B63E0CE010BDF84E991E1C1
:107380000F94C19B63E0CE0104DF86E990E00F9487
:10739000C19B62E0CE01FDDE13C06062CE017DDFE5
:1073A00084E991E10F94C19B6F856062CE0175DF26
:1073B00086E990E00F94C19B6F856062CE016DDF1E
:1073C0006F856062CE0169DF8CE390E00F94C19B12
:1073D00084E0888BCE019BDF8CE390E00F94C19B0F
:1073E000CE015DDF88EB9BE00F94C19B82E0898B2F
:1073F00066E0CE0152DF8CE390E00F94C19B1D8AC2
:10740000DF91CF9108956F927F928F92AF92CF923A
:10741000EF920F931F93CF93DF93CDB7DEB73C016D
:10742000162F842F5E854F8538899989F3018483CF
:1074300025830683E782C086A18682865387448798
:107440003587968761E00F94469DF30185818F3FD4
:1074500019F061E00F94469D61E0F30186810F947D
:10746000469D112319F0F301178603C080E1F30153
:10747000878720E041E060E1C301DF91CF911F9158
:107480000F91EF90CF90AF908F907F906F9046CFFD
:107490008F92AF92CF92EF920F93DC0113961C92D2
:1074A0001E921297EEE5F3E0ED93FC931F921F926C
:1074B0001F921F928C2CAE2CC02EE22E042F2FEF89
:1074C000462F61E0A0DF0F900F900F900F900F916B
:1074D000EF90CF90AF908F900895CF93DF93EC0112
:1074E000423018F08F8588608F874B8B1C8A22234F
:1074F00029F0413019F48F8584608F8780E593EC03
:107500000F94C19B60E08C810F947F9D60E08E8121
:107510000F947F9D8D818F3F19F060E00F947F9DC8
:107520006F8564FD19C063E0CE0133DE84E991E12B
:107530000F94C19B63E0CE012CDE84E991E10F94AE
:10754000C19B63E0CE0125DE86E990E00F94C19BEC
:1075500062E0CE011EDE13C06062CE019EDE84E9D1
:1075600091E10F94C19B6F856062CE0196DE86E942
:1075700090E00F94C19B6F856062CE018EDE6F85B7
:107580006062CE018ADE8CE390E00F94C19B84E0C0
:10759000888BCE01BCDE8CE390E00F94C19BCE01C2
:1075A00084DE80E496E00F94C19B82E0898B66E0E4
:1075B000CE0173DE8CE390E00F94C19B40E068E065
:1075C000CE0179DE67E576E0CE010F941A9E41E0A8
:1075D00068E0CE0170DE67E576E0CE010F941A9E7A
:1075E00042E066E0CE0167DE65E576E0CE01DF9140
:1075F000CF910D941A9EFC0160896D7F608B68604D
:107600004CCECF93DF93EC01262F8D898230B0F0E2
:10761000FE01E80FF11D658B3E8980ED860F8A30F3
:1076200058F4316081E090E00D8802C0880F991F06
:107630000A94E2F7382B01C03E7F3E8B4D8981E0F2
:10764000840F8D8B50E04830510508F0B6C0FA0128
:10765000EE58FF4F0D9447A92B3109F0AEC0AEC0D4
:107660001E8A2B3509F0A9C0A9C0223309F4A6C08F
:107670002F3309F4A3C08E897AC08F89823331F009
:107680008F3349F4223309F098C098C02A3419F492
:10769000CE0105DE92C08E8982FF8FC02B3309F0A8
:1076A00066C08CC08F898F3341F4888D823309F096
:1076B00084C0253309F081C081C08E8982FF7DC0DE
:1076C000988D9B3311F480FD79C083FF76C02B33F6
:1076D00009F073C073C04F894F3371F4888D8233C2
:1076E00009F06BC0898D853309F067C02C3609F02D
:1076F00064C0CE0180DF61C08E8982FF5EC0988D3C
:107700009B3339F484FF05C0283489F54053698DD3
:107710002CC083FF52C0998D9B3309F04EC027C007
:107720008E8982FF4AC0488D4B3361F4982F907345
:10773000903341F4283431F44F8940536A8D6053BB
:10774000898D32C083FF39C0998D9B33B1F585FF98
:1077500034C0283461F440538F89880F8056982FA5
:10776000990F990F980F490F6A8D605324C080FFBD
:1077700024C024C08E89982F9C709C30F1F4998D80
:107780009B33D9F480768036C1F42834B1F4488D27
:1077900040538F89880F8056982F990F990F980F13
:1077A000490F6B8D60538A8D880F8056982F990FE3
:1077B000990F980F690FCE017EDD1D8A81E090E060
:1077C000DF91CF910895CF92DF92EF92FF920F93C6
:1077D0001F93CF93DF931F921F92CDB7DEB78C011B
:1077E000677088E0689FB00111246064C801498314
:1077F0005A8353DD4981C42E5A81D52EE12CF12CB8
:10780000D6016D916D01D801ED91FC910190F0814F
:10781000E02DC8011995BFEFEB1AFB0AE8E0EE1660
:10782000F10471F70F900F90DF91CF911F910F919D
:10783000FF90EF90DF90CF900895FC0125892111F2
:1078400002C06B3109F4DDCE41E001DD81E090E062
:1078500008959091A107911107C09091C00095FFE4
:10786000FCCF8093C6000895913031F49091C80008
:1078700095FFFCCF8093CE0008951F920F920FB614
:107880000F9211240BB60F922F933F934F935F9358
:107890006F938F939F93EF93FF938091C00084FF2A
:1078A00003C08091C6001DC06091C6008091A107F1
:1078B000811117C020919D0730919E07C901019643
:1078C0008F77992740919F075091A00784179507BC
:1078D00041F0F901E35EF84F608390939E07809337
:1078E0009D07FF91EF919F918F916F915F914F91C4
:1078F0003F912F910F900BBE0F900FBE0F901F90D6
:1079000018951F920F920FB60F9211240BB60F927B
:107910002F933F934F935F936F938F939F93EF9327
:10792000FF938091C80084FF03C08091CE001DC0EA
:107930006091CE008091A1078130B9F420919D071C
:1079400030919E07C90101968F77992740919F0733
:107950005091A0078417950741F0F901E35EF84FB5
:10796000608390939E0780939D07FF91EF919F9175
:107970008F916F915F914F913F912F910F900BBE1F
:107980000F900FBE0F901F901895CF92DF92EF923D
:10799000FF926A017B01411581EE5807610571056F
:1079A00009F463C082E08093C00060E079E08DE379
:1079B00090E0A70196010F942BA9215031094109AC
:1079C0005109CA01B90122E030E040E050E00F94D3
:1079D0002BA991E03093C5002093C4008091C10091
:1079E00080618093C1008091C10088608093C10054
:1079F0008091C10080688093C1008091A10781308F
:107A0000D1F5992341F082E08093C80060E079E0ED
:107A10008DE390E006C01092C80060E874E88EE143
:107A200090E0A70196010F942BA92150310941093B
:107A30005109CA01B90122E030E040E050E00F9462
:107A40002BA93093CD002093CC008091C900806198
:107A50008093C9008091C90088608093C90080919B
:107A6000C90080688093C90006C01092C00090E0F1
:107A700020E130E0AFCFFF90EF90DF90CF900895FE
:107A800020919F073091A00780919D0790919E07BC
:107A90008217930771F0F901E35EF84F80812F5F41
:107AA0003F4F2F7733273093A00720939F0790E015
:107AB00008958FEF9FEF089580919F079091A00701
:107AC00090939E0780939D0708954F925F926F92C7
:107AD0007F928F929F92AF92BF92CF92DF92EF925E
:107AE000FF920F931F93CF93DF93CDB7DEB7A0978D
:107AF0000FB6F894DEBF0FBECDBF4115510561052D
:107B00007105C1F480E3A0960FB6F894DEBF0FBEF6
:107B1000CDBFDF91CF911F910F91FF90EF90DF903C
:107B2000CF90BF90AF909F908F907F906F905F901D
:107B30004F908FCECE0101967C01812C912C540167
:107B40008C01422E512C612C712C9FEF891A990ABD
:107B5000A90AB90ACB01BA01A30192010F9409A99C
:107B6000CA01F70161937F01A901BC0141155105CB
:107B70006105710551F775016401F1E0CF1AD10873
:107B8000E108F108F801EC0DFD1D80818A3010F448
:107B9000805D01C0895C5DDE81E0C81AD108E10822
:107BA000F1089FEFC916D906E906F90659F7A0961C
:107BB0000FB6F894DEBF0FBECDBFDF91CF911F91FE
:107BC0000F91FF90EF90DF90CF90BF90AF909F907C
:107BD0008F907F906F905F904F90089521153105A1
:107BE00011F4842F36CE71CF0F931F93CF93DF9371
:107BF00000D01F92CDB7DEB78C0177FF11C08DE2A8
:107C000049835A836B837C8324DE49815A816B814B
:107C10007C8170956095509541955F4F6F4F7F4F78
:107C20002AE0C8010F900F900F900F90DF91CF9135
:107C30001F910F914ACF2115310511F4842F09CEE0
:107C40002A30310509F4D0CF40CF9A01462F55276D
:107C500047FD5095652F752FEECF9A01AB01662732
:107C600057FD6095762FE7CF8DE0F3DD8AE0F1CD0B
:107C70000F931F93CF93DF938C01EB01899188239E
:107C800011F0E7DDFBCFC801DF91CF911F910F917C
:107C9000EBCFCF93DF93EC019A01AB01662757FD41
:107CA0006095762FC8DFCE01DF91CF91DDCFCF93E6
:107CB000DF93EC019A01AB0160E070E08FDFCE0151
:107CC000DF91CF91D1CF8F929F92AF92BF92CF92FF
:107CD000DF92EF92FF921F93CF93DF93EC016A0143
:107CE0007B01122F20E030E0A901C701B6010F94FB
:107CF00032A487FF06C08DE2ACDDF7FAF094F7F806
:107D0000F094B12C60E070E080E09FE3B11641F0A8
:107D100020E030E040E251E40F9439A4B394F6CF70
:107D20009B01AC01C701B6010F9459A36B017C0103
:107D30000F94A6A44B015C010F94D2A49B01AC014B
:107D4000C701B6010F9458A36B017C012AE0B5016D
:107D5000A401CE01BADE112359F083EAA82E84E0F3
:107D6000B82EF50181915F01882311F072DDF9CF02
:107D7000112319F120E030E040E251E4C701B601DF
:107D80000F9407A76B017C010F94A1A44B01AA24B7
:107D900097FCA094BA2CB501A401CE0125DFC50142
:107DA000B4010F94D4A49B01AC01C701B6010F9498
:107DB00058A36B017C011150DBCFDF91CF911F9154
:107DC000FF90EF90DF90CF90BF90AF909F908F90FB
:107DD000089579CFCF93DF93EC0175DFCE01DF916A
:107DE000CF9142CFFC016591759185919491089551
:107DF000EF92FF920F931F93CF93DF93EC01CC0F81
:107E0000DD1FCC0FDD1FCE018153944FEBDF9E01B0
:107E10002258374F79018E010E58174FF8012081F3
:107E20003181428153810F9459A3F701608371839B
:107E300082839383CE018951944FD4DF9E012A5CC3
:107E40003D4F7901F80120813181428153810F94A6
:107E500059A3F7016083718382839383CE01855296
:107E6000944FC0DFC65DDD4FF80120813181428132
:107E700053810F9459A3688379838A839B83DF910D
:107E8000CF911F910F91FF90EF9008952091520E86
:107E90003091530EBC01C901895A914F0F9431ADF5
:107EA0009093490E8093480E21E0892B09F420E03D
:107EB000822F0895CF93C82F40910E0250910F0248
:107EC000609110027091110240933508509336086A
:107ED0006093370870933808209158023091590206
:107EE0003093FD082093FC0824E630E030935902DB
:107EF000209358020F945B9B609330087093310875
:107F000080933208909333088C2FCF910D948D0578
:107F100080E00F948D058091350890913608A091EE
:107F20003708B091380880930E0290930F02A09307
:107F30001002B09311028091FC089091FD0890937B
:107F40005902809358020F945B9B609330087093A2
:107F5000310880933208909333080895682F77276B
:107F600067FD70958091520E9091530E895A914FF2
:107F70000F94F9AC9093490E8093480E21E0892B21
:107F800009F420E0822F08958091480E9091490EC7
:107F90004AE050E060E070E001960F940AABCB013C
:107FA00008958091480E9091490E4AE050E060E0BB
:107FB00070E001960D940AAB8091480E9091490EA5
:107FC00060E070E001960D94A2A99091A107911133
:107FD00007C09091C00095FFFCCF8093C600089524
:107FE000913031F49091C80095FFFCCF8093CE0082
:107FF0000895EBDF80E090E008952F923F924F923A
:108000005F926F927F928F929F92AF92BF92CF9228
:10801000DF92EF92FF920F931F93CF93DF93CDB731
:10802000DEB760970FB6F894DEBF0FBECDBF1C0160
:108030002A013B014801590120E030E04CE052E4C4
:10804000C301B2010F9458A325E535E547E052E49A
:108050000F9439A46B017C010F940FA50F94A1A478
:108060008B0177FF12C020E030E040E85FE3C701FA
:10807000B6010F9435A618160CF05DC0C12CD12C9A
:10808000E0E8EE2EEFE3FE2E56C066307105DCF020
:108090002AEA3AE24CE453E4C301B2010F9458A334
:1080A00025E535E547E052E40F9439A46B017C01E6
:1080B00020E030E0A9010F9432A487FF3FC0C12C1B
:1080C000D12C76013BC0882777FD8095982F0F949F
:1080D000D4A425E535E547E052E40F9407A720E056
:1080E00030E04CE052E40F9459A39B01AC01C30172
:1080F000B2010F9458A325E535E547E052E40F940B
:1081000039A46B017C0120E030E0A9010F9432A476
:1081100087FD17C020E030E040E85FE3C701B6010B
:108120000F9435A6181684F4C12CD12C70E8E72ED4
:108130007FE3F72E09C000E010E006C005E010E084
:1081400003C0C12CD12C760120E030E040EC50E49B
:10815000C501B4010F9458A32BEA3AEA42E052E475
:108160000F9439A42B013C010F940FA50F94A1A4E7
:10817000788B6F8777FF12C020E030E040E85FE344
:10818000C301B2010F9435A618160CF05FC0412C44
:10819000512C60E8662E6FE3762E58C0AF85B88903
:1081A0001697E4F026E535E549E253E4C501B4014C
:1081B0000F9458A32BEA3AEA42E052E40F9439A410
:1081C0002B013C0120E030E0A9010F9432A487FD8F
:1081D00040C0E5E0F0E0F88BEF8746C0882777FDE8
:1081E0008095982F0F94D4A42BEA3AEA42E052E407
:1081F0000F9407A720E030E040EC50E40F9459A31F
:108200009B01AC01C501B4010F9458A32BEA3AEAD3
:1082100042E052E40F9439A42B013C0120E030E00D
:10822000A9010F9432A487FD1CC020E030E040E893
:108230005FE3C301B2010F9435A61816ACF4412CCC
:10824000512C50E8652E5FE3752E0EC0188A1F86EC
:108250000BC0412C512C320125E030E0388B2F87A8
:1082600003C0412C512C3201A701960160E070E05F
:1082700080E89FE30F9458A369837A838B839C8360
:10828000C80101969E838D83AF85B8891196BA8700
:10829000A987A301920160E070E080E89FE30F945A
:1082A00058A36B877C878D879E8747E02F85388909
:1082B000429FF001439FF00D1124F887EF83E00FF8
:1082C000F11FEE0FFF1FEE0FFF1FE20DF31D2181C7
:1082D00032814381548169817A818B819C810F94A1
:1082E00007A74B015C01EF81F8858D819E81E80F26
:1082F000F91FEE0FFF1FEE0FFF1FE20DF31D21818F
:10830000328143815481C701B6010F9407A79B01B5
:10831000AC01C501B4010F9459A39B01AC016B855D
:108320007C858D859E850F9407A74B015C0127E016
:10833000E985FA852E9FD0012F9FB00D1124B887B3
:10834000AF83FD01E00FF11FEE0FFF1FEE0FFF1FC8
:10835000E20DF31D218132814381548169817A814B
:108360008B819C810F9407A769837A838B839C837D
:10837000AF81B8858D819E81A80FB91FAA0FBB1F41
:10838000AA0FBB1FA20DB31D11962D913D914D91CA
:108390005C911497C701B6010F9407A79B01AC012C
:1083A00069817A818B819C810F9459A39B01AC01D7
:1083B000C301B2010F9407A79B01AC01C501B40131
:1083C0000F9459A360960FB6F894DEBF0FBECDBFD1
:1083D000DF91CF911F910F91FF90EF90DF90CF90A1
:1083E000BF90AF909F908F907F906F905F904F90D5
:1083F0003F902F9008954F925F926F927F929F923D
:10840000AF92BF92CF92DF92EF92FF920F931F93A2
:10841000CF93DF937C015B018A01E901909090107A
:10842000911014C0FC0180819181A281B381FA0175
:1084300080839183A283B383FB0180819181A28198
:10844000B38188839983AA83BB837FC091FE55C083
:10845000FC012081318142815381609180107091B3
:10846000811080918210909183100F9407A72B01A7
:108470003C01F5012081318142815381609184105A
:108480007091851080918610909187100F9407A7A6
:108490009B01AC01C301B2010F9459A3F8016083A1
:1084A000718382839383F7012081318142815381DB
:1084B000609188107091891080918A1090918B1032
:1084C0000F9407A76B017C01F50120813181428166
:1084D000538160918C1070918D1080918E109091CD
:1084E0008F100F9407A79B01AC01C701B6010F9431
:1084F00059A3688379838A839B8390FE26C0209149
:1085000068103091691040916A1050916B10F80119
:1085100060817181828193810F9459A3F8016083F6
:1085200071838283938320916C1030916D10409100
:108530006E1050916F10688179818A819B810F94B0
:1085400059A3688379838A839B83DF91CF911F919D
:108550000F91FF90EF90DF90CF90BF90AF909F90E2
:108560007F906F905F904F9008952F923F924F921F
:108570005F926F927F928F929F92AF92BF92CF92B3
:10858000DF92EF92FF920F931F93CF93DF93CDB7BC
:10859000DEB728970FB6F894DEBF0FBECDBF8C01B3
:1085A0001B019E012F5F3F4FAE014B5F5F4F23DFEB
:1085B00020E030E0A9016D817E818F8198850F9444
:1085C00032A487FF07C01D821E821F821886FF24E7
:1085D000F39401C0F12C20E030E040E850EC6981D8
:1085E0007A818B819C810F9432A487FF0AC080E03E
:1085F00090E0A0E8B0EC89839A83AB83BC83FF242E
:10860000F39420E030E04FE753E46D817E818F8169
:1086100098850F9435A6181654F480E090E0AFE7E3
:10862000B3E48D839E83AF83B887FF24F39420E067
:1086300030E042E553E469817A818B819C810F941B
:1086400035A618164CF480E090E0A2E5B3E48983E7
:108650009A83AB83BC8303C0FF2009F483C0C98025
:10866000DA80EB80FC808D809E80AF80B884709033
:10867000901071100BC0F80180829182A282B382A7
:10868000F101C082D182E282F3826AC070FE1CC016
:10869000209168103091691040916A1050916B10D0
:1086A000C501B4010F9458A34B015C0120916C10DB
:1086B00030916D1040916E1050916F10C701B6014E
:1086C0000F9458A36B017C0171FE4AC02091701079
:1086D000309171104091721050917310C501B40126
:1086E0000F9407A72B013C01209174103091751055
:1086F0004091761050917710C701B6010F9407A7EB
:108700009B01AC01C301B2010F9459A3F80160832E
:1087100071838283938320917810309179104091F6
:108720007A1050917B10C501B4010F9407A74B013B
:108730005C0120917C1030917D1040917E10509111
:108740007F10C701B6010F9407A79B01AC01C501BB
:10875000B4010F9459A3F1016083718382839383E1
:10876000FF24F3948F2D28960FB6F894DEBF0FBE2A
:10877000CDBFDF91CF911F910F91FF90EF90DF90D0
:10878000CF90BF90AF909F908F907F906F905F90B1
:108790004F903F902F900895CF93DF931F92CDB7C6
:1087A000DEB7BE016F5F7F4F0F94256E0F90DF9194
:1087B000CF910895682F87EF9FE00D946FB00895D3
:1087C0000F931F93CF93DF9300D01F92CDB7DEB7E7
:1087D0008C01FC018491882371F049835A836B8357
:1087E0007C83F3DB0F5F1F4FF80184917C816B81E9
:1087F0005A814981F0CF22E030E08CE197E00F9080
:108800000F900F900F90DF91CF911F910F91E1CAC0
:108810000F931F93CF93DF9300D01F92CDB7DEB796
:108820008C01FC018491882371F049835A836B8306
:108830007C83CBDB0F5F1F4FF80184917C816B81C0
:108840005A814981F0CF2AE030E08CE197E00F9027
:108850000F900F900F90DF91CF911F910F91BEC994
:10886000EF92FF920F931F93CF93DF931F92CDB799
:10887000DEB789830F94CF2E8981823009F495C0A9
:108880000CF062C0882309F46EC0813009F025C164
:108890009FB7F894809102018460809302019FBF8A
:1088A000EFEFF1EE24E0E150F0402040E1F700C0AE
:1088B00000009FB7F894809102018B7F80930201A2
:1088C0009FBF40E050E0BA018DEE9FE00F9481B071
:1088D00040E050E0BA0181EF9FE00F9481B060E08A
:1088E00086E69FE00F946FB060E088E69FE00F940B
:1088F0006FB060E085E69FE00F946FB060E084E6C3
:108900009FE00F946FB060E070E085E09FE00F940F
:1089100089B060E070E083E09FE00F9489B060E090
:1089200070E081E09FE00F9489B060E070E08FEF2D
:108930009EE00F9489B00F90DF91CF911F910F911E
:10894000FF90EF900D94854C833009F461C0843022
:1089500009F0C3C00F90DF91CF911F910F91FF904D
:10896000EF900D9480749FB7F89480910201846019
:10897000809302019FBF2FEF81EE94E02150804051
:108980009040E1F700C000009FB7F8948091020189
:108990008B7F809302019FBF0F90DF91CF911F913A
:1089A0000F91FF90EF900D94B92F0F94B92F80EF96
:1089B00001DF61E08FE59FE00F948DB01092DC182D
:1089C0001092DB186091DD1884EC9FE00F946FB07B
:1089D0006BED78E181EC9FE00F940D2F9FB7F89439
:1089E000809102018460809302019FBF8FEF91EE1E
:1089F000E4E081509040E040E1F700C000009FB704
:108A0000F894809102018B7F809302019FBF65C023
:108A100086EA9BE00F945C4145E95BE062E081E01F
:108A20000F940C529FB7F894809102018460809358
:108A300002019FBFFFEF21EE84E0F1502040804013
:108A4000E1F700C000009FB7F894809102018B7F8E
:108A5000809302019FBF10921C0810921B084EE8E1
:108A60005BE063E083E00F940C5240911B0850914F
:108A70001C0863E083E00F94DA2EE12CF12C09E26C
:108A800010E06FEFC7010F948DB0C701B8010F94CC
:108A9000F6A8892BD9F480911B0890911C080196A7
:108AA00090931C0880931B0847E85BE063E083E039
:108AB0000F940C5240911B0850911C0863E083E016
:108AC0000F94DA2E85E89BE00F945C419FEFE91A42
:108AD000F90AE114E0E1FE06A1F60F90DF91CF91D3
:108AE0001F910F91FF90EF9008956DE078E085E57C
:108AF0009BE00D9467AD84E090E090931802809322
:108B000017028091000186FD39C02FEF83ED90E3BD
:108B1000215080409040E1F700C0000080910001AA
:108B200086FD2CC00F94CF2E87E49BE00F945C4110
:108B3000809101018460809301019FB7F894809136
:108B400002018460809302019FBF8091000186FF33
:108B5000FCCF9FB7F894809102018B7F8093020134
:108B60009FBF2FEF87EA91E6215080409040E1F7C8
:108B700000C000000F94D03260E072DE82E090E02E
:108B800090931802809317020895E091CC08F0E0CA
:108B9000EE0FFF1FE25CF84B859194910F945D7A84
:108BA00081E00D94E66D1F93CF93DF930E94F7F160
:108BB000EC01DF93CF938DED9AE09F938F930F9409
:108BC00094AD87E69FE00F945DB0182F0F900F9043
:108BD0000F900F90CD2B29F481E080934F1010E07F
:108BE00002C010924F1084ED9AE00F94E4AD11236F
:108BF00049F08BEC9AE00F94E4ADDF91CF911F9197
:108C00000C9454BC81EC9AE00F94E4ADDF91CF91C9
:108C10001F910C9471BC8F929F92AF92BF92CF9292
:108C2000DF92EF92FF92CF93DF938091DD18811155
:108C300085C00F945B9B6B017C0120911202222363
:108C400009F474C040911702509118024130510547
:108C500009F46CC08091130290911402A091150246
:108C6000B091160246015701881A990AAA0ABB0A4E
:108C700030E0A8EEB3E00F944DA986169706A8063B
:108C8000B9060CF45BC04430510541F14CF442305C
:108C900051050CF44BC0E3EFFBE08491EF0109C0F8
:108CA0004530510509F042C0E3EFFBE08491EF014C
:108CB0002BC0882329F089D92196FE018491F9CF10
:108CC000ECE9FAE08491EF01882329F07ED921961E
:108CD000FE018491F9CF8AE078D928C0E3EFFBE068
:108CE0008491EF01882329F070D92196FE018491A7
:108CF000F9CFE6E8FAE08491EF01882361F365D9C2
:108D00002196FE018491F9CF882329F05ED921961E
:108D1000FE018491F9CFEFE6FAE08491EF01882318
:108D2000D1F253D92196FE018491F9CFC09213025A
:108D3000D0921402E0921502F0921602DF91CF91C8
:108D4000FF90EF90DF90CF90BF90AF909F908F906B
:108D50000895CF93C0E020914E0E30914F0E232BFB
:108D6000A9F082E693E092D881110EC086E693E0E6
:108D70008DD8811109C080914D0E811102C00E94D1
:108D8000F3B410924D0EE7CFC1E0F5CF8C2FCF9109
:108D900008952F923F924F925F926F927F928F929F
:108DA0009F92AF92BF92CF92DF92EF92FF920F937A
:108DB0001F93CF93DF93CDB7DEB729970FB6F89403
:108DC000DEBF0FBECDBF3C0181E00F948D058F83C8
:108DD00082E06816710408F077C2F301EC54F44F96
:108DE000E491D301AA0FBB1FAA0FBB1FBA83A983AB
:108DF000A65ABD4FBE83AD838D919D910D90BC91C0
:108E0000A02D80930E0290930F02A0931002B093B6
:108E10001102E981FA81E258F74FF987E887108259
:108E2000118212821382E0908608F09087080091E8
:108E30008808109189082091820830918308409118
:108E400084085091850860917E0870917F08809118
:108E5000800890918108EAE8CE2EE8E0DE2E0F949B
:108E60005802E981FA81E75BF74F2F0180E090E03B
:108E7000A0E4B0E480839183A283B38320E030E058
:108E800040E752E460910E0270910F02809110024F
:108E9000909111020F9439A44B015C01E0905108AC
:108EA000F0905208009153081091540820914D08F9
:108EB00030914E0840914F085091500860914908F8
:108EC00070914A0880914B0890914C08FAE62F2E39
:108ED000F8E03F2E3F922F92A5E5CA2EA8E0DA2EA9
:108EE0000E9488F70F94350D0F94750580E00F945C
:108EF0008D05A885B9851D921D921D921C92139710
:108F0000E0908608F0908708009188081091890801
:108F100020918208309183084091840850918508FF
:108F200060917E0870917F088091800890918108FF
:108F3000BAE8CB2EB8E0DB2E0F94580280E090E028
:108F4000A0E8BFEBF20180839183A283B38320E08A
:108F500030E040E752E460910E0270910F02809180
:108F60001002909111020F9439A44B015C01E09022
:108F70005108F09052080091530810915408209124
:108F80004D0830914E0840914F0850915008609123
:108F9000490870914A0880914B0890914C083F9283
:108FA0002F92E5E5CE2EE8E0DE2E0E9488F70F94A2
:108FB000350D81E00F948D0589819A818D53944FF1
:108FC0000E94F23E2DEC3CEC4CE85FEB0F9407A7BF
:108FD000D2016D937D938D939C93139720E030E0A5
:108FE00040E752E460910E0270910F0280911002EE
:108FF000909111020F9439A44B015C01E09051084B
:10900000F0905208009153081091540820914D0897
:1090100030914E0840914F08509150086091490896
:1090200070914A0880914B0890914C083F922F9282
:109030000E9488F70F94350D0F94750580E00F940A
:109040008D05E885F9851082118212821382E090E5
:109050008608F0908708009188081091890820916F
:10906000820830918308409184085091850860916E
:109070007E0870917F088091800890918108FAE8BD
:10908000CF2EF8E0DF2E0F94580280E090E0A0E2AF
:10909000B1E4F20180839183A283B38320E030E0C6
:1090A00040E752E460910E0270910F02809110022D
:1090B000909111020F9439A44B015C01E09051088A
:1090C000F0905208009153081091540820914D08D7
:1090D00030914E0840914F085091500860914908D6
:1090E00070914A0880914B0890914C083F922F92C2
:1090F000A5E5CA2EA8E0DA2E0E9488F70F94350D58
:109100000F94750581E00F948D0580E090E0A0E755
:10911000B1ECF20180839183A283B38320E030E03D
:1091200040E05FE3AD81BE816D917D918D919C9119
:109130000F9407A760930E0270930F0280931002A2
:109140009093110220E030E040E752E40F9439A4FC
:109150004B015C01E0905108F090520800915308D7
:109160001091540820914D0830914E0840914F08BD
:10917000509150086091490870914A0880914B08BD
:1091800090914C083F922F920E9488F70F94350DD2
:10919000C3010E94F83EF301E159F74F81E080835B
:1091A0000F94750580E00F948D052AE037ED43E2BA
:1091B0005FE3E885F98560817181828193810F94F5
:1091C00058A3A885B9856D937D938D939C93139730
:1091D000E0908608F090870800918808109189082F
:1091E000209182083091830840918408509185082D
:1091F00060917E0870917F0880918008909181082D
:10920000BAE8CB2EB8E0DB2E0F9458022AE037EDF7
:1092100043E25FE3E885F985608171818281938112
:109220000F9459A3A885B9856D937D938D939C93D5
:109230001397F20160837183828393832AE939E96A
:1092400049E95EE360910E0270910F028091100275
:10925000909111020F9407A720E030E040E752E41C
:109260000F9439A44B015C01E0905108F090520832
:10927000009153081091540820914D0830914E08E8
:1092800040914F08509150086091490870914A08E8
:1092900080914B0890914C083F922F92E5E5CE2E9D
:1092A000E8E0DE2E0E9488F70F94350D10920E0232
:1092B00010920F0210921002109211020FB6F89441
:1092C000DEBF0FBECDBF62C192E06916710409F026
:1092D0005DC1E6EBFBE0749010928608109287085F
:1092E0001092880810928908209182083091830892
:1092F000409184085091850860917E0870917F08A4
:109300008091800890918108EAE8CE2EE8E0DE2E78
:10931000E12CF12C87010F9458028BEC9BE00E940A
:10932000F23E4B015C01672D772767FD7095872F13
:10933000972F0F94D4A42B013C0120E030E040ECA7
:109340005FE3C501B4010F9407A7A30192010F9435
:1093500007A769837A838B839C83609351087093FA
:109360005208809353089093540860916202709160
:109370006302809164029091650260930E02709383
:109380000F02809310029093110220E030E040E73A
:1093900052E40F9439A44B015C0120914D083091A7
:1093A0004E0840914F0850915008609149087091C3
:1093B0004A0880914B0890914C08FAE62F2EF8E06D
:1093C0003F2E3F922F92A5E5CA2EA8E0DA2EE98023
:1093D000FA800B811C810E9488F70F94350D109242
:1093E00086081092870810928808109289082091A8
:1093F00082083091830840918408509185086091DB
:109400007E0870917F088091800890918108BAE869
:10941000CB2EB8E0DB2EE12CF12C87010F94580203
:109420008FEB9BE00E94F23E9058A30192010F94B3
:1094300007A769837A838B839C8360935108709319
:109440005208809353089093540820E030E040E79E
:1094500052E460910E0270910F028091100290917F
:1094600011020F9439A44B015C0120914D083091F9
:109470004E0840914F0850915008609149087091F2
:109480004A0880914B0890914C083F922F9215E525
:10949000C12E18E0D12EE980FA800B811C810E9438
:1094A00088F70F94350D8FEB9BE00E94F23E9B01F5
:1094B000AC010F9459A3A30192010F9407A72B01AC
:1094C0003C01609351087093520880935308909325
:1094D000540820E030E040E05FE360916202709168
:1094E000630280916402909165020F9407A76093D4
:1094F0000E0270930F02809310029093110220E0ED
:1095000030E040E752E40F9439A44B015C01209114
:109510004D0830914E0840914F085091500860918D
:10952000490870914A0880914B0890914C083F92ED
:109530002F92830172010E9488F70F94350D82E00B
:1095400090E00E94F83E8091860890918708A09153
:109550008808B09189088093510890935208A0938D
:109560005308B093540810920E0210920F021092FA
:109570001002109211020F94750581E0809371081A
:109580000F900F900F900F900F900F908F81299652
:109590000FB6F894DEBF0FBECDBFDF91CF911F9104
:1095A0000F91FF90EF90DF90CF90BF90AF909F9082
:1095B0008F907F906F905F904F903F902F900D9481
:1095C0008D05CF92DF92EF92FF920F931F9380E170
:1095D000EEE7F8E0A9E4B8E001900D928A95E1F792
:1095E00080E090E0D6DB81E090E0D3DBE09086087D
:1095F000F0908708009188081091890820918208CE
:1096000030918308409184085091850860917E08CC
:1096100070917F088091800890918108FAE8CF2EA0
:10962000F8E0DF2E0F9458021F910F91FF90EF90FA
:10963000DF90CF900D9475050F945B9B609330087D
:10964000709331088093320890933308089520E096
:1096500030E0A90168EB71E084E50F94B39F69E104
:1096600070E080E090E00F948A9B84E50F94D7A28D
:1096700064E170E080E090E00D948A9B8F929F926D
:10968000AF92BF92CF92DF92EF92FF920F931F9310
:10969000CF93DF9300D01F92CDB7DEB71092FA17A9
:1096A0001092F9171092F8171092F7170F94CF2E07
:1096B0008DEA9AE00F945C418E010F5F1F4F7E018F
:1096C00025E0E20EF11C8CE197E00E94403D8F3FC7
:1096D000EFEF9E07C1F3F80181938F01EE15FF05AF
:1096E00091F789809A80AB80BC808BE20E94E53F35
:1096F000C12CD12C76018091CB08882309F447C076
:109700000EEB17E0C814D904EA04FB04A1F08CE1C5
:1097100097E00E94403D8F3FFFEF9F07C1F32FEF7F
:10972000C21AD20AE20AF20AF80181938F01F7E025
:109730000E3F1F0739F76EEB77E086E099E00E9455
:10974000D4A98BE20E94E53F0F94A218C814D90453
:10975000EA04FB0481F67BDF60E086E099E00E948A
:1097600005AA1092CB08E8E7F7E4E590F490F7013A
:109770008491882331F00E94E53FFFEFEF1AFF0A42
:10978000F6CF8AE00E94E53F80E090E000C00F90B5
:109790000F900F900F90DF91CF911F910F91FF903D
:1097A000EF90DF90CF90BF90AF909F908F900895F3
:1097B0002F923F924F925F926F927F928F929F92E1
:1097C000AF92BF92CF92DF92EF92FF920F931F93CF
:1097D000CF93DF9300D01F921F92CDB7DEB7382E04
:1097E000811112C01092F8171092F7171092FA1701
:1097F0001092F9171092FC171092FB171092FE1797
:109800001092FD170F94342F80E00F94E66D81E9DC
:1098100090E10E94E1EB0E9410CE0E9432EB109288
:109820006F08109270081092710881E00E945A3FF0
:10983000E2E6F8E4859194910E94CC43C2DE80E098
:109840000F948D0520E030E040EA50E460917E08FE
:1098500070917F0880918008909181080F9459A39E
:109860002B013C0160937E0870937F0880938008F1
:109870009093810820E030E040EA50E46091820853
:109880007091830880918408909185080F9459A362
:109890006A837B838C839D836093820870938308A3
:1098A000809384089093850820E030E040E252E401
:1098B00060916202709163028091640290916502EE
:1098C0000F9439A44B015C01E0908608F090870862
:1098D00000918808109189088AE698E09F938F93F9
:1098E0002AE8C22E28E0D22E2A813B814C815D815C
:1098F000C301B2010E9488F70F94350D832D0F9498
:10990000478A0F900F90882309F498C195DE311093
:1099100058C084E090E09093180280931702E09181
:10992000CC08F0E0EE0FFF1FE05DFA4B85919491BB
:1099300040E060E00F943770882359F0E091CC0844
:10994000F0E0EE0FFF1FEC5DF94B859194910F94C1
:109950005D7AE091CC08F0E0EE0FFF1FE652F84B85
:10996000859194910F945D7AE091CC08F0E0EE0F30
:10997000FF1FE258F94B859194910F945D7A82E034
:1099800090E09093180280931702E091CC08F0E0E9
:10999000EE0FFF1FE059F84B859194910E94CC4344
:1099A00041E050E062E080E00F94DA2EE091CC08D4
:1099B000F0E0EE0FFF1FE459F84B859194910F945E
:1099C0005C4180E090E0A0EAB0E480938608909348
:1099D0008708A0938808B093890881E00F948D05CB
:1099E000282E20E030E040E252E460916202709163
:1099F000630280916402909165020F9439A44B0137
:109A00005C01E0908608F09087080091880810912A
:109A100089082091820830918308409184085091F0
:109A2000850860917E0870917F08809180089091F0
:109A30008108EAE6F8E0FF93EF93EAE8CE2EE8E04B
:109A4000DE2E0E9488F70F94350D822D0F948D0520
:109A500082E00F94A00D0F900F9020E030E040EADC
:109A600050E40F9432A48111E5C086E50E94AE3F18
:109A7000882361F0E091480EF091490E8181893090
:109A800039F08F7D41F00E94C43F03C01A8205C0A7
:109A900081E08A8302C091E09A833320B1F00E9472
:109AA000883F0E9465CE0E94B7CF0E948FE4882332
:109AB00009F4C4C087EF9FE00F945DB0803F09F0C8
:109AC000BFC081E00E94DA43BBC08AEF0E94DA4344
:109AD00060E070E088EF9FE00F9489B01982BE01CA
:109AE0006F5F7F4F8A810E945CE13C010E94883F4A
:109AF000212C312CB0EA4B2EB0E45B2E209286084C
:109B000030928708409288085092890820E030E01F
:109B100040E252E4609162027091630280916402BB
:109B2000909165020F9439A44B015C012091820849
:109B300030918308409184085091850860917E0897
:109B400070917F088091800890918108AAE6B8E022
:109B5000BF93AF931AE8C12E18E0D12E8201710194
:109B60000E9488F70F94350D0F900F9077FC47C037
:109B7000198281E990E10E94E1EB0E94D7CD81E05A
:109B80000E945A3F1EDDAE014F5F5F4F6A8181E048
:109B90000E94B1E63C010E94883F209286083092E4
:109BA0008708409288085092890820E030E040E21F
:109BB00052E460916202709163028091640290911C
:109BC00065020F9439A44B015C0120918208309109
:109BD0008308409184085091850860917E087091B7
:109BE0007F088091800890918108AAE6B8E0BF9331
:109BF000AF930E9488F70F94350D0F900F906981F5
:109C0000C3010F941E8C77FC19C086EE0E94DA43C4
:109C10008FE59FE00F945DB0813091F0E091CC082A
:109C2000F0E0EE0FFF1FE85AF74B859194910F94E7
:109C30005D7A06C089E39AE00F945D7A10E001C076
:109C400011E081E00F94E66D812F0F900F900F903F
:109C50000F900F90DF91CF911F910F91FF90EF9098
:109C6000DF90CF90BF90AF909F908F907F906F903C
:109C70005F904F903F902F900895CF93DF938CE1AA
:109C800097E00E945C3DE2E2F6E4C591D491FE01CA
:109C90008491882321F00E94E53F2196F8CF4091DE
:109CA000380E5091390E60913A0E70913B0E4F5F15
:109CB0005F4F6F4F7F4F2AE030E08CE197E00E94CA
:109CC0001B3E8AE00E94E53F0F945B9B6093300847
:109CD000709331088093320890933308E2E8F6E4F9
:109CE000C591D491FE018491882321F00E94E53F23
:109CF0002196F8CF8AE0DF91CF910C94E53FCF9386
:109D0000DF930F945B9B60933008709331088093CE
:109D1000320890933308E091520EF091530EEC5AB2
:109D2000F14F8081813089F4E2E8F6E4C591D49165
:109D3000FE018491882321F00E94E53F2196F8CF0F
:109D40008AE0DF91CF910C94E53FDF91CF910895A8
:109D50008F929F92AF92BF92CF92DF92EF92FF923B
:109D60000F931F93CF93DF9333E6E32E34E0F32E6C
:109D70000EE718E0C9E4D8E04EEFC42E48E0D42E38
:109D8000F70181917F010E94AE3F882319F10E9463
:109D9000DC3F4B015C01F6018081811103C06091C1
:109DA000340801C061E070E080E090E00F94D4A43A
:109DB000F80120813181428153810F9407A79B01D3
:109DC000AC01C501B4010F9459A3688379838A83D8
:109DD0009B8309C0F80180819181A281B38188832E
:109DE0009983AA83BB830C5F1F4F2496FFEFCF1A82
:109DF000DF0A87E6E81684E0F80611F686E40E949A
:109E0000AE3F8823D9F00E94DC3F6B017C01609358
:109E1000390870933A0880933B0890933C0820E0FF
:109E200030E0A9010F9435A6181644F4C0920E0232
:109E3000D0920F02E0921002F0921102DF91CF91C6
:109E40001F910F91FF90EF90DF90CF90BF90AF9058
:109E50009F908F9008957CDF89E40E94AE3F882315
:109E600059F00E94DC3F60933D0870933E08809358
:109E70003F089093400808C010923D0810923E0899
:109E800010923F08109240088AE40E94AE3F882357
:109E900059F00E94DC3F6093410870934208809320
:109EA0004308909344080895109241081092420884
:109EB00010924308109244080895CF92DF92EF92D7
:109EC000FF92CF93DF93EC01BC016C5F7F4F0E9448
:109ED000B54220E030E0A90160913E0270913F025E
:109EE00080914002909141020F9459A36B017C0133
:109EF0009B01AC01688579858A859B850F9432A486
:109F000087FF04C0C886D986EA86FB86C0903202E5
:109F1000D0903302E0903402F0903502A701960110
:109F2000688579858A859B850F9435A6181624F453
:109F3000C886D986EA86FB86DF91CF91FF90EF90A5
:109F4000DF90CF9008952F923F924F925F926F9241
:109F50007F928F929F92AF92BF92CF92DF92EF92B9
:109F6000FF920F931F93CF93DF93CDB7DEB7AB97DD
:109F70000FB6F894DEBF0FBECDBF9F878E87798B5B
:109F8000688B5B8B4A8B3D8B2C8B1F8B0E8BED82F2
:109F9000DC018D909D90AD90BC9040907E085090DB
:109FA0007F086090800870908108DB018D919D9101
:109FB0000D90BC91A02D88879987AA87BB87C090F8
:109FC0008208D0908308E0908408F0908508209162
:109FD0008608309187084091880850918908EA895D
:109FE000FB8960817181828193810F9458A3688F6E
:109FF000798F8A8F9B8F80919110811173C0AE8968
:10A00000BF898D909D90AD90BC90EA89FB89E080DE
:10A01000F18002811381A889B9892D913D914D91DB
:10A020005C91EE85FF856081718182819381FE0163
:10A030003596FF93EF93CC88DD880E9488F7EE85F4
:10A04000FF8580819181A281B38180937E08909366
:10A050007F08A0938008B0938108E889F9898081FE
:10A060009181A281B3818093820890938308A09309
:10A070008408B0938508EA89FB8980819181A28157
:10A08000B3818093860890938708A0938808B09343
:10A090008908EC89FD8980819181A281B3818093B7
:10A0A0008A0890938B08A0938C08B0938D080F902A
:10A0B0000F90AB960FB6F894DEBF0FBECDBFDF9109
:10A0C000CF911F910F91FF90EF90DF90CF90BF90B5
:10A0D000AF909F908F907F906F905F904F903F9048
:10A0E0002F900895A3019201C501B4010F9458A3C4
:10A0F0002B013C0120E030E0A9010F9435A653016B
:10A100004201181624F0B7FAB094B7F8B094A7013A
:10A110009601688579858A859B850F9458A3688701
:10A1200079878A879B8720E030E0A9010F9435A6C4
:10A13000288539854A855B8518160CF05058C5016D
:10A14000B4010F9459A36B017C0120E030E0A90118
:10A150000F9435A618160CF052CF20E030E040EFF7
:10A1600051E4C701B6010F9439A40F941FA40F94B2
:10A17000A1A47D876C87623071050CF440CF2091DB
:10A180008A0830918B0840918C0850918D08AC89D9
:10A19000BD896D917D918D919C910F9458A36C8F89
:10A1A0007D8F8E8F9F8F22242394312C8C859D85CB
:10A1B000AA2797FDA095BA2F88A799A7AAA7BBA7FA
:10A1C000DE011596BF83AE83B101882777FD8095A8
:10A1D000982F0F94D4A46B017C0168A579A58AA55A
:10A1E0009BA50F94D4A49B01AC01C701B6010F94A9
:10A1F00039A46B017C01EE89FF8980809180A28067
:10A20000B3802C8D3D8D4E8D5F8D0F9407A79B01E4
:10A21000AC0160918A0870918B0880918C089091B4
:10A220008D080F9459A369837A838B839C83288D2F
:10A23000398D4A8D5B8DC701B6010F9407A7209118
:10A2400086083091870840918808509189080F94BA
:10A2500059A368A379A38AA39BA3288539854A8536
:10A260005B85C701B6010F9407A720918208309142
:10A27000830840918408509185080F9459A36CA3DA
:10A280007DA38EA39FA3A3019201C701B6010F94E2
:10A2900007A720917E0830917F0840918008509157
:10A2A00081080F9459A3FF81FF932E812F93DE0124
:10A2B00011966D01E8A0F9A00AA11BA12CA13DA156
:10A2C0004EA15FA10E9488F7BFEF2B1A3B0A0F90A7
:10A2D0000F90EC85FD852E163F0609F075CF8FCEC9
:10A2E0004F925F926F927F928F929F92AF92BF92A6
:10A2F000CF92DF92EF92FF920F931F93CF93DF9352
:10A30000CDB7DEB728970FB6F894DEBF0FBECDBF2E
:10A3100089E498E0D2DD0F945B9B609330087093E2
:10A3200031088093320890933308809149089091C6
:10A330004A08A0914B08B0914C088D839E83AF834F
:10A34000B8879C01AD0160917E0870917F08809173
:10A350008008909181080F9432A4811197C0409099
:10A360004D0850904E0860904F0870905008A3011F
:10A370009201609182087091830880918408909185
:10A3800085080F9432A4811181C020E030E040E7BD
:10A3900052E460910E0270910F0280911002909130
:10A3A00011020F9439A44B015C01E0905108F09028
:10A3B000520800915308109154088AE698E09F9340
:10A3C0008F9365E5C62E68E0D62EA30192016D81BC
:10A3D0007E818F8198850E9488F70F900F908091E1
:10A3E000490890914A08A0914B08B0914C0880937D
:10A3F0007E0890937F08A0938008B0938108809195
:10A400004D0890914E08A0914F08B091500880934C
:10A41000820890938308A0938408B0938508809164
:10A42000510890915208A0915308B091540880931C
:10A43000860890938708A0938808B0938908809134
:10A44000550890915608A0915708B09158088093EC
:10A450008A0890938B08A0938C08B0938D08289657
:10A460000FB6F894DEBF0FBECDBFDF91CF911F9125
:10A470000F91FF90EF90DF90CF90BF90AF909F90A3
:10A480008F907F906F905F904F900895E0906A0852
:10A490006091580270915902882777FD8095982F16
:10A4A0000F94D4A420910E0230910F02409110021B
:10A4B000509111020F9407A72EE333EC4EE259E3BB
:10A4C0000F9407A769837A838B839C838E010F5F28
:10A4D0001F4F25E538E041E558E06DE478E089E478
:10A4E00098E031DD7CCF4F925F926F927F928F9296
:10A4F0009F92AF92BF92CF92DF92EF92FF920F9313
:10A500001F93CF93C62FE0916A08F0E0882309F4E7
:10A51000D9C0DF01AA59B74F8C918111AFC1809189
:10A520007E0890917F08A0918008B0918108809367
:10A53000490890934A08A0934B08B0934C08809127
:10A54000820890918308A0918408B0918508809337
:10A550004D0890934E08A0934F08B09350088091F7
:10A56000860890918708A0918808B0918908809307
:10A57000510890935208A0935308B0935408C09088
:10A580008A08D0908B08E0908C08F0908D08C092DB
:10A590005508D0925608E0925708F0925808EE0FEE
:10A5A000FF1FEE0FFF1FEE5BFD4F208131814281C7
:10A5B0005381662349F060912202709123028091B9
:10A5C00024029091250208C0609126027091270212
:10A5D00080912802909129020F9439A49B01AC012B
:10A5E000C701B6010F9459A360938A0870938B0832
:10A5F00080938C0890938D088AE898E00F94CD039F
:10A6000080900E0290900F02A0901002B090110264
:10A6100020E030E040E752E460911E0270911F029A
:10A6200080912002909121020F9407A760930E025F
:10A6300070930F028093100290931102E0916A08C8
:10A64000F0E0EA59F74F81E080834ADE209162080A
:10A6500030916308409164085091650860918608C4
:10A660007091870880918808909189080F9458A369
:10A670007B018C016093860870938708809388081B
:10A680009093890820918208309183084091840832
:10A690005091850860917E0870917F0880918008B4
:10A6A00090918108EAE8CE2EE8E0DE2E0F94580261
:10A6B00017DE80920E0290920F02A0921002B092CA
:10A6C0001102DCC0EA59F74F8081882309F4D6C013
:10A6D00080907E0890907F08A0908008B0908108BC
:10A6E0008092490890924A08A0924B08B0924C0878
:10A6F000409082085090830860908408709085088C
:10A7000040924D0850924E0860924F087092500847
:10A7100060918608709187088091880890918908D7
:10A720006093510870935208809353089093540893
:10A7300000918A0810918B0820918C0830918D0827
:10A7400000935508109356082093570830935808E3
:10A750002091620830916308409164085091650827
:10A760000F9459A37B018C0160938608709387082E
:10A7700080938808909389087AE8C72E78E0D72ECE
:10A78000A3019201C501B4010F94580210916A0807
:10A79000CC2389F020915A0830915B0840915C08E5
:10A7A00050915D08609122027091230280912402F1
:10A7B0009091250210C020915E0830915F08409171
:10A7C0006008509161086091260270912702809183
:10A7D0002802909129020F9459A324E0129FF001BE
:10A7E0001124EE5BFD4F20813181428153810F9412
:10A7F00039A49B01AC0160918A0870918B0880910B
:10A800008C0890918D080F9458A360938A087093D8
:10A810008B0880938C0890938D088AE898E00F94B9
:10A82000CD03C0900E02D0900F02E0901002F09085
:10A83000110220E030E040E752E460911A0270918A
:10A840001B0280911C0290911D020F9407A7609338
:10A850000E0270930F028093100290931102E09108
:10A860006A08F0E0EA59F74F10823ADDC0920E0212
:10A87000D0920F02E0921002F0921102CF911F913C
:10A880000F91FF90EF90DF90CF90BF90AF909F908F
:10A890008F907F906F905F904F900895AF92BF928E
:10A8A000CF92DF92EF92FF920F931F93CF93DF939C
:10A8B000D82F20914108309142084091430850918F
:10A8C000440860913D0870913E0880913F08909146
:10A8D00040080F9442A6C62F172F082FF92E60911B
:10A8E000580270915902882777FD8095982F0F9410
:10A8F000D4A420910E0230910F0240911002509189
:10A9000011020F9407A720E030E040E752E40F94D3
:10A9100039A420E030E048EC52E40F9439A42091AF
:10A920006A082F93DF93FF920F931F93CF935B01DE
:10A930006C01B2E0EB2E01E020E04DE358E069E469
:10A9400078E08EE798E00E94C6ED809149089091EA
:10A950004A08A0914B08B0914C0880937E089093D0
:10A960007F08A0938008B093810880914D08909152
:10A970004E08A0914F08B0915008809382089093A0
:10A980008308A0938408B093850880915108909122
:10A990005208A0915308B091540880938608909370
:10A9A0008708A0938808B0938908809155089091F2
:10A9B0005608A0915708B091580880938A08909340
:10A9C0008B08A0938C08B0938D080F945B9B6093C9
:10A9D00030087093310880933208909333080F90B9
:10A9E0000F900F900F900F900F90DF91CF911F91CC
:10A9F0000F91FF90EF90DF90CF90BF90AF900895B0
:10AA0000CF93DF931F92CDB7DEB77C01EBECF7E07D
:10AA100084918F01882349F069830E94E53F0F5F8D
:10AA20001F4FF80184916981F5CF70E04AE050E052
:10AA30008CE197E00E94493EF8940F94C815179A4C
:10AA400010926F08169A10927008149AE9EFFBE0C2
:10AA500084918F01882339F00E94E53F0F5F1F4FDB
:10AA6000F8018491F7CFECEAF7E405911491F8012D
:10AA70008491882329F00E94E53F0F5F1F4FF7CF95
:10AA80008AE00E94E53FE114F10499F0F701849116
:10AA90008701882339F00E94E53F0F5F1F4FF801BF
:10AAA0008491F7CF8AE00E94E53FC7010E94CC4322
:10AAB00006C0E0E1F7E4859194910F9454307894C6
:10AAC00006E010E00150110951F068EC70E080E000
:10AAD00090E00F948A9B80E00F94186BF3CFF8946A
:10AAE000A895FECFCF93DF930F94C81580911E08D1
:10AAF000811136C081E080931E088091380E9091BC
:10AB0000390EA0913A0EB0913B0E8093340E909383
:10AB1000350EA093360EB093370EE9EFFBE084912B
:10AB2000EF01882331F00E94E53F2196FE018491D8
:10AB3000F8CFE2EAF7E4C591D491FE01849188232D
:10AB400021F00E94E53F2196F8CF8AE00E94E53F80
:10AB5000ECE2F5E485919491DF91CF910D9428304A
:10AB6000DF91CF91089580911E080895FF920F9371
:10AB70001F93CF93DF93EC0180916A0880931F08A5
:10AB800084E50E94AE3F811102C080E06AC00E944D
:10AB9000DC3F0F94A6A4F62E60931F086623A9F34A
:10ABA000E3EFFBE084918F01882339F00E94E53FB9
:10ABB0000F5F1F4FF8018491F7CFCD36D10559F1C2
:10ABC00064F4C836D105A9F0C936D10509F03DC0F5
:10ABD000E0EFF6E4C591D49118C0CA3DD10529F142
:10ABE000CD3DD10509F031C0E0EEF6E4C591D49138
:10ABF00026C0E2EFF6E4C591D491FE01849188234A
:10AC000021F10E94E53F2196F8CF89918823E9F050
:10AC10000E94E53FFACFEEEEF6E4C591D49189911A
:10AC2000882399F00E94E53FFACFE2EEF6E4C59161
:10AC3000D4918991882349F00E94E53FFACF899108
:10AC4000882319F00E94E53FFACF6F2D70E04AE0AB
:10AC500050E08CE197E00E942D3E8AE00E94E53FA3
:10AC600081E0DF91CF911F910F91FF9008954F9256
:10AC70005F926F927F928F929F92AF92BF92CF928C
:10AC8000DF92EF92FF92CF93DF9300D01F92CDB768
:10AC9000DEB72B013C0129833A834B835C838DEE25
:10ACA0009FE00F945DB08F3F01F58EEE9FE00F9413
:10ACB0005DB08F3FD1F48FEE9FE00F945DB08F3F7A
:10ACC000A1F480EF9FE00F945DB08F3F71F440E0FE
:10ACD00050E0BA018DEE9FE00F9481B040E050E06B
:10ACE000BA0181EF9FE00F9481B081EF9FE00F9454
:10ACF00065B04B015C018DEE9FE00F9465B06B0178
:10AD00007C0169817A818B819C812CE330E040E079
:10AD100050E00F9409A9C20ED31EE41EF51EB70120
:10AD2000A6018DEE9FE00F9481B0C301B20128EE21
:10AD300033E040E050E00F9409A9BA01A901480DA1
:10AD4000591D6A1D7B1D81EF9FE00F9481B0109209
:10AD5000C5081092C6081092C7081092C8080F9034
:10AD60000F900F900F90DF91CF91FF90EF90DF90B9
:10AD7000CF90BF90AF909F908F907F906F905F909B
:10AD80004F900895CF92DF92EF92FF9220918E081C
:10AD90002223F1F020E030E040E05FE30F9407A7CA
:10ADA0006B017C0120E030E0A9010F9432A48823DC
:10ADB00079F0A7019601C701B6010F9407A72BED03
:10ADC0003FE049E450E40F9407A79B01AC0104C0A5
:10ADD00020E030E040E85FE360E070E080E89FE37F
:10ADE0000F9439A4FF90EF90DF90CF900895609179
:10ADF0004602709147028091480290914902C2DF59
:10AE00006093420270934302809344029093450200
:10AE10000895CF93DF93EC010F94A21881E05FD1E6
:10AE200080E00F94186B209799F0C233D10540F061
:10AE300062E370E080E090E00F948A9BE297ECCFB1
:10AE4000BE0180E090E00F948A9BC0E0D0E0E4CFA8
:10AE5000DF91CF9108958F929F92AF92BF92CF9240
:10AE6000DF92EF92FF920F931F93CF93DF9315988A
:10AE700081E08093C00882E090E09093BE088093C8
:10AE8000BD08E091CC08F0E0EE0FFF1FE450F94B55
:10AE9000859194910F94283020E030E04CE852E402
:10AEA00060918A0870918B0880918C0890918D0830
:10AEB0000F9459A360938A0870938B0880938C0831
:10AEC00090938D08E0908608F0908708009188089C
:10AED000109189082091820830918308409184085C
:10AEE0005091850860917E0870917F08809180085C
:10AEF00090918108CAE6D8E0DF93CF93812C912C02
:10AF0000E0ECAE2EE0E4BE2EFAE8CF2EF8E0DF2E25
:10AF10000E9488F720E030E048EC51E460918A0814
:10AF200070918B0880918C0890918D080F9459A393
:10AF300060938A0870938B0880938C0890938D0897
:10AF4000E0908608F09087080091880810918908A1
:10AF5000209182083091830840918408509185089F
:10AF600060917E0870917F0880918008909181089F
:10AF7000DF93CF93812C912CA0E8AA2EAFE3BA2EB9
:10AF80000E9488F70F94350D20E030E0A90164EFAE
:10AF900071E084E50F94B39F82E390E03ADF84E5AB
:10AFA0000F94D7A20F900F900F900F908091DD1803
:10AFB000882331F181E00F94E66D82E00F94186BE5
:10AFC000E091CC08F0E0EE0FFF1FE458FB4B8591B9
:10AFD00094910F9428301092BF081092C0081092DC
:10AFE000BE081092BD08DF91CF911F910F91FF9085
:10AFF000EF90DF90CF90BF90AF909F908F9008958B
:10B000008091BF088823B1F2E091CC08F0E0EE0F08
:10B01000FF1FE857F84B8591949141E060E00F9451
:10B02000377091E0811101C090E0CAE6D8E091113B
:10B03000C1CF81E00F94E66D82E00F94186B20E0A1
:10B0400030E048EC51E460918A0870918B0880915F
:10B050008C0890918D080F9459A360938A0870937F
:10B060008B0880938C0890938D08E0908608F09070
:10B0700087080091880810918908209182083091F2
:10B080008308409184085091850860917E087091F2
:10B090007F088091800890918108DF93CF93812C65
:10B0A000912CE0E8AE2EEFE3BE2EFAE8CF2EF8E0CA
:10B0B000DF2E0E9488F70F94350DE091CC08F0E068
:10B0C000EE0FFF1FE857F84B8591949141E060E047
:10B0D0000F9437700F900F9081116CCFAACFCF9241
:10B0E000DF92EF92FF920F931F93CF93C82F80911F
:10B0F0006A0220914A108823F1F080910602882389
:10B10000D1F080914E10811116C080916411909100
:10B110006311891B8F7079F48091080981110BC02C
:10B120008091FB08811107C08091E1189091E2188D
:10B13000089709F067C021110E94FDBC80914E0E56
:10B1400090914F0E039714F40E9435B70F945B9BB8
:10B1500000912C0810912D0820912E0830912F0875
:10B16000C0903008D0903108E0903208F090330859
:10B170006C197D098E099F090617170728073907DB
:10B1800040F4012B022B032B21F064E08BEB94E0C5
:10B1900037DC40910A0250910B0260910C027091D1
:10B1A0000D02452B462B472B21F10F945B9B009101
:10B1B0003008109131082091320830913308601B1B
:10B1C000710B820B930B00910A0210910B022091DC
:10B1D0000C0230910D02061717072807390748F4AB
:10B1E0009091641180916311981303C0CC2309F4EA
:10B1F00070C0CF911F910F91FF90EF90DF90CF9093
:10B200000C94B6F5222309F461C00E9404BD882382
:10B2100009F494CF20E030E04EE353E46091F1175D
:10B220007091F2178091F3179091F4170F9435A64F
:10B230001816CCF40E94FDBC20E030E0A90168EEB5
:10B2400073E084E50F94B39F82E390E0E2DD84E550
:10B250000F94D7A281E08093BF0861E082ED97E070
:10B260000E948DB66BCF80E00F94E66D0F94CF2EC9
:10B2700040E060E08CE598E10E945B39E091CC0809
:10B28000F0E0EE0FFF1FEE54F84B859194910F9470
:10B290005C4142E060E08CE598E10E945B39E0911E
:10B2A000CC08F0E0EE0FFF1FE25BF94B8591949123
:10B2B0000F945C4160ED77E080E090E00F948A9B12
:10B2C0000F94CF2E81E00F94E66D38CF0E94DFBC43
:10B2D00035CF179A10926F08169A10927008149A28
:10B2E00088CF2F923F924F925F926F927F928F9270
:10B2F0009F92AF92BF92CF92DF92EF92FF920F9305
:10B300001F93CF93DF934B015C01CC24CA94DC2CB8
:10B31000760154EC252E57E0352E00EC17E068EE50
:10B32000462E63E0562E612C712C809159088111B4
:10B3300012C12FEFC216D206E206F20651F0F7FC58
:10B340000AC10F945B9B6C197D09683B7B4008F038
:10B3500002C10F945B9B681979098A099B09693EB0
:10B3600073408105910508F470C08091DD1881114A
:10B3700068C0E8ECF7E08491EF01882331F00E9487
:10B38000E53F2196FE018491F8CFE0911F0824E06B
:10B39000E29FF0011124EF50F84E4081518162810B
:10B3A000738121E030E08CE197E00E94E93EF101F9
:10B3B0008491C4ECD7E0882331F00E94E53F2196C8
:10B3C000FE018491F8CF60911F0870E04AE050E0E0
:10B3D0008CE197E00E942D3EF8018491C0ECD7E00B
:10B3E000882331F00E94E53F2196FE018491F8CF39
:10B3F000F7FE03C0C5E6D6E01BC00F945B9B4B0174
:10B400005C01C701B6016854744F8F4F9F4F681994
:10B4100079098A099B09A30192010F9409A9BA012C
:10B42000A9012AE030E08CE197E00E941B3E06C0B3
:10B430008991882319F00E94E53FFACF8AE00E94A3
:10B44000E53F0F945B9B4B015C010F94A21880E0D9
:10B4500046DE80E00F94186BFFEFCF16DF06EF0695
:10B46000FF0609F042C080911D08E0911F08F0E03E
:10B47000EF01CC0FDD1FCC0FDD1FCF50D84EEE0FEC
:10B48000FF1FE750F84E608171818823B9F088274B
:10B4900077FD8095982F0F94D4A420E030E040E809
:10B4A0005FE30F9458A39B01AC01688179818A8185
:10B4B0009B810F9435A687FF49C037CF882777FD3A
:10B4C0008095982F0F94D4A420E030E040E85FE30B
:10B4D0000F9459A39B01AC01688179818A819B817A
:10B4E0000F9432A4181694F520CFF7FC1ECFE091EC
:10B4F0001F08F0E0EF01CC0FDD1FCC0FDD1FCF5098
:10B50000D84EEE0FFF1FE750F84E608171818827FB
:10B5100077FD8095982F0F94D4A49B01AC0168818E
:10B5200079818A819B810F9458A30F94A1A497FFDE
:10B5300007C090958095709561957F4F8F4F9F4F75
:10B5400066307105810591050CF4EFCE0F945B9B7D
:10B550006B017C01EACEDF91CF911F910F91FF909B
:10B56000EF90DF90CF90BF90AF909F908F907F90A3
:10B570006F905F904F903F902F9008950F931F937F
:10B58000CF93DF931F921F92CDB7DEB7BE016F5FDF
:10B590007F4F88EF9FE00F941E2F89819A818156FB
:10B5A000904F803A9F4000F11A821982E7E9F7E054
:10B5B00084918F01882339F00E94E53F0F5F1F4F70
:10B5C000F8018491F7CF8AE00E94E53FBE016F5FEA
:10B5D0007F4F88EF9FE00F940D2F8AE597E00F943F
:10B5E0005D7A81E00F94E66D0F900F90DF91CF911F
:10B5F0001F910F9108952F923F924F925F926F92F9
:10B600007F928F929F92AF92BF92CF92DF92EF92F2
:10B61000FF920F931F93CF93DF93CDB7DEB7CA5836
:10B62000D2400FB6F894DEBF0FBECDBFC958DD4F74
:10B63000688379838A839B83C757D240FE01E75F83
:10B64000FD4F88E2DF011D928A95E9F7E850F2404C
:10B6500080E991E0DF019C011D9221503040E1F72B
:10B66000C75ADD4F19821882C955D240CE01875A78
:10B670009D4F5C014E019FE6891A9EEF990ADE01FB
:10B68000AF51BE4F3D0190EBC92E9FE0D92E23E272
:10B69000E22EF12C00E010E0C359DD4F8882CD5638
:10B6A000D240CD58DD4F9882C357D240B70188278A
:10B6B00077FD8095982F0F94D4A4D3016D937D933B
:10B6C0008D939D933D01F501619171915F018827F3
:10B6D00077FD8095982F0F94D4A4D4016D937D931A
:10B6E0008D939D934D010F5F1F4F0630110559F04B
:10B6F000B501C6010F941E2FB5E0EB0EF11CE2E080
:10B70000CE0ED11CD3CFCF51DE4F288139814A8153
:10B710005B81C15ED140C958DD4F688179818A81E2
:10B720009B81C757D2400F9432A487FD2BC3FE01E3
:10B73000EF51FE4F7F016E01FFE2CF1AFEEFDF0AED
:10B740003E012BEB621A2DEF720AC359DD4F0881BF
:10B75000CD56D240CD58DD4F1881C357D24085E039
:10B7600090E0CF58DD4F99838883C157D240CF589E
:10B77000DD4FA881B981C157D2401197CF58DD4F15
:10B78000B983A883C157D240F70120893189428902
:10B79000538964897589868997890F9458A34B01C9
:10B7A0005C01D80150962D913D914D915C9153973C
:10B7B00054966D917D918D919C9157970F9458A3BC
:10B7C000A50194010F9439A4F60192938293729388
:10B7D00062936F01D301BE92AE929E928E923D0112
:10B7E00004501109B4E0EB1AF108CF58DD4FE8819D
:10B7F000F981C157D240EF2B09F0B9CF6E01FFECB0
:10B80000CF1AFDEFDF0A3E0127E4621A2EEF720A1B
:10B810002E013DE3430E511CCE0101967C0101E057
:10B8200010E0D6018D909D90AD90BC90139714962A
:10B830002D913D914D915C911797C501B4010F94E5
:10B8400059A39B01AC010F9459A3F70164A775A7F5
:10B8500086A797A70130110541F080A691A6A2A660
:10B86000B3A684829582A682B7820F5F1F4FD30151
:10B8700014962D913D914D915C91179718966D916D
:10B880007D918D919C911B970F9458A320E030E0FF
:10B8900040EC50E40F9407A7F20160837183828328
:10B8A0009383F4E0CF0ED11C2CE2E20EF11C34E0C5
:10B8B000630E711C88E2480E511C0530110509F019
:10B8C000B0CF8E010B5A1F4F6E0191E5C90ED11CEE
:10B8D00022242394312C2C0E3D1EA8ED2A0E311C5F
:10B8E000F801B8972081318142815381F80160814C
:10B8F0007181828193810F9439A44B015C01E12C09
:10B90000F12C3601F8E26F1A710826014E0C5F1C0B
:10B91000F301EE0DFF1D2481358146815781C5015C
:10B92000B4010F9407A79B01AC01D20114966D914D
:10B930007D918D919C9117970F9458A3F201648388
:10B94000758386839783F4E0EF0EF11C24E1E21601
:10B95000F104D9F6045D1F4F38E2C30ED11C021565
:10B96000130509F0BDCF1E0185EB280E311C6E01B9
:10B9700091EBC90ED11C3E01A7EE6A1AADEF7A0A0F
:10B9800014E0E12EF12C270100E010E0812C912C35
:10B99000A12CB12CF601E00FF11FD301A00FB11FB4
:10B9A0002D913D914D915C91608171818281938156
:10B9B0000F9407A79B01AC01B401C5010F9459A3D3
:10B9C0004B015C01BFEF4B1A5B0A0C5F1F4FE5E0B8
:10B9D0004E165104F9F69B01AC01D1016D917D9198
:10B9E0008D919C910F9458A3F60120813181428161
:10B9F00053810F9439A4D3016D937D938D939C93C0
:10BA00001397B1E0EB1AF108E8E22E1A3108FCE2D4
:10BA1000CF1AD10824E0621A7108E114F10409F088
:10BA2000B2CFCB50DE4F88819981AA81BB81C55F9F
:10BA3000D140C957DD4F88839983AA83BB83C758F8
:10BA4000D2408E01075F1D4FDE01AF5CBD4FC55870
:10BA5000DD4FB983A883CB57D240C359DD4F28802F
:10BA6000CD56D240CD58DD4F3880C357D240FE016D
:10BA7000EF51FE4FC358DD4FF983E883CD57D240D5
:10BA8000C358DD4FA881B981CD57D240CD90DD900C
:10BA9000ED90FD90C358DD4FB983A883CD57D240B8
:10BAA000C958DD4F288139814A815B81C757D2400F
:10BAB000C701B6010F9432A41816B4F0C358DD4F75
:10BAC000E881F981CD57D240208131814281538173
:10BAD000C958DD4F688179818A819B81C757D240DF
:10BAE0000F9432A41816FCF4CF58DD4F2881398109
:10BAF000C157D2402430310509F01FC1C957DD4F6D
:10BB0000288139814A815B81C758D240C958DD4FAD
:10BB1000688179818A819B81C757D2400F9435A66D
:10BB200018160CF00AC1D80114968D919D910D90B4
:10BB3000BC91A02DC158DD4F88839983AA83BB8314
:10BB4000CF57D240F8014080518062807380C55841
:10BB5000DD4FA881B981CB57D2408D919D910D9039
:10BB6000BC91A02DC359DD4F88839983AA83BB83E1
:10BB7000CD56D240D1018D919D910D90BC91A02DBB
:10BB8000CD57DD4F88839983AA83BB83C358D240A6
:10BB9000A7019601C958DD4F688179818A819B810F
:10BBA000C757D2400F9458A3CD58DD4F688379838F
:10BBB0008A839B83C357D24020E030E040E450E4C6
:10BBC0000F946AA76B017C01A3019201C158DD4F5C
:10BBD000688179818A819B81CF57D2400F9458A385
:10BBE0004B015C0120E030E040EC50E4C359DD4FF4
:10BBF000688179818A819B81CD56D2400F9407A7B5
:10BC00009B01AC01C501B4010F9439A4A7019601B1
:10BC10000F9407A76B017C0120E030E040E05FE378
:10BC2000C301B2010F9407A74B015C01CD58DD4F52
:10BC3000288139814A815B81C357D240CA01B90149
:10BC40000F9407A79B01AC01C501B4010F9407A78E
:10BC50009B01AC01C701B6010F9459A36B017C0194
:10BC6000CD57DD4F288139814A815B81C358D2404D
:10BC7000F10164817581868197810F9458A3C3591E
:10BC8000DD4F288139814A815B81CD56D2400F94A6
:10BC900039A44B015C01C359DD4F288139814A81A8
:10BCA0005B81CD56D240CA01B9010F9459A3A301BB
:10BCB00092010F9407A72B013C01C359DD4F288146
:10BCC00039814A815B81CD56D240C158DD4F6881B0
:10BCD00079818A819B81CF57D2400F9407A79B011E
:10BCE000AC01C301B2010F9459A320E030E040EC55
:10BCF00050E40F9439A49B01AC01C501B4010F9429
:10BD000058A3CD58DD4F288139814A815B81C357C3
:10BD1000D2400F9407A79B01AC01C701B6010F9455
:10BD200059A3CD57DD4F288139814A815B81C358A2
:10BD3000D2400F9459A34B015C01CF58DD4F2881AD
:10BD40003981C157D2402F5F3F4FCF58DD4F3983E4
:10BD50002883C157D2400C5F1F4FC558DD4F8881E3
:10BD60009981CB57D2400496C558DD4F998388837B
:10BD7000CB57D24094E0290E311C2530310509F013
:10BD80007FCE04C0812C912CA12CB12CB401C50113
:10BD9000C657DD4F0FB6F894DEBF0FBECDBFDF91A3
:10BDA000CF911F910F91FF90EF90DF90CF90BF90B8
:10BDB000AF909F908F907F906F905F904F903F904B
:10BDC0002F900895CF92DF92EF92FF926B017C014A
:10BDD0008091F9088823A1F086EA9FE00F945DB076
:10BDE000882371F0C701B60106DC2091F816309166
:10BDF000F9164091FA165091FB160F9439A403C01E
:10BE000060E070E0CB01FF90EF90DF90CF9008955D
:10BE10004F925F926F927F928F929F92AF92BF925A
:10BE2000CF92DF92EF92FF920F931F93CF93DF9306
:10BE3000CDB7DEB728970FB6F894DEBF0FBECDBFE3
:10BE40000F94350D80915802909159029093FD08FE
:10BE50008093FC08E0916A08F0E0EE0FFF1FE750C6
:10BE6000F84E60817181882777FD8095982F0F9417
:10BE7000D4A46093ED087093EE088093EF0890933C
:10BE8000F00880916808909169089093EC0880937D
:10BE9000EB080F945B9B6093D3087093D408809356
:10BEA000D5089093D60880917E0890917F08A09144
:10BEB0008008B091810889839A83AB83BC83809387
:10BEC000DB089093DC08A093DD08B093DE08409077
:10BED0008208509083086090840870908508409292
:10BEE000DF085092E0086092E1087092E2088091C9
:10BEF000860890918708A0918808B09189088D8361
:10BF00009E83AF83B8878093E3089093E408A0935F
:10BF1000E508B093E60860918A0870918B088091DB
:10BF20008C0890918D086093E7087093E8088093DF
:10BF3000E9089093EA0820E030E040E85FE30F94DE
:10BF400058A360938A0870938B0880938C08909311
:10BF50008D088AE698E09F938F93812C912CB8EC02
:10BF6000AB2EB3E4BB2E1AE8C12E18E0D12EED8023
:10BF7000FE800F811885A301920169817A818B81EE
:10BF80009C810E9488F720E030E040EA51E4609113
:10BF900086087091870880918808909189080F948D
:10BFA00059A32B013C010F900F9020E030E042E5B7
:10BFB00053E40F9435A618164CF040928608509220
:10BFC000870860928808709289080CC080E090E031
:10BFD000A2E5B3E48093860890938708A09388082D
:10BFE000B0938908E0908608F0908708009188084F
:10BFF000109189082091820830918308409184082B
:10C000005091850860917E0870917F08809180082A
:10C0100090918108AAE66A2EA8E07A2E7F926F920C
:10C02000812C912CB0E7AB2EB1E4BB2EEAE8CE2EEA
:10C03000E8E0DE2E0E9488F71092FA171092F917A6
:10C040001092FC171092FB171092FE171092FD171A
:10C0500080E090E0A8E4B2E480937E0890937F08AB
:10C06000A0938008B093810880E090E0AEE3B3E451
:10C070008093820890938308A0938408B0938508E6
:10C08000E0908608F0908708009188081091890850
:10C090007F926F92812C912CF8E4AF2EF2E4BF2EA8
:10C0A0009C01AD01C501B4010E9488F71092690896
:10C0B000109268080F900F900F900F9028960FB66F
:10C0C000F894DEBF0FBECDBFDF91CF911F910F91CE
:10C0D000FF90EF90DF90CF90BF90AF909F908F90A8
:10C0E0007F906F905F904F900D94350D0F931F933D
:10C0F000CF93DF9300D01F92CDB7DEB7E0916A08EF
:10C1000084E0E89FF0011124EF50F84E4081518106
:10C1100062817381E7E5F7E084918F01882379F0EC
:10C1200049835A836B837C830E94E53F0F5F1F4FD7
:10C13000F80184917C816B815A814981EFCF22E0A3
:10C1400030E08CE197E00E94E93EE3E5F7E084917E
:10C150008F01882339F00E94E53F0F5F1F4FF801E0
:10C160008491F7CF60916A0870E04AE050E08CE17A
:10C1700097E00E942D3EEFE4F7E084918F01882341
:10C1800039F00E94E53F0F5F1F4FF8018491F7CF10
:10C190004091E1175091E2176091E3177091E41715
:10C1A00021E030E08CE197E00E94E93E8AE00F90C8
:10C1B0000F900F900F90DF91CF911F910F910C94E2
:10C1C000E53F2F923F924F925F926F927F928F92B4
:10C1D0009F92AF92BF92CF92DF92EF92FF920F9316
:10C1E0001F93CF93DF93CDB7DEB7C755D1090FB6F5
:10C1F000F894DEBF0FBECDBF82E090E090931802AE
:10C20000809317028BE693E00E94463F8823B1F0AB
:10C210008091480E9091490E6AE270E005960F9465
:10C22000F9AC009711F0DC011C928091480E9091BE
:10C23000490E05960F941B300C94E48780E793E039
:10C240000E94463F882309F4A2C186E793E00E943A
:10C25000463F882391F08091DD18882311F40C94D7
:10C26000E4870F945B9B60930209709303098093AA
:10C270000409909305090C94E4878BE793E00E94EE
:10C28000463F882361F06091C9087091CA084AE06E
:10C2900050E08CE197E00E94573E0C94E4878FE7D2
:10C2A00093E00E94463F882309F442C003E813E06C
:10C2B000F80181918F01882319F00E94E53FF8CFA2
:10C2C0008091AA089091AB082CE3289FB001299F88
:10C2D000700D11244AE050E08CE197E00E942D3E61
:10C2E00067E873E08CE197E00E94383E0CE813E0C9
:10C2F000D8018D918D01882319F00E94E53FF8CF78
:10C300008091AC089091AD082CE3289FB001299F43
:10C31000700D11244AE050E08CE197E00E942D3E20
:10C3200067E873E08CE197E00E94383E0C94E48764
:10C3300082E993E00E94463F8823C1F08091DD1896
:10C34000882361F06091DB187091DC184AE050E0BE
:10C350008CE197E00E94493E0C94E48765E973E024
:10C360008CE197E00E94383E0C94E48787EA93E0E2
:10C370000E94463F882369F16091480E7091490EF2
:10C380006D5F7F4F21E041E086E099E00E9466AA60
:10C3900080916A0B90916B0BA0916C0BB0916D0B1F
:10C3A0008093170C9093180CA093190CB0931A0C4F
:10C3B00082E69BE00E94599A8C010E94E53F0A3078
:10C3C000110531F760E086E099E00E9405AA0C941F
:10C3D000E4878AEA93E00E94463F882399F00E940E
:10C3E000274B81E08093CB086091480E7091490EF5
:10C3F0006C5F7F4F21E040E086E099E00E9466AAF2
:10C400000C94E4878EEA93E00E94463F8823D9F19A
:10C410008091DD18882309F4A1CF1092A10701EBC8
:10C4200013E0F80181918F01882319F00E94E53F04
:10C43000F8CF00E010E0FF24F39480919D079091E5
:10C440009E0720919F073091A007821B930B8F7747
:10C450009927892B69F08CE197E00E94403DF0928A
:10C46000A1070E94E53F0F5F1F4F1092A107E5CF84
:10C470000331110514F381E08093A1078AE00E9443
:10C48000E53F0C94E48784EB93E00E94463F8823C9
:10C4900079F008EB13E0D8018D918D01882319F014
:10C4A0000E94E53FF8CF8AE00E94E53F0C94E487C4
:10C4B00082EC93E00E94463F882351F006EC13E0A3
:10C4C000F80181918F01882371F30E94E53FF8CF35
:10C4D00085EE93E00E94463F882321F00F94B92F08
:10C4E0000C94E4878AEE93E00E94463F882341F053
:10C4F00060E070E088EF9FE00F940D2F0C94E487CC
:10C500008DEE93E00E94463F882359F06DEE73E074
:10C510008CE197E00E94383E40E052EC61E070E030
:10C5200010C088EF93E00E94463F882381F068EFB7
:10C5300073E08CE197E00E94383E40E054E961E10D
:10C5400070E08CE197E00E94C53C0C94738D84E010
:10C5500094E00E94463F882361F00F945B9B6093B8
:10C56000F5087093F6088093F7089093F8080C94F8
:10C57000E48789E094E00E94463F882311F40C94FC
:10C58000E48761E080E00E9430440C94E4878EE50B
:10C590000E94AE3F81110C94E48787E40E94AE3F75
:10C5A000882311F40C94AC710E94DC3F0F94A1A479
:10C5B0006C34710509F410C47CF56430710509F41C
:10C5C00008C154F46230710509F4EBC00CF0F5C0F9
:10C5D00077FF77C00C9498716C31710509F450C1E4
:10C5E0007CF46A30710509F445C16B30710511F0B6
:10C5F0000C94987160E080E00E9473520C94E48780
:10C600006E31710509F430C36B34710511F00C946F
:10C61000987108E210E0CDC36835710511F40C94EF
:10C62000E4870CF56135710511F40C94687064F4BD
:10C630006F34710511F40C947F6B6035710511F442
:10C640000C94BE6B0C9498716635710511F40C94C2
:10C6500018716735710511F00C94987181E00E9492
:10C66000DA430C94E4876C35710511F40C94217154
:10C670007CF46A35710511F40C941D716B357105EC
:10C6800011F00C94987181E0809334080C94E48745
:10C690006236710511F40C9483716336710511F0E3
:10C6A0000C9498711092DD180F94BE2F6091DD18D4
:10C6B00084EC9FE00F946FB082E00F94186B0C94A1
:10C6C000E48780911E0881110C94E4870E94A84E93
:10C6D0006091C5087091C6088091C7089091C808FC
:10C6E0000F94D2A46B017C0140908A0850908B0873
:10C6F00060908C0870908D08809055089090560836
:10C70000A0905708B0905808A5019401C301B20148
:10C710000F9458A320E030E048EC52E40F9407A7B0
:10C720009B01AC01C701B6010F9435A61816E4F4BD
:10C73000A3019201C501B4010F9458A320E030E099
:10C7400048EC52E40F9407A79B01AC01C701B60166
:10C750000F9459A30F94A6A46093C5087093C608BC
:10C760008093C7089093C808809167088823A9F030
:10C7700088E50E94AE3F811110C089E50E94AE3F5E
:10C7800081110BC08AE50E94AE3F811106C085E48D
:10C790000E94AE3F81110C94ED870E9470510C9461
:10C7A000E48780911E0881110C94E4870E942B4F2E
:10C7B00081E00E944E540C94E48780911E08811100
:10C7C0000C94E4870E942B4F80E00E944E540C94FE
:10C7D000E48780E50E94AE3F882339F00E94DC3F69
:10C7E0000F94A6A46B017C0103C0C12CD12C76014F
:10C7F00083E50E94AE3F882361F00E94DC3F20E089
:10C8000030E04AE754E40F9407A70F94A6A46B0105
:10C810007C01C114D104E104F10431F0EEEBF7E442
:10C82000859194910F9428300F94350D0F945B9B54
:10C830004B015C018C0C9D1CAE1CBF1C0F945B9BC0
:10C8400060933008709331088093320890933308D6
:10C850000F945B9B681579058A059B0510F00C9475
:10C86000E4870F94A21880E00E946F5880E00F9434
:10C87000186BEECF60E081E00E9473520C94E48765
:10C880000F94350D81E08093FA0888E50E94AE3F51
:10C89000182F89E50E94AE3F082F8AE50E94AE3F1F
:10C8A000782E101308C0181711F0012F04C0772438
:10C8B000739401E011E00E9410CE609091101092EC
:10C8C000911082E00F94A00D609386087093870802
:10C8D000809388089093890871100E9417EB40910B
:10C8E0000E0250910F02609110027091110240935C
:10C8F0003508509336086093370870933808809154
:10C900005802909159029093FD088093FC0884E6A8
:10C9100090E090935902809358020F945B9B609330
:10C92000300870933108809332089093330881E087
:10C930000F948D0580E1EEE7F8E0A9E4B8E00190FE
:10C940000D928A95E1F710920E0210920F0210924A
:10C95000100210921102112321F080E090E00E9459
:10C96000C946002321F081E090E00E94C94688E595
:10C970000E94AE3F882341F00E94D13F672B682B75
:10C98000692B11F00C941C8889E50E94AE3F882326
:10C9900041F00E94D13F672B682B692B11F00C945A
:10C9A0003288772009F4F1C080916F08882321F044
:10C9B00080917008811108C080E090E00E94C94613
:10C9C00081E090E00E94C9460E9465CEEFE2F9E462
:10C9D00085919591A591B49189839A83AB83BC830A
:10C9E000EBE2F9E485919591A591B4918F8F98A38D
:10C9F000A9A3BAA32DE438E049E458E0BE016F5F73
:10CA00007F4FCE014F960E94FB410E94D7CD20E080
:10CA100030E040E850EC60914D0870914E088091F4
:10CA20004F08909150080F9432A487FF0CC080E00B
:10CA300090E0A0E8B0EC80934D0890934E08A0934E
:10CA40004F08B093500880E090E0A0EAB0E48093F3
:10CA5000510890935208A0935308B093540820E0D3
:10CA600030E040E251E46091620270916302809193
:10CA70006402909165020F9439A460930E02709342
:10CA80000F02809310029093110210928608109268
:10CA90008708109288081092890880E00F948D050D
:10CAA000E0908608F0908708009188081091890826
:10CAB0002091820830918308409184085091850824
:10CAC00060917E0870917F08809180089091810824
:10CAD000FAE8CF2EF8E0DF2E0F94580280900E0275
:10CAE00090900F02A0901002B0901102E0905108B7
:10CAF000F0905208009153081091540820914D086D
:10CB000030914E0840914F0850915008609149086B
:10CB100070914A0880914B0890914C08EAE6F8E041
:10CB2000FF93EF93A5E5CA2EA8E0DA2E0E9488F7BE
:10CB30000F94350D8091490890914A08A0914B08B7
:10CB4000B0914C0880937E0890937F08A093800852
:10CB5000B093810880914D0890914E08A0914F08A4
:10CB6000B09150088093820890938308A093840822
:10CB7000B093850881E00F948D050F94750582E0D0
:10CB800090E00E94C9460F900F908AE50E94AE3F48
:10CB9000882341F00E94D13F672B682B692B11F04D
:10CBA0000C944888E0908608F090870800918808E7
:10CBB000109189082091820830918308409184085F
:10CBC0005091850860917E0870917F08809180085F
:10CBD00090918108EAE8CE2EE8E0DE2E0F9458020C
:10CBE00080E00F948D058091350890913608A091D2
:10CBF0003708B091380880930E0290930F02A093EB
:10CC00001002B09311028091FC089091FD0890935E
:10CC10005902809358020F945B9B60933008709385
:10CC2000310880933208909333080F9475050E9461
:10CC300065CE0E94B7CF88E50E94AE3F81110C946B
:10CC4000B08789E50E94AE3F81110C94B08787E5DB
:10CC50000E94AE3F81110C94B0878AE50E94AE3FDE
:10CC600081110C94B08786C50F94350D81E00E9428
:10CC70005A3F8091620290916302A0916402B09148
:10CC8000650280930E0290930F02A0931002B0935E
:10CC9000110220E030E043E060E070E080E291ECDF
:10CCA0000E9446D0E6E5F8E405911491F8018491DC
:10CCB000882329F00E94E53F0F5F1F4FF7CFE4E381
:10CCC000FAE084918F01882339F00E94E53F0F5FDD
:10CCD0001F4FF8018491F7CF40917E0850917F0853
:10CCE000609180087091810825E030E08CE197E048
:10CCF0000E94E93EEFE2FAE084918F01882339F047
:10CD00000E94E53F0F5F1F4FF8018491F7CF4091DC
:10CD1000820850918308609184087091850825E00D
:10CD200030E08CE197E00E94E93EEAE2FAE084918B
:10CD30008F01882339F00E94E53F0F5F1F4FF801F4
:10CD40008491F7CF409186085091870860918808B8
:10CD50007091890825E030E08CE197E00E94E93E7F
:10CD6000E8E2FAE084918F01882339F00E94E53FE0
:10CD70000F5F1F4FF8018491F7CF0E94883F0C94FA
:10CD8000E487B801882777FD8095982F0F94D4A465
:10CD90000E94FB5AAB01BC0122E030E08CE197E03D
:10CDA0000E94EA3E0F5F1F4F0F36110511F40C94DD
:10CDB000E4874AE050E0B8018CE197E00E942D3E04
:10CDC00059E5E52E56E0F52ED7018D917D0188239A
:10CDD000C1F20E94E53FF8CFEEE0F5E48591949131
:10CDE0000F945D7AE091CC08F0E0EE0FFF1FE05D5C
:10CDF000FA4B8591949140E060E00F94377088235E
:10CE000059F0E091CC08F0E0EE0FFF1FEC5DF94B1C
:10CE1000859194910F945D7A80916F08882341F0F9
:10CE200080917008882321F080917108811109C0D8
:10CE30000E9428B761E081E29AE00E948DB60C94CE
:10CE4000E48781E090E09093180280931702E3E07A
:10CE5000FAE084918F01882339F00E94E53F0F5F4B
:10CE60001F4FF8018491F7CF8AE00E94E53F1A82B4
:10CE70001982C090EB17D090EC17E090ED17F0906E
:10CE8000EE1720E030E040EA50E4C701B6010F940D
:10CE900039A40F94A1A445E0469F9001479F300D0F
:10CEA0001124B901882777FD8095982F0F94D4A479
:10CEB0002B013C0120E030E04CE052E40F9432A41E
:10CEC00087FF06C0412C512C2CE0622E22E4722EEA
:10CED000A7019601C301B2010F9432A487FF0AC0D3
:10CEE00020E030E040EA50E4C301B2010F9459A3BE
:10CEF0002B013C01EFEEF9E084918F01882339F09A
:10CF00000E94E53F0F5F1F4FF8018491F7CF22E0A9
:10CF100030E0B301A2018CE197E00E94EA3E20E0FC
:10CF200030E040EF51E4C301B2010F9458A320E078
:10CF300030E04CE852E40F9459A30F94A1A47093ED
:10CF4000F8176093F71784E090E09093BE08809301
:10CF5000BD0881E090E09093BC088093BB08E0910D
:10CF6000CC08F0E0EE0FFF1FE45EFA4B8591949140
:10CF700021E0892B09F420E02093C00880E090E0B4
:10CF8000A0EAB1E480937E0890937F08A093800884
:10CF9000B093810880E090E0A0E7B2E4809382083B
:10CFA00090938308A0938408B09385088AE999E94F
:10CFB000A9E1BEE38093860890938708A093880830
:10CFC000B09389088AE698E09F938F93812C912CE7
:10CFD00018E4A12E12E4B12E0AE8C02E08E0D02EEB
:10CFE0001AE9E12E19E9F12E09E11EE320E030E013
:10CFF00040E752E460E070E080EA91E40E9488F744
:10D000000F94350D0F900F90A30192016091EB17D3
:10D010007091EC178091ED179091EE170F9432A458
:10D0200087FF06C088EE93E00E9409575FD8ECCFD7
:10D0300060E086EA9FE00F946FB080E090E0A0EAA5
:10D04000B0E48093860890938708A0938808B093F3
:10D05000890820918208309183084091840850917A
:10D06000850860917E0870917F088091800890917A
:10D070008108EAE6F8E0FF93EF93812C912CE8E435
:10D08000AE2EE2E4BE2EFAE8CF2EF8E0DF2EE12C41
:10D09000F12C00EA10E40E9488F7EBE2F9E48591B4
:10D0A0009591A591B49180937E0890937F08A09369
:10D0B0008008B0938108EFE2F9E42591359145911C
:10D0C00054912093820830938308409384085093AE
:10D0D0008508E0908608F0908708009188081091F4
:10D0E000890860917E0870917F08809180089091F6
:10D0F0008108EAE6F8E0FF93EF93812C912CB8E4E5
:10D10000AB2EB2E4BB2E0E9488F70F94350D20E0C1
:10D1100030E043E060E070E080E89FEB0E9446D0A2
:10D120008091860890918708A0918808B09189081D
:10D130008AAF9BAFACAFBDAFEEEEF9E084910F903C
:10D140000F900F900F908F01882339F00E94E53FD8
:10D150000F5F1F4FF8018491F7CF8AE00E94E53FEF
:10D16000E7EEF9E084918F01882339F00E94E53FD2
:10D170000F5F1F4FF8018491F7CF409186085091BF
:10D180008708609188087091890822E030E08CE17E
:10D1900097E00E94E93EE6EEF9E084918F01882352
:10D1A00039F00E94E53F0F5F1F4FF8018491F7CFE0
:10D1B0008AE00E94E53F2EEA222E2FE0322E33E253
:10D1C000E32EF12C0FEF1FEFB701882777FD809535
:10D1D000982F0F94D4A44B015C01EFEDF9E08491FA
:10D1E0006F01882341F00E94E53FFFEFCF1ADF0A6D
:10D1F000F6018491F6CF4AE050E0B8016E5F7F4FB0
:10D200008CE197E00E942D3EE2EDF9E084916F0100
:10D21000882341F00E94E53FFFEFCF1ADF0AF601B5
:10D220008491F6CF8AE00E94E53FEEEBF9E084912D
:10D230006F01882341F00E94E53FFFEFCF1ADF0A1C
:10D24000F6018491F6CF4AE050E0B7018CE197E017
:10D250000E942D3EEFEAF9E084916F01882341F0AE
:10D260000E94E53FFFEFCF1ADF0AF6018491F6CF67
:10D270004AE050E060E070E08CE197E00E942D3ED3
:10D28000EEEAF9E084916F01882341F00E94E53FC6
:10D29000FFEFCF1ADF0AF6018491F6CF8AE00E94F1
:10D2A000E53F0F3FFFEF1F0731F0BE016F5F7F4F7C
:10D2B000C1010F940D2FA5019401C301B2010F9478
:10D2C00032A4181664F40F5F1F4F25E0E20EF11C24
:10D2D00032E0230E311C0530110509F075CF3801FD
:10D2E00067E2661A68EF760A660C771C280183E00D
:10D2F000480E511C85E0809FD001819FB00D112404
:10D30000212C312C9D96B9AFA8AFC2010297059789
:10D310000CF0BCC168AD79AD620D731D882777FD37
:10D320008095982F0F94D4A422966CAF7DAF8EAFCA
:10D330009FAF2297E7EAF9E084918F01882339F0C3
:10D340000E94E53F0F5F1F4FF8018491F7CF4AE03D
:10D3500050E0B2018CE197E00E942D3EE4EAF9E052
:10D3600084918F01882339F00E94E53F0F5F1F4FA2
:10D37000F8018491F7CF8AE00E94E53F5092BC0803
:10D380004092BB0820E030E040EF51E422966CADC3
:10D390007DAD8EAD9FAD22970F9458A320E030E075
:10D3A00040E251E40F9407A720E030E040EA50E467
:10D3B0000F9439A420E030E048E452E40F9459A3DC
:10D3C0000F94A1A47093F8176093F71780E090E092
:10D3D000A0EAB1E480937E0890937F08A093800830
:10D3E000B093810880E090E0A0E7B2E480938208E7
:10D3F00090938308A0938408B09385088AE999E9FB
:10D40000A9E1BEE38093860890938708A0938808DB
:10D41000B0938908AAE6B8E0BF93AF93812C912C12
:10D42000B8E4AB2EB2E4BB2E1AE8C12E18E0D12E20
:10D430001AE9E12E19E9F12E09E11EE320E030E0BE
:10D4400040E752E460E070E080EA91E40E9488F7EF
:10D450000F94350D0F900F9022962CAD3DAD4EAD33
:10D460005FAD22976091EB177091EC178091ED17EB
:10D470009091EE170F9432A487FF07C088EE93E0D7
:10D480000E9409570E947660E7CF80E090E0A0EA12
:10D49000B0E48093860890938708A0938808B0939F
:10D4A0008908209182083091830840918408509126
:10D4B000850860917E0870917F0880918008909126
:10D4C0008108AAE6B8E0BF93AF93812C912C08E4C1
:10D4D000A02E02E4B02EEAE8CE2EE8E0DE2EE12C0B
:10D4E000F12C00EA10E40E9488F7EBE2F9E4859160
:10D4F0009591A591B49180937E0890937F08A09315
:10D500008008B0938108EFE2F9E4259135914591C7
:10D510005491209382083093830840938408509359
:10D520008508E0908608F09087080091880810919F
:10D53000890860917E0870917F08809180089091A1
:10D540008108AAE6B8E0BF93AF93812C912CA8E4A0
:10D55000AA2EA2E4BA2E0E9488F70F94350D20E07F
:10D5600030E043E060E070E080E89FEB0E9446D04E
:10D570002AAD3BAD4CAD5DAD6091860870918708DA
:10D5800080918808909189080F9458A32091F816EB
:10D590003091F9164091FA165091FB160F9407A797
:10D5A0000F94A1A47A836983E3EAF9E084910F9050
:10D5B0000F900F900F908F01882339F00E94E53F64
:10D5C0000F5F1F4FF8018491F7CF8AE00E94E53F7B
:10D5D000EFE8F9E084918F01882339F00E94E53F5C
:10D5E0000F5F1F4FF8018491F7CF4091EB175091D7
:10D5F000EC176091ED177091EE1722E030E08CE1AE
:10D6000097E00E94E93EE0E8F9E084918F018823E9
:10D6100039F00E94E53F0F5F1F4FF8018491F7CF6B
:10D620002AAD3BAD4CAD5DAD609186087091870829
:10D6300080918808909189080F9458A3AB01BC0190
:10D6400022E030E08CE197E00E94E93EEFE7F9E06C
:10D6500084918F01882339F00E94E53F0F5F1F4FAF
:10D66000F8018491F7CF8AE00E94E53FBE016F5F29
:10D670007F4FC3010F940D2FF2E06F0E711C2FEF3F
:10D68000421A520A35E0230E311C3FCE1092BE08DA
:10D690001092BD081092C00861E086EA9FE00F94E6
:10D6A0006FB0E0E4F9E084918F01882339F00E94A3
:10D6B000E53F0F5F1F4FF8018491F7CF8AE00E948A
:10D6C000E53F179A10926F08169A10927008149AF4
:10D6D0001092F8171092F717E091CC08F0E0EE0FD7
:10D6E000FF1FE85EFA4B859194910F945D7A81E07B
:10D6F0000F94E66D82E00F94186B0C94E4870FEFA3
:10D7000010E0BDE3CB2EB9E0DB2E10936908009347
:10D710006808A4E6EA2EF12C84E690E00E940957FE
:10D72000F1E0EF1AF108C1F74AE050E0B8018CE1EE
:10D7300097E00E942D3EF6018491FDE3EF2EF9E083
:10D74000FF2E882341F00E94E53FFFEFEF1AFF0A0A
:10D75000F7018491F6CF6091AC087091AD084AE072
:10D7600050E08CE197E00E94493E0550110969F6AE
:10D770000C94E4870F94350D1092FA0881E08093A1
:10D78000CE0886E50E94AE3F882359F0E091480E0E
:10D79000F091490E8181893021F08F7D11F00E9436
:10D7A000C43F20916F088091E1189091E2182223E4
:10D7B00041F020917008222321F02091710821115D
:10D7C0000FC0029749F00E9428B761E086E399E014
:10D7D0000E948DB60C94E4871092CE080C94E487D6
:10D7E0001092A207029721F41092CE080C94E487BD
:10D7F000F091C0082896FFAF28972091BD0830917E
:10D80000BE082A963FAF2EAF2A978091BB08909111
:10D81000BC082C969FAF8EAF2C9781E08093C008F8
:10D8200081E090E09093BE088093BD0883E190E092
:10D830009093BC088093BB0881E00F94186B81E93A
:10D8400090E10E94E1EB0E9417EB80E090E0A0EAFB
:10D85000B0E48093860890938708A0938808B093DB
:10D86000890820E030E040E752E460916202709164
:10D87000630280916402909165020F9439A44B0178
:10D880005C01209182083091830840918408509176
:10D89000850860917E0870917F0880918008909142
:10D8A0008108EAE6F8E0FF93EF931AE8C12E18E04A
:10D8B000D12EE12CF12C00EA10E40E9488F7EBE273
:10D8C000F9E485919591A591B49180937E08909308
:10D8D0007F08A0938008B0938108EFE2F9E4859176
:10D8E0009591A591B4918093820890938308A09319
:10D8F0008408B093850862E878E08EE798E00E949B
:10D90000B54220E030E040EF51E460915A0270915E
:10D910005B0280915C0290915D020F9439A44B01EF
:10D920005C01E0908608F0908708009188081091CB
:10D930008908209182083091830840918408509191
:10D94000850860917E0870917F0880918008909191
:10D950008108EAE6F8E0FF93EF930E9488F70F94BE
:10D96000350D20E030E040EA51E460915A027091B8
:10D970005B0280915C0290915D020F9439A40F9438
:10D98000A1A48B0120E030E040E252E46091620209
:10D990007091630280916402909165020F9439A4A2
:10D9A0000F94A1A47B010E94C3CD23968FAF239730
:10D9B00080E00E945A3F0F900F900F900F90ABE2C3
:10D9C000B9E4BBAFAAAF212C312CC701AA2797FD20
:10D9D000A095BA2F60968CAF9DAFAEAFBFAF6097EA
:10D9E000C801AA2797FDA095BA2F64968CAF9DAF6A
:10D9F000AEAFBFAF6497C10163E070E00F94F6A8CB
:10DA00007FAF6EAF99AF88AF60FF06C0A2E0B0E015
:10DA1000A81BB90BB9AFA8AF2396BFAD2397BB2303
:10DA200079F12114310461F18EAD9FAD880F991FFA
:10DA3000EEADFFAD8E0F9F1F28AD39AD820F931F46
:10DA4000880F991F8D53904F0F946AB0BC0188279F
:10DA500077FD8095982F0F94D4A42AE037ED43E208
:10DA60005CE30F9407A7209192103091931040919E
:10DA70009410509195100F9459A32B013C0103C0B1
:10DA8000412C512C320180E090E0A0EAB0E4809378
:10DA9000860890938708A0938808B09389086096B9
:10DAA0006CAD7DAD8EAD9FAD60970F94D4A42796DD
:10DAB0006CAF7DAF8EAF9FAF2797209182083091DA
:10DAC0008308409184085091850860917E08709188
:10DAD0007F088091800890918108AAE6B8E0BF9302
:10DAE000AF9327968CAC9DACAEACBFAC2797EAE861
:10DAF000CE2EE8E0DE2EE12CF12C00EA10E40E94AC
:10DB000088F70F94350DEAADFBAD85919591A59100
:10DB1000B49180937E0890937F08A0938008B0937F
:10DB20008108EAADFBAD349685919591A591B491AC
:10DB30008093820890938308A0938408B09385080B
:10DB400062E878E08EE798E00E94B54264966CAD9A
:10DB50007DAD8EAD9FAD64970F94D4A44B015C0155
:10DB6000E0908608F0908708009188081091890855
:10DB70002091820830918308409184085091850853
:10DB800060917E0870917F08809180089091810853
:10DB9000AAE6B8E0BF93AF930E9488F70F94350DC3
:10DBA0000F900F900F900F902396FFAD2397FF23B8
:10DBB00061F02114310449F020E030E040E85FE3F7
:10DBC000C301B2010F9458A304C060E070E080E28A
:10DBD00091EC20E030E043E00E9446D0811108C083
:10DBE000E091CC08F0E0EE0FFF1FE05DF74B1FC0A7
:10DBF000C0908608D0908708E0908808F090890847
:10DC0000A701960160E070E080EA90E40F9458A3C9
:10DC10002DEC3CEC4CEC5DE30F9432A487FF0AC082
:10DC2000E091CC08F0E0EE0FFF1FE45DF74B65904C
:10DC3000749066C023962FAD23972223B9F0A701D5
:10DC40009601C301B2010F9458A39F7720E030E002
:10DC500040E85FE30F9435A6181644F4E091CC0831
:10DC6000F0E0EE0FFF1FEC5CF74BE1CF6091EB179C
:10DC70007091EC178091ED179091EE170E94E25E83
:10DC80009B01AC01A7E08EAD9FADA89F8001A99F2D
:10DC9000100D1124E8ADF9AD0E0F1F1F000F111F5D
:10DCA000000F111F0F561F4E609186087091870854
:10DCB00080918808909189080F9458A3D8011196F3
:10DCC0006D937D938D939C9314978091BB08909155
:10DCD000BC0801979093BC088093BB08BFEF2B1A38
:10DCE0003B0A81E00F94186BEAADFBAD3896FBAFB1
:10DCF000EAAFF9E02F16310409F07DCE612C712CCA
:10DD000080E090E0A0EAB0E48093860890938708D2
:10DD1000A0938808B09389082091820830918308E5
:10DD2000409184085091850860917E0870917F0829
:10DD30008091800890918108EAE6F8E0FF93EF93E4
:10DD400027968CAC9DACAEACBFAC2797EAE8CE2E44
:10DD5000E8E0DE2EE12CF12C00EA10E40E9488F7C6
:10DD60000F94350D0F900F9029E02216310421F009
:10DD700060E0C3010C94C3770E94883F0E94FFEAD1
:10DD800080EC9FE00F945DB0A82ECE0101963C017F
:10DD9000B12C52E5952E66E4862E9CE499839A82F6
:10DDA0008B8282E48C83D3018D913D010E94AE3F32
:10DDB000882319F00E94D13F1DC0B1E0AB1231C1E0
:10DDC000BB1528F0B11009C08FEB9FE00BC0E2E05B
:10DDD000BE1206C08DEB9FE005C08EEB9FE002C037
:10DDE0008CEB9FE00F945DB0682F772767FD7095EF
:10DDF000872F972F611571058105910509F411C1D0
:10DE00000F94D4A42FE632E143E85AE30F9407A716
:10DE10006B017C019F7727E139ED4EEC5DE30F94B8
:10DE200035A618160CF033C0E9EFFBE084918F01A2
:10DE3000882339F00E94E53F0F5F1F4FF80184915E
:10DE4000F7CFE2E1F9E084918F01882339F00E9455
:10DE5000E53F0F5F1F4FF8018491F7CF22E030E0DC
:10DE6000B701A6018CE197E00E94E93EE9E0F9E004
:10DE700084918F01882339F00E94E53F0F5F1F4F87
:10DE8000F8018491F7CF8AE00E94E53FCAC0F2E032
:10DE9000BF1609F469C023E0B21609F494C031E05A
:10DEA000B31689F120E030E040E05FE3C701B6013E
:10DEB0000F9407A71B012C0102E910E1A2019101B7
:10DEC000D80114966D917D918D919C9117970F9427
:10DED00059A3F8016483758386839783A70196010C
:10DEE00060817181828193810F9459A3D8016D93D0
:10DEF0007D938D939C931397045E1F4FB0E1063E74
:10DF00001B07E1F68EC020E030E040E05FE3C70190
:10DF1000B6010F9407A71B012C0106E910E1A2012D
:10DF20009101F80160817181828193810F9459A3DD
:10DF3000D8016D937D938D939C931397A7019601C0
:10DF400014966D917D918D919C9117970F9459A383
:10DF5000F8016483758386839783045E1F4FF0E125
:10DF60000A3E1F07E1F65DC020E030E040E05FE3DD
:10DF7000C701B6010F9407A71B012C0102E910E1AC
:10DF8000A2019101D8015C966D917D918D919C913A
:10DF90005F970F9459A3F801648F758F868F978FC1
:10DFA000A701960160817181828193810F9459A3A9
:10DFB000D8016D937D938D939D938D01B0E10E39C2
:10DFC0001B07F1F62EC020E030E040E05FE3C70120
:10DFD000B6010F9407A71B012C010EEA10E1A20164
:10DFE0009101F80160817181828193810F9459A31D
:10DFF000D8016D937D938D939D938D01A70196011B
:10E0000058966D917D918D919C915B970F9459A33A
:10E01000F801608F718F828F938FF0E10A3B1F07A9
:10E02000F1F6B39424E0B212B8CE81E990E10E94F7
:10E03000FCEB81E0809391100E9429E4E0916A0852
:10E0400034E0E39FF0011124EF50F84E20E030E07F
:10E050004EE353E460817181828193810F9435A6F0
:10E06000181694F48091F908882371F086EA9FE0ED
:10E070000F945DB0882341F08091F7179091F817C5
:10E08000C29714F00C945E8881E090E0909318029F
:10E090008093170228966FAD28976093C0082A9640
:10E0A0008EAD9FAD2A979093BE088093BD082C96A5
:10E0B000AEADBFAD2C97B093BC08A093BB08109237
:10E0C000CE081092CD0882E00F94186B0C94E48770
:10E0D00080919110882309F49CC0EFEFF8E08491BF
:10E0E0008F01882339F00E94E53F0F5F1F4FF80131
:10E0F0008491F7CF4AE050E067E070E08CE197E070
:10E100000E942D3EEDEFF8E084918F01882339F0D5
:10E110000E94E53F0F5F1F4FF8018491F7CF4AE05F
:10E1200050E067E070E08CE197E00E942D3EEAEE5F
:10E13000F8E084918F01882339F00E94E53F0F5F5A
:10E140001F4FF8018491F7CF4AE050E065E070E09E
:10E150008CE197E00E942D3EE8EDF8E084918F017C
:10E16000882339F00E94E53F0F5F1F4FF80184912B
:10E17000F7CF8AE00E94E53F00E010E035EDA32EE6
:10E1800038E0B32E43ED842E48E0942EE12CF12CA0
:10E190009801275C3E4E6901F501849125ED622EC0
:10E1A00028E0722E882341F00E94E53FFFEF6F1AAE
:10E1B0007F0AF3018491F6CFF601EE0DFF1D418138
:10E1C00052816381748125E030E08CE197E00E9408
:10E1D000E93EF4E0EF0EF11C2CE1E216F104E1F669
:10E1E000F401849193EDE92E98E0F92E882341F013
:10E1F0000E94E53FFFEFEF1AFF0AF7018491F6CF87
:10E200000C5111090C33FFEF1F0709F0BFCF0C941D
:10E21000E487E5EBF8E084918F01882311F40C94F6
:10E2200053620E94E53F0F5F1F4FF8018491F5CFC5
:10E2300086EE0E94DA430C94E487109234080C9422
:10E24000E48785E40E94AE3F811102C00F94350D32
:10E2500013E6612E14E0712E02E7802E08E0902E66
:10E260008EE7A82E88E0B82E512CD3018D913D0168
:10E270000E94AE3F8823D9F1B3E05B120CC00E942C
:10E28000DC3FF50160837183828393838AE898E0A1
:10E290000F94CD032CC00E94DC3FD4012D913D9101
:10E2A0004D915C910F9459A3F50160837183828332
:10E2B0009383E0908608F090870800918808109179
:10E2C00089082091820830918308409184085091F8
:10E2D000850860917E0870917F08809180089091F8
:10E2E0008108BAE8CB2EB8E0DB2E0F945802539485
:10E2F000F4E08F0E911C24E0A20EB11C34E0531206
:10E30000B4CF0C94E48781E08093DD180F945B9B7D
:10E31000609302097093030980930409909305099F
:10E320006091DD1884EC9FE00F946FB00C94E4874B
:10E330008091520E9091530E895A914F9F938F93D3
:10E3400080EA98E09F938F930F9494AD0F900F9075
:10E350000F900F900C94E4878DE40E94AE3F8823C9
:10E3600011F40C94BA86E091480EF091490E319662
:10E3700081918032E9F38930D9F380538A30A0F05B
:10E380008091520E9091530E895A914F9F938F9383
:10E390008BE898E09F938F930F9494AD0F900F901C
:10E3A0000F900F900C94E4870E94DC3F0F94A1A47F
:10E3B0006837710511F40C94A37D0CF0D7C06C3252
:10E3C000710509F4A6C50CF064C06831710509F443
:10E3D000D9C30CF038C06231710511F40C945F7B25
:10E3E000CCF477FF02C00C94A786623071050CF460
:10E3F000C5C26131710511F00C94A786E6E8F6E418
:10E40000859194910F942830179816981598149820
:10E410000C94E4876531710509F48DC354F46431BB
:10E42000710511F00C94A786E6E0F8E405911491CB
:10E4300063C36631710509F484C36731710509F45A
:10E4400086C30C94A7866D31710511F40C94E48792
:10E4500084F46A31710509F4ABC30CF4A3C36B31C6
:10E46000710509F4B3C36C31710509F4B5C30C949B
:10E47000A7866F31710509F4ACC40CF4DCC36032BB
:10E48000710509F410C46A32710509F4FBC40C94D7
:10E49000A7866936710509F489C5C4F56335710528
:10E4A00011F40C945A7BFCF46F32710509F440C5E9
:10E4B00064F46D32710511F00C94A7868AE50E9410
:10E4C000AE3F0E94D84B0C94E4876135710511F47E
:10E4D0000C94347B6235710511F00C94A786109270
:10E4E00001090C94E4876535710511F40C94987B4F
:10E4F00014F40C945F7B6C35710511F40C94B37BB0
:10E500006836710509F41EC50C94A786603771053D
:10E5100009F436C59CF46B36710511F40C942E7B0E
:10E5200014F40C94FE7A6D36710509F469C66E36E2
:10E53000710511F40C94367C0C94A7866237710532
:10E5400011F40C94A37C14F40C94497C633771058A
:10E5500011F40C946F7C6737710511F00C94A78649
:10E56000E6EEF6E4059114910C94A87D6F3281E0FB
:10E57000780711F40C9428830CF081C06F3C71056E
:10E5800011F40C9457800CF045C0693C710511F4EE
:10E590000C94377FD4F46C38710509F4F6C454F444
:10E5A0006937710511F00C94A78681E00F948D05F1
:10E5B0000C94E4876E3B710509F4CCC6683C710588
:10E5C00011F40C94C27E0C94A7866C3C710511F476
:10E5D0000C94717F6CF46B3C710511F00C94A78660
:10E5E00003E614E040E0E42E47E1F42E0C94627F51
:10E5F0006D3C710511F40C94937F6E3C710511F024
:10E600000C94A78603E614E032E7E32E38E0F32EFD
:10E610000C944880623E710511F40C943981A4F485
:10E62000613D710511F40C94B28014F40C948C804B
:10E630006C3D710511F40C9404816D3D710511F46C
:10E640000C9413810C94A7866C32A1E07A0711F424
:10E650000C9495813CF4603F710511F40C94E487AF
:10E660000C94A7866D32E1E07E0711F40C94CB8107
:10E670006E32714011F40C941A830C94A78668359D
:10E6800022E0720711F40C945C840CF040C0643FEB
:10E6900081E0780711F40C946083ECF46E35A1E00E
:10E6A0007A0711F40C94FA853CF46033714011F44C
:10E6B0000C9486820C94A7866F35F1E07F0711F4E5
:10E6C0000C9431866039714011F00C94A7860F9438
:10E6D000350D0C94E487663F31E0730711F40C9418
:10E6E0006C8314F40C946683673F91E0790711F40E
:10E6F0000C946F836D3F714011F00C94A7860F94BA
:10E70000B92FE3EFFBE084918F010C9473836335A1
:10E71000B3E07B0711F40C948A830CF0FFC06A35D8
:10E72000F2E07F0711F40C94C68514F40C94B885BC
:10E730006D3B32E0730711F40C948D866E3B724092
:10E7400011F00C94A78650906A0210926A0281E040
:10E750008093C00882E090E09093BE088093BD084B
:10E76000E091CC08F0E0EE0FFF1FE050FB4B8591ED
:10E7700094910F94283020E030E044E352E460911B
:10E780008A0870918B0880918C0890918D080F9465
:10E7900058A360938A0870938B0880938C08909399
:10E7A0008D08E0908608F090870800918808109105
:10E7B0008908209182083091830840918408509103
:10E7C000850860917E0870917F0880918008909103
:10E7D0008108EAE66E2EE8E07E2E7F926F92812C11
:10E7E000912CFCEAAF2EF2E4BF2EAAE8CA2EA8E0D4
:10E7F000DA2E0E9488F70F94350D20E030E040E7D4
:10E8000051E460918A0870918B0880918C089091F6
:10E810008D080F9458A360938A0870938B08809397
:10E820008C0890938D08E0908608F09087080091FE
:10E8300088081091890820918208309183084091BE
:10E8400084085091850860917E0870917F088091BE
:10E850008008909181087F926F92812C912CB0E872
:10E86000AB2EB1E4BB2E0E9488F70F94350D20E04B
:10E8700030E040EA51E460918A0870918B08809101
:10E880008C0890918D080F9458A360938A08709318
:10E890008B0880938C0890938D08E0908608F09008
:10E8A000870800918808109189082091820830918A
:10E8B0008308409184085091850860917E0870918A
:10E8C0007F0880918008909181087F926F920E94CA
:10E8D00088F70F94350DE091CC08F0E0EE0FFF1FA4
:10E8E000E85DF94B859194910E94CC43149A64E6BB
:10E8F00070E080E090E00F948A9B9FB7F89480913D
:10E9000002018460809302019FBF0F900F900F90CF
:10E910000F900F900F9010E00C94A2866C3893E04B
:10E92000790711F40C94E4873CF46B38734011F4CC
:10E930000C94D4850C94A786603AE3E07E0709F432
:10E940001BC2673E734011F00C94A78610921E08FC
:10E950000F9459308091340E9091350EA091360E5F
:10E96000B091370E8093380E9093390EA0933A0EE3
:10E97000B0933B0E0E943D4E0C94E4870091480EEC
:10E980001091490E0E5F1F4F80E50E94AE3F882315
:10E9900079F00E94DC3F0F94A6A46B017C01BB249C
:10E9A000B394611571058105910531F4B12C04C052
:10E9B000B12CC12CD12C760183E50E94AE3F882377
:10E9C00099F00E94DC3F20E030E04AE754E40F94E5
:10E9D00007A70F94A6A46B017C01AA24A394611538
:10E9E00071058105910509F4A12C6AE270E0C80166
:10E9F0000F94F9AC009711F0DC011C92F801CF01E3
:10EA000021912032E1F3B11007C0A11005C02223EB
:10EA100019F00F941B3006C0E2EFF4E48591949155
:10EA20000F94283081E00F94FB2F0F94350D0F9435
:10EA30005B9B609330087093310880933208909309
:10EA40003308C114D104E104F104F1F00F945B9B8D
:10EA50004B015C018C0C9D1CAE1CBF1C84E090E043
:10EA600090931802809317020F945B9B68157905A9
:10EA70008A059B0510F00C94A0880F94B331811186
:10EA80000C94A0880C94AB880F94B131882311F4B6
:10EA90000C94E48784E090E090931802809317022E
:10EAA0000F94B331811109C00F94A21881E00E9424
:10EAB0006F5880E00F94186BF3CF82E090E0909352
:10EAC00018028093170280910809E091CC08F0E0C9
:10EAD000EE0FFF1F882341F0E65EF94B859194917C
:10EAE0000F9428300C94E487E458FB4B8591949163
:10EAF0000F9428300C94E487F8018491882329F03E
:10EB00000E94E53F0F5F1F4FF7CF8AE00E94E53F6D
:10EB100086E099E00E94CBA7E6EBF7E4059114911B
:10EB2000F8018491882311F40C9453620E94E53F0C
:10EB30000F5F1F4FF5CF86E099E00E9438B00C942C
:10EB4000E48786E099E00E9412A80C94E487809103
:10EB5000480E9091490E6AE270E004960F94F9AC69
:10EB6000009711F0DC011C926091480E7091490EE3
:10EB70006C5F7F4F21E041E086E099E00E9466AA49
:10EB80000C94E48786E099E00E9416A80F945B9BA2
:10EB9000609328087093290880932A0890932B0883
:10EBA0000C94E48786E099E00E941EA80C94E48708
:10EBB00080910909882311F40C94E48783E50E946D
:10EBC000AE3F81110C94B5880C94E48786E099E0FF
:10EBD0000E9493A80C94E4878091480E9091490E6E
:10EBE0006AE270E004960F94F9AC8C010097A9F0EA
:10EBF0008091520E9091530E6EE470E0895A914FBD
:10EC00000F94F9AC60E270E00F94F9AC0196909328
:10EC1000490E8093480EF80110826091480E709161
:10EC2000490E6C5F7F4F21E040E086E099E00E9452
:10EC300066AA0C94E48780910909882311F40C9446
:10EC4000E48760E086E099E00E9405AA8091480E82
:10EC50009091490E6AE270E004960F94F9AC8C0131
:10EC60000097A9F08091520E9091530E6EE470E0DF
:10EC7000895A914F0F94F9AC60E270E00F94F9ACAF
:10EC800001969093490E8093480ED8011C92609192
:10EC9000480E7091490E6C5F7F4F86E099E00E94AC
:10ECA000ECB10C94E4878091080981110F94350D23
:10ECB0000091480E1091490E0C5F1F4F6AE270E000
:10ECC000C8010F94F9AC7C0161E270E0C8010F94B7
:10ECD000F9AC009719F08C010F5F1F4FE114F1049C
:10ECE00011F0F701108280E50E94AE3FF82E2091CE
:10ECF000480E3091490E0217130708F4F12C809149
:10ED00000909882311F40C94E48721E02F2541E0C0
:10ED1000B80186E099E00E9466AA83E50E94AE3FB2
:10ED20008823B9F02091480E3091490E2017310701
:10ED300080F40E94D13FAB01BC014093170C50936B
:10ED4000180C6093190C70931A0C82E69BE00E94D9
:10ED5000229B86E099E00E9416A8F1100C94E487AB
:10ED60000F945B9B609328087093290880932A086E
:10ED700090932B080C94E4878091480E9091490E53
:10ED80006AE270E005960F94F9AC8C010097A9F047
:10ED90008091520E9091530E6EE470E0895A914F1B
:10EDA0000F94F9AC60E270E00F94F9AC0196909387
:10EDB000490E8093480ED8011C926091480E7091C4
:10EDC000490E6B5F7F4F86E099E00E9436AD0C9450
:10EDD000E4870F945B9B60932408709325088093CD
:10EDE000260890932708009128081091290820915F
:10EDF0002A0830912B08601B710B820B930B28EEB5
:10EE000033E040E050E00F9409A9CA01B9012CE3B6
:10EE100030E040E050E00F9409A97F936F933F9357
:10EE20002F938CE798E09F938F93CE0101969F9349
:10EE30008F930F9441AEE3EFFBE084910FB6F8940B
:10EE4000DEBF0FBECDBF03EF1BE0882339F00E9469
:10EE5000E53F0F5F1F4FF8018491F7CF8E010F5FE1
:10EE60001F4FD8018D918D01882319F00E94E53F35
:10EE7000F8CF8AE00E94E53FCE0101960F941B3047
:10EE80000C94E48783E50E94AE3F882311F40C9430
:10EE9000E4870E94DC3F0F94A1A4F62EE72E862F74
:10EEA0009E2D8C0180E50E94AE3F882331F00F3FFC
:10EEB000110509F010F40C94C6880DE010E0EBE2A7
:10EEC000F4E0819191918017910711F40C94E487FB
:10EED000B4E0E336FB07A9F70630110539F48F2DAE
:10EEE0009E2D909369088093680804C017FF02C0A4
:10EEF0000C94E48761E0802F0F94469D6F2D802F46
:10EF00000F947F9D6F2D7E2D802F0F942E9C0C943F
:10EF1000E4878FEF0E94DA4360E070E088EF9FE0C3
:10EF20000F9489B00E947DCD0E9410CE0C94E4878E
:10EF300084E090E090931802809317020F94CC45E0
:10EF40000C94E48788E690E00E94B65581110C94F9
:10EF5000E48783E50E94AE3F882371F000911F088B
:10EF60000E94DC3F10E0000F111F0750184E0F9455
:10EF7000A1A4F801718360830F94C7150C94E487F2
:10EF800063E08BEB94E00E94005583E50E94AE3F66
:10EF9000882311F40C94E4870E94DC3F0F94A1A411
:10EFA0007093F8176093F7170C94E48789E690E064
:10EFB0000E94B65581110C94E487E6E7F8E084914D
:10EFC0008F01882339F00E94E53F0F5F1F4FF80142
:10EFD0008491F7CFE0911F0824E0E29FF001112413
:10EFE000EF50F84E408151816281738121E030E021
:10EFF0008CE197E00E94E93EE3E7F8E084918F011D
:10F00000882339F00E94E53F0F5F1F4FF80184917C
:10F01000F7CFE0911F08F0E0EE0FFF1FE750F84E2A
:10F0200060817181882777FD8095982F0F94D4A4F3
:10F03000AB01BC0121E030E08CE197E00E94E93EA9
:10F04000EFE6F8E084918F01882339F00E94E53FD4
:10F050000F5F1F4FF8018491F7CF4091E117509156
:10F06000E2176091E3177091E41721E030E08CE142
:10F0700097E00E94E93EECE6F8E084918F01882356
:10F0800039F00E94E53F0F5F1F4FF8018491F7CFE1
:10F090006091F7177091F817882777FD8095982F62
:10F0A0000F94D4A4AB01BC0121E030E08CE197E0E7
:10F0B0000E94E93EE9E6F8E084918F01882339F067
:10F0C0000E94E53F0F5F1F4FF8018491F7CF4AE0A0
:10F0D00050E060E070E08CE197E00E942D3EE7E6B2
:10F0E000F8E084918F01882339F00E94E53F0F5F9B
:10F0F0001F4FF8018491F7CF4091F1175091F2170B
:10F100006091F3177091F41721E030E08CE197E003
:10F110000E94E93EE4E6F8E084918F01882339F00B
:10F120000E94E53F0F5F1F4FF8018491F7CF609178
:10F13000F9177091FA17882777FD8095982F0F940B
:10F14000D4A4AB01BC0121E030E08CE197E00E9447
:10F15000E93EE0E6F8E084918F01882339F00E94CF
:10F16000E53F0F5F1F4FF8018491F7CF80911F0893
:10F1700090E00F94D4144AE050E0BC018CE197E099
:10F180000E942D3EEBE5F8E084918F01882339F051
:10F190000E94E53F0F5F1F4FF8018491F7CF8FEF7B
:10F1A0009FEF0F94D4144AE050E0BC018CE197E04B
:10F1B0000E942D3EE7E5F8E084918F01882339F025
:10F1C0000E94E53F0F5F1F4FF8018491F7CF4091F8
:10F1D000EB175091EC176091ED177091EE1721E04D
:10F1E00030E08CE197E00E94E93E8AE00E94E53F32
:10F1F00081E090E090931802809317020C94738D35
:10F200008DE690E00E94B65581110C94E487E09160
:10F21000CC08F0E0EE0FFF1FE65CF84B859194916F
:10F220000F94283081E090E09093C4088093C30845
:10F230008091DD18882321F081E090E00F94AE3BAF
:10F2400083E50E94AE3F882391F000911F080E9441
:10F25000DC3F10E0000F111F0750184E0F94A1A4BF
:10F26000D8016D937C9381E08093080215C082E5FC
:10F270000E94AE3F882381F000911F080E94DC3F6E
:10F2800010E0000F111F0750184E0F94A1A4F801B1
:10F2900071836083109208020F94C7150F945B9BD3
:10F2A0006B017C0100911F0810E0F801EE0FFF1FB9
:10F2B000E750F84E60817181882777FD8095982FFF
:10F2C0000F94D4A4F801EE0FFF1FEE0FFF1FEF50B5
:10F2D000F84E11E020813181428153810F9435A68F
:10F2E00018160CF010E010931D0881E090E0909348
:10F2F00018028093170210925908C701B6010E94A4
:10F300007159E091CC08F0E0EE0FFF1FEA5CF84B7A
:10F31000859194910F94283082E090E090931802A8
:10F32000809317029093C4088093C3088091DD18DE
:10F33000882321F082E090E00F94AE3B0F945B9B1A
:10F3400060933008709331088093320890933308AB
:10F350000C94E487E091CC08F0E0EE0FFF1FE85C2E
:10F36000F74B859194910F94283083E090E090932F
:10F37000C4088093C3088091DD18882321F081E0C0
:10F3800090E00F94AE3B83E50E94AE3F882361F08E
:10F390000E94DC3F0F94A1A47093F8176093F717B5
:10F3A00081E0809308020FC082E50E94AE3F88236F
:10F3B00051F00E94DC3F0F94A1A47093F817609362
:10F3C000F717109208020F945B9B4B015C0110929F
:10F3D00059086091F7177091F817882777FD809585
:10F3E000982F0F94D4A411E02091E1173091E217E7
:10F3F0004091E3175091E4170F9435A618160CF0BE
:10F4000010E010931D0881E090E090931802809323
:10F41000170204E518E0F0E5EF2EF8E0FF2EACE46B
:10F42000CA2EA8E0DA2E80911D086091F71770911E
:10F43000F817882309F4A8C0809159088111A4C045
:10F44000882777FD8095982F0F94D4A42091E117F9
:10F450003091E2174091E3175091E4170F9435A6CD
:10F4600018160CF0A8C00F945B9B681979098A09DB
:10F470009B09693E73408105910508F47CC0809129
:10F48000DD18811174C0E0916A0824E0E29FF00168
:10F490001124EF50F84E4081518162817381F8014F
:10F4A0008491E4E5AE2EE8E0BE2E882301F1659656
:10F4B0004FAF659766965FAF669767966FAF679732
:10F4C00068967FAF68970E94E53FFFEFAF1ABF0ACB
:10F4D000F501849168967FAD689767966FAD6797E1
:10F4E00066965FAD669765964FAD6597DECF22E075
:10F4F00030E08CE197E00E94E93EF701849130E52D
:10F50000A32E38E0B32E882341F00E94E53FFFEFA1
:10F51000AF1ABF0AF5018491F6CF60916A0870E0D6
:10F520004AE050E08CE197E00E942D3EF601849184
:10F530002CE4A22E28E0B22E882341F00E94E53F61
:10F54000FFEFAF1ABF0AF5018491F6CF4091E117A2
:10F550005091E2176091E3177091E41721E030E0D9
:10F560008CE197E00E94E93E8AE00E94E53F0F941B
:10F570005B9B4B015C010F94A21880E00E946F58C6
:10F5800080E00F94186B4FCF882777FD8095982FD8
:10F590000F94D4A42091E1173091E2174091E31722
:10F5A0005091E4170F9432A487FF05C080910802A0
:10F5B000882309F458CFE091CC08F0E0EE0FFF1F4C
:10F5C000E45CF74B859194910F94283082E090E0B1
:10F5D000909318028093170284E090E09093C408FF
:10F5E0008093C3080F945B9B60933008709331083D
:10F5F00080933208909333080C94E48783E50E944B
:10F60000AE3F882319F10E94DC3F20E030E0A901E1
:10F610000F9432A487FD0FC00E94DC3F20E030E051
:10F620004FE753E40F9435A6181644F00E94DC3FD0
:10F630000F94A1A405C060E070E002C06FEF70E01D
:10F6400070936908609368080C94E4878FEF90E0EA
:10F6500090936908809368080C94E4871092690875
:10F66000109268080C94E4870F94C8150F94350D18
:10F67000149A0F94B30D109269081092680868EEFE
:10F6800073E080E090E00F948A9B10921902E4E806
:10F69000F6E4459154912AE438E068E478E08CE09F
:10F6A00094E00E9492BE0F94283080E00F94186B73
:10F6B0000C94E48781E0809301090C94E48783E54E
:10F6C0000E94AE3F882399F00E94DC3F20E030E0AA
:10F6D0004AE754E40F9407A70F94A6A460930A0284
:10F6E00070930B0280930C0290930D021DC088E56D
:10F6F0000E94AE3F81110C94CD8889E50E94AE3FF7
:10F7000081110C94CD888AE50E94AE3F81110C9442
:10F71000CD8885E40E94AE3F81110C94CD880F9472
:10F72000350D149A0F94B30D1092BA080C94E48717
:10F7300083E50E94AE3F882311F40C94E4870E9475
:10F74000DC3F20E030E04AE754E40F9407A70F9431
:10F75000A6A460932C0870932D0880932E08909394
:10F760002F080C94E48723E634E039AF28AF00EF8C
:10F7700016E1B0E0CB2EB7E1DB2E80EBE82E86E180
:10F78000F82E312CA8ADB9AD8D91B9AFA8AF0E94BC
:10F79000AE3F882309F45CC0B3E03B1252C00E9424
:10F7A000DC3F2B013C0120E030E040EA51E40F94C3
:10F7B00032A487FF3FC0A3019201F80160817181EB
:10F7C000828193810F9439A44B015C019B01AC01B0
:10F7D0006091D0167091D1168091D2169091D31667
:10F7E0000F9407A76093D0167093D1168093D2160A
:10F7F0009093D316A5019401D6016D917D918D91C1
:10F800009C910F9407A7F601608371838283938391
:10F81000D7016D917D918D919C910F94D2A4A501FA
:10F8200094010F9407A70F94A6A4F7016083718336
:10F8300082839383D8014D925D926D927C9213974F
:10F8400007C00E94DC3FF801608371838283938349
:10F8500033940C5F1F4FF4E0CF0ED11C24E0E20E76
:10F86000F11C34E033128ECF0C94E4878EE40E94B6
:10F87000AE3F882311F40C94E4870E94D13F60933B
:10F88000380E7093390E80933A0E90933B0E0C9481
:10F89000E48783E50E94AE3F882331F00E94C43F95
:10F8A000809312020C94E487E3EFFBE084918F01D4
:10F8B000882339F00E94E53F0F5F1F4FF8018491C4
:10F8C000F7CF4091120250E060E070E081E498E0F0
:10F8D0000E9408448AE00E94E53F0C94E48786E594
:10F8E0000E94AE3F882371F00F94BF978C01F801FE
:10F8F0008491882311F40C9453620E94E53F0F5FBA
:10F900001F4FF5CF85E50E94AE3F882369F08091B7
:10F91000480E9091490E01969093490E8093480E9F
:10F920000F94309A0C94E487ECEEF6E40591149170
:10F93000F8018491882311F40C94E4870E94E53F38
:10F940000F5F1F4FF5CFEEE3F8E084918F0188231E
:10F9500039F00E94E53F0F5F1F4FF8018491F7CF08
:10F9600040917E0850917F086091800870918108D5
:10F9700022E030E08CE197E00E94E93EEAE3F8E023
:10F9800084918F01882339F00E94E53F0F5F1F4F5C
:10F99000F8018491F7CF40918208509183086091DB
:10F9A00084087091850822E030E08CE197E00E94A5
:10F9B000E93EE6E3F8E084918F01882339F00E9464
:10F9C000E53F0F5F1F4FF8018491F7CF4091860804
:10F9D00050918708609188087091890822E030E092
:10F9E0008CE197E00E94E93EE2E3F8E084918F0128
:10F9F000882339F00E94E53F0F5F1F4FF801849183
:10FA0000F7CF40918A0850918B0860918C087091D3
:10FA10008D0822E030E08CE197E00E94E93EE0EDC5
:10FA2000F7E405911491F8018491882329F00E944C
:10FA3000E53F0F5F1F4FF7CF0F94920D0F94D4A4A3
:10FA40002091F0163091F1164091F2165091F31674
:10FA50000F9439A4AB01BC0122E030E08CE197E0C7
:10FA60000E94E93EEEE2F8E084918F01882339F0AC
:10FA70000E94E53F0F5F1F4FF8018491F7CF81E0AF
:10FA80000F94920D0F94D4A42091F4163091F51692
:10FA90004091F6165091F7160F9439A4AB01BC01B2
:10FAA00022E030E08CE197E00E94E93EEAE2F8E0F3
:10FAB00084918F01882339F00E94E53F0F5F1F4F2B
:10FAC000F8018491F7CF82E00F94920D0F94D4A4A3
:10FAD0002091F8163091F9164091FA165091FB16C4
:10FAE0000F9439A4AB01BC0122E030E08CE197E037
:10FAF0000E94E93EE6E2F8E084918F01882339F024
:10FB00000E94E53F0F5F1F4FF8018491F7CF83E01C
:10FB10000F94920D0F94D4A42091FC163091FD16F1
:10FB20004091FE165091FF160F9439A4AB01BC0111
:10FB300022E030E08CE197E00E94E93E8AE00E94FA
:10FB4000E53F0C94E48780E00F948D050C94E487E6
:10FB5000F8018491882329F00E94E53F0F5F1F4F31
:10FB6000F7CF8AE00E94E53FE2E9F4E405911491C1
:10FB7000F8018491882329F00E94E53F0F5F1F4F11
:10FB8000F7CF1E9B15C0EAEBF7E405911491F8013D
:10FB90008491882329F00E94E53F0F5F1F4FF7CF24
:10FBA0008AE00E94E53FE4E9F4E4059114910DC078
:10FBB000E8EBF7E405911491F8018491882381F32F
:10FBC0000E94E53F0F5F1F4FF7CFF8018491882314
:10FBD00029F00E94E53F0F5F1F4FF7CF379B15C0FD
:10FBE000EAEBF7E405911491F8018491882329F058
:10FBF0000E94E53F0F5F1F4FF7CF8AE00E94E53F6D
:10FC0000E6E8F4E4059114910DC0E8EBF7E4059102
:10FC10001491F8018491882381F30E94E53F0F5FDE
:10FC20001F4FF7CFF8018491882329F00E94E53F08
:10FC30000F5F1F4FF7CF1D9B15C0EAEBF7E405914F
:10FC40001491F8018491882329F00E94E53F0F5F09
:10FC50001F4FF7CF8AE00E94E53FE8E8F4E4059102
:10FC600014910DC0E8EBF7E405911491F80184912B
:10FC7000882381F30E94E53F0F5F1F4FF7CFF80104
:10FC80008491882329F00E94E53F0F5F1F4FF7CF33
:10FC9000029B15C0EAEBF7E405911491F8018491F9
:10FCA000882329F00E94E53F0F5F1F4FF7CF8AE0BE
:10FCB0000E94E53FE0E8F4E4059114910DC0E8EB03
:10FCC000F7E405911491F8018491882381F30E944F
:10FCD000E53F0F5F1F4FF7CFF8018491882329F08C
:10FCE0000E94E53F0F5F1F4FF7CF1C9B15C0EAEB4B
:10FCF000F7E405911491F8018491882329F00E947A
:10FD0000E53F0F5F1F4FF7CF8AE00E94E53FE2E833
:10FD1000F4E4059114910DC0E8EBF7E4059114911A
:10FD2000F8018491882381F30E94E53F0F5F1F4F04
:10FD3000F7CFF8018491882329F00E94E53F0F5FF7
:10FD40001F4FF7CF01990FC0EAEBF7E4059114912B
:10FD5000F8018491882311F40C9453620E94E53FCA
:10FD60000F5F1F4FF5CFE8EBF7E405911491F80111
:10FD70008491882311F40C9453620E94E53F0F5F35
:10FD80001F4FF5CF80916A0880931F0884E50E9479
:10FD9000AE3F882319F10E94DC3F0F94A6A4609324
:10FDA0001F086623D9F0E3EFFBE084918F018823DD
:10FDB00039F00E94E53F0F5F1F4FF8018491F7CFA4
:10FDC000E4EEF6E405911491D8018D918D0188231C
:10FDD00011F40C94E4870E94E53FF6CF84E40E947E
:10FDE000AE3F882311F40C94E4870E94DC3F20E0AE
:10FDF00030E0A9010F9432A4811103C010928E0843
:10FE000032C000911F0810E00E94DC3FF801EE0FA5
:10FE1000FF1FEE0FFF1FEA5BFD4F6083718382833C
:10FE20009383E0904602F0904702009148021091BF
:10FE3000490220E030E0A901B701C8010F9432A4C3
:10FE4000811104C0E12CF12C00E410E4C701D801B9
:10FE50008093460290934702A0934802B0934902D0
:10FE600081E080938E080E94F7560C94E48703E6A5
:10FE700014E050EEE52E56E1F52EF80181918F0148
:10FE80000E94AE3F882351F00E94DC3F0F94A6A44D
:10FE9000D7016D937D938D939C931397B4E0EB0EF4
:10FEA000F11CE4E007361E0741F70F94F3030C94AE
:10FEB000E487F4E0EF0EF11C24E00736120711F49A
:10FEC0000C94E487D8018D918D010E94AE3F882368
:10FED00081F30E94DC3FF701608371838283938307
:10FEE000E8CF83E50E94AE3F882351F00E94DC3FBB
:10FEF0006093D8167093D9168093DA169093DB1618
:10FF000084E50E94AE3F882311F40C94E4870E949C
:10FF1000DC3F6093D4167093D5168093D6169093D9
:10FF2000D7160C94E48783E50E94AE3F882351F0F6
:10FF30000E94DC3F6093DC167093DD168093DE1622
:10FF40009093DF1684E50E94AE3F882351F00E9413
:10FF5000DC3F6093C0167093C1168093C2169093D5
:10FF6000C31682E40E94AE3F882361F00E94DC3F0A
:10FF70000F94A6A460931017709311178093121713
:10FF80009093131788E50E94AE3F882391F00E945A
:10FF9000DC3F6093C8167093C9168093CA1690937D
:10FFA000CB166093C4167093C5168093C6169093B3
:10FFB000C71689E50E94AE3F882351F00E94DC3FBE
:10FFC0006093C8167093C9168093CA169093CB1687
:10FFD0008AE50E94AE3F882351F00E94DC3F609387
:10FFE000CC167093CD168093CE169093CF1685E4E1
:10FFF0000E94AE3F882351F00E94DC3F6093D016F0
:020000021000EC
:100000007093D1168093D2169093D31620E030E0EF
:1000100040E251E46091C4167091C5168091C616F5
:100020009091C7160F9435A6181664F480E090E0FE
:10003000A0E2B1E48093C4169093C516A093C616AF
:10004000B093C71620E030E040E251E46091C8165A
:100050007091C9168091CA169091CB160F9435A64F
:1000600018160CF0B1C780E090E0A0E2B1E48093F4
:10007000C8169093C916A093CA16B093CB16A4C7FE
:10008000F4E0EF0EF11C24E00636120709F49CC7D9
:10009000D8018D918D010E94AE3F882389F30E9483
:1000A000DC3FF7016083718382839383E9CF83E52B
:1000B0000E94AE3F882351F00E94DC3F60932602ED
:1000C00070932702809328029093290286E40E946D
:1000D000AE3F882381F00E94DC3F20E030E040E723
:1000E00052E40F9439A460931E0270931F02809310
:1000F0002002909321028AE50E94AE3F882309F4F2
:1001000063C70E94DC3F609362087093630880932A
:1001100064089093650858C783E50E94AE3F882322
:1001200051F00E94DC3F60935E0870935F088093FB
:1001300060089093610886E40E94AE3F882309F42A
:1001400043C70E94DC3F20E030E040E752E40F94D8
:1001500039A460931A0270931B0280931C0290933F
:100160001D0232C783E50E94AE3F882309F42CC7E5
:100170000E94DC3F0F94A1A46115710549F0613024
:10018000710559F481E080936708109266081CC7D6
:10019000109267081092660817C7E3EFFBE084919E
:1001A0008F01882339F00E94E53F0F5F1F4FF80150
:1001B0008491F7CFE4E0F5E405911491F80184917E
:1001C000882329F00E94E53F0F5F1F4FF7CF009172
:1001D000520E1091530E095A114FD8018D918D0175
:1001E000882319F00E94E53FF8CFE1E2F8E084911E
:1001F0008F01882311F40C9453620E94E53F0F5F36
:100200001F4FF8018491F5CF83E50E94AE3F88230C
:1002100009F4DAC60E94DC3F0F94A1A4709359023E
:1002200060935802D1C683E50E94AE3F882309F44B
:10023000CBC60E94DC3F0F94A1A46B017C0184E536
:100240000E94AE3F882381F08DED90E00E94B6556C
:100250008111BAC6E0911F08F0E0EE0FFF1FEC5AC3
:10026000FD4FD182C082B0C6D0925702C0925602D2
:10027000ABC680E50E94AE3F882309F4A5C60E9464
:10028000DC3F0F94A1A4D62E062F172F83E50E94E2
:10029000AE3F882331F00E94DC3F0F94A1A47B0184
:1002A00003C0EE24EA94FE2CC7010196039708F0E0
:1002B0008BC6EBE2F4E0819191918017910709F4EC
:1002C00083C624E0E336F207B1F717FD7DC60F942D
:1002D000350DCD2C60E08D2D0F94469D3FEFE3163C
:1002E000F30631F0EA94EF2871F000E010E00DC061
:1002F0008D2D0F94B49D31E020E0892B09F030E082
:10030000032F122F02C001E010E08C2D0F94B49D3A
:100310008017910709F458C60F94A21880E00E9434
:100320006F5880E00F94186BF0CF83E50E94AE3FCA
:10033000882331F00E94DC3F0F94A1A48B0102C0FE
:100340000EE610E080E50E94AE3F882331F00E9467
:10035000DC3F0F94A1A4CB0102C088EE93E06C01B6
:10036000EE24D7FCE094FE2C101611067CF420E05D
:1003700030E0A901B80184E50F94B39FC701B6012D
:100380000F948A9B84E50F94D7A21EC6C701B601BD
:100390000F948A9B19C680E50E94AE3F882351F0D6
:1003A0000E94DC3F6093AA027093AB028093AC0280
:1003B0009093AD0289E40E94AE3F882361F00E94D1
:1003C000DC3F0F94CC226093A6027093A702809327
:1003D000A8029093A90284E40E94AE3F882361F0B2
:1003E0000E94DC3F0F94D8226093A2027093A30274
:1003F0008093A4029093A50283E40E94AE3F8823D9
:1004000051F00E94DC3F60939E0270939F028093A4
:10041000A0029093A1020F94A714E2E8F6E40591DC
:100420001491F8018491882329F00E94E53F0F5F21
:100430001F4FF7CF0BE114E0D8018D918D01882378
:1004400019F00E94E53FF8CF4091AA025091AB020B
:100450006091AC027091AD0222E030E08CE197E057
:100460000E94E93E0FE114E0F80181918F01882399
:1004700019F00E94E53FF8CF6091A6027091A702A3
:100480008091A8029091A9020F94D222AB01BC01E5
:1004900022E030E08CE197E00E94E93E03E214E0C4
:1004A000D8018D918D01882319F00E94E53FF8CF86
:1004B0006091A2027091A3028091A4029091A50282
:1004C0000F94DE22AB01BC0122E030E08CE197E02A
:1004D0000E94E93E07E214E0F80181918F01882330
:1004E00019F00E94E53FF8CF40919E0250919F0283
:1004F0006091A0027091A10222E030E08CE197E0CF
:100500000E94E93E8AE00E94E53F5EC580E50E94C8
:10051000AE3F882351F00E94DC3F60939A027093B3
:100520009B0280939C0290939D0289E40E94AE3FBF
:10053000882361F00E94DC3F0F94CC2260939602E6
:1005400070939702809398029093990284E40E949A
:10055000AE3F882361F00E94DC3F0F94D822609365
:1005600092027093930280939402909395020F9459
:10057000A714E2E8F6E405911491F8018491882328
:1005800029F00E94E53F0F5F1F4FF7CF0BE114E00A
:10059000D8018D918D01882319F00E94E53FF8CF95
:1005A00040919A0250919B0260919C0270919D0231
:1005B00022E030E08CE197E00E94E93E0FE114E098
:1005C000F80181918F01882319F00E94E53FF8CF4F
:1005D0006091960270919702809198029091990291
:1005E0000F94D222AB01BC0122E030E08CE197E015
:1005F0000E94E93E03E214E0D8018D918D01882329
:1006000019F00E94E53FF8CF609192027091930239
:1006100080919402909195020F94DE22AB01BC016F
:1006200022E030E08CE197E00E94E93E8AE00E94FF
:10063000E53FCAC483E50E94AE3F882319F00E94BB
:10064000DC3F03C060E070E0CB010F94EA03BCC460
:1006500085E40E94AE3F882341F00E94DC3F0F9466
:10066000A1A48B0177FF03C009C000E010E0C12CFA
:10067000D12C86E1E82E83E4F82E06C0C12CD12CC3
:10068000BCE8EB2EB2E4FB2E83E50E94AE3F88234C
:1006900021F00E94DC3F6B017C0183E40E94AE3FAD
:1006A000882331F00E94DC3F0F94A1A49B0102C07B
:1006B00025E030E0A801C701B6010F94221C84C4D4
:1006C00060E084E190E00E94FC307EC460E084E160
:1006D00090E00E94593778C40E94D53575C480E0F7
:1006E0000E94033271C4882339F00E94E53F0F5FF6
:1006F0001F4FF8018491F7CFE1E1F8E084918F0179
:10070000882309F461C40E94E53F0F5F1F4FF80181
:100710008491F6CF8AE50E94AE3F882309F497C002
:100720000E94DC3F6B017C0120E030E040E751ECAF
:100730000F9435A687FD43C020E030E040EA50EC3E
:10074000C701B6010F9432A418160CF438C0F7FA9A
:10075000F094F7F8F094C0926B08D0926C08E09295
:100760006D08F0926E08E3EFFBE084918F0188231F
:1007700039F00E94E53F0F5F1F4FF8018491F7CFDA
:10078000E2E8F6E445915491E4E8F4E4859194912B
:1007900020E138E06AE576E00E9492BE8C01F80123
:1007A0008491882329F00E94E53F0F5F1F4FF7CF08
:1007B0008AE00E94E53F8AE00E94E53F05C4E3EF3E
:1007C000FBE084918F01882339F00E94E53F0F5FA1
:1007D0001F4FF8018491F7CFE4E8F4E405911491F8
:1007E000F8018491882329F00E94E53F0F5F1F4F95
:1007F000F7CFE0E8F4E405911491F801849188239F
:1008000029F00E94E53F0F5F1F4FF7CF4AE050E00D
:1008100061EF7FEF8CE197E00E942D3EE2E8F4E487
:1008200005911491F8018491882329F00E94E53FF5
:100830000F5F1F4FF7CF4AE050E06BEF7FEF8CE187
:1008400097E00E942D3E8AE00E94E53FBDC3E3EFA2
:10085000FBE084918F01882339F00E94E53F0F5F10
:100860001F4FF8018491F7CFE4E8F4E48591949167
:100870006CE078E00E9471BE8C01F80184918823BD
:1008800029F00E94E53F0F5F1F4FF7CF8AE00E94DB
:10089000E53F40916B0850916C0860916D08709134
:1008A0006E08705822E030E08CE197E00E94E93E4B
:1008B0008AE00E94E53F88C350906A0210926A0263
:1008C0000F94350D8091DD18882321F086E190E0AA
:1008D0000F94AE3B809158029091590290934B0235
:1008E00080934A02E0916A08F0E0EE0FFF1FE750A4
:1008F000F84E608071802090680830906908C09040
:100900007E08D0907F08E0908008F0908108CF8E1C
:10091000D8A2E9A2FAA2009182081091830820913E
:100920008408309185080BA31CA32DA33EA34091FE
:1009300086085091870860918808709189084FA3B4
:1009400058A769A77AA780918A0890918B08A091EF
:100950008C08B0918D088BA79CA7ADA7BEA7C982B4
:10096000DA82EB82FC820D831E832F8338874987CE
:100970005A876B877C878D879E87AF87B88B85E486
:100980000E94AE3F882359F00E94DC3F9B01AC01DE
:100990006BA57CA58DA59EA50F9459A30AC020E048
:1009A00030E040E050E46BA57CA58DA59EA50F949A
:1009B00058A36BA77CA78DA79EA7EFA0F8A409A5B5
:1009C0001AA52BA13CA14DA15EA16F8D78A189A193
:1009D0009AA1EAE6F8E0FF93EF93812C912CE8EEE0
:1009E000AE2EE2E4BE2EDE019B966D010E9488F7DA
:1009F0008AE50E94AE3F0F900F90882349F00E9435
:100A0000DC3F9B01AC016FA178A589A59AA51EC00A
:100A100020E030E040E050E46FA178A589A59AA5D8
:100A20000F9459A36B017C016FA378A789A79AA79C
:100A300020E030E040E251E40F9432A487FF0CC084
:100A400020E030E040E251E4C701B6010F9459A321
:100A50006FA378A789A79AA7EFA0F8A409A51AA55C
:100A60002BA13CA14DA15EA16F8D78A189A19AA176
:100A7000EAE6F8E0FF93EF93812C912CB0E7AB2EE0
:100A8000B1E4BB2EFE01BB966F010E9488F788E59A
:100A90000E94AE3F0F900F90882379F00E94DC3FB8
:100AA0009B01AC016F8D78A189A19AA10F9459A3E4
:100AB0006F8F78A389A39AA308C080E090E0A3E594
:100AC000B3E48F8F98A3A9A3BAA389E50E94AE3F90
:100AD000882339F00E94DC3F6BA37CA38DA39EA3E7
:100AE00004C01BA21CA21DA21EA2EFA0F8A409A56F
:100AF0001AA52BA13CA14DA15EA16F8D78A189A162
:100B00009AA1EAE6F8E0FF93EF93812C912CE8E4B8
:100B1000AE2EE2E4BE2EDE019B966D010E9488F7A8
:100B20000F94350D84E090E09093180280931702A3
:100B300010926908109268080F945B9B4B015C014E
:100B4000E091CC08F0E0EE0FFF1FEE5BF94B8591D2
:100B500094910E94CC430F900F90412C00E010E044
:100B6000411085C30F94B331882309F480C31EC498
:100B70008091E1189091E218892B09F025C285E057
:100B800090E09093E2188093E1181EC28091E118E2
:100B90009091E218892B09F017C286E090E09093BB
:100BA000E2188093E11810C288E50E94AE3F8823C6
:100BB00039F00E94DC3F0F94A1A480E00F94B40EA2
:100BC0008AE50E94AE3F882339F00E94DC3F0F94F3
:100BD000A1A481E00F94B40E85E40E94AE3F882367
:100BE00009F4F2C10E94DC3F0F94A1A482E00F94AB
:100BF000B40EEAC183E50E94AE3F811104C003E652
:100C000014E0F12C10C010E00E94DC3F0F94A6A469
:100C1000812F0F948E0F1F5F1530B1F7F0CFF39433
:100C2000B4E0FB1679F0D8018D918D010E94AE3FA2
:100C30008823A9F30E94DC3F0F94A6A48F2D0F9464
:100C40008E0FEDCF82E40E94AE3F882339F00E94E0
:100C5000DC3F0F94A6A484E00F948E0F0F945110E4
:100C6000B3C183E50E94AE3F882309F453C00E94BC
:100C7000DC3F0F94A1A46130710541F06230710531
:100C800009F048C003E614E0F12C25C003E614E0A7
:100C9000F12CF80181918F010E94AE3F882341F031
:100CA0000E94DC3F0F94A1A44FEF8F2D0F94500FA3
:100CB000F394F4E0FF12EDCF82E40E94AE3F88236C
:100CC00049F10E94DC3F0F94A1A44FEF20C0F394A0
:100CD000B4E0FB1689F0D8018D918D010E94AE3FE2
:100CE0008823A9F30E94DC3F0F94A1A4462F6FEF45
:100CF0008F2D0F94500FEBCF82E40E94AE3F8823DC
:100D000049F00E94DC3F0F94A1A4462F6FEF84E0CE
:100D10000F94500F0F94511057C10E942B5754C17C
:100D2000123309F4B6C6163040F09FB7F89480919C
:100D300002018B7F809302019FBF84E690E00E94B6
:100D400009571F5F0F94B3318111A3C6E9CF80917A
:100D5000520E9091530E895A914F9F938F938EEE1E
:100D600097E09F938F930F9494AD0F900F900F90F7
:100D70000F902AC184E50E94AE3F882309F4B9C0D0
:100D80000F94350DE091480EF091490E3196819106
:100D90008032E9F38930D9F390ED980F9A30B0F0B2
:100DA0008F3379F0EEEDF7E084918F01882311F411
:100DB0000C9453620E94E53F0F5F1F4FF80184912E
:100DC000F5CF0F949F9680931F0806C00E94DC3FCA
:100DD0000F94A6A460931F0820911F08E22EF12C07
:100DE00081E090E0022E01C0880F0A94EAF790910A
:100DF000BA08982B9093BA08222309F433C0E3EF82
:100E0000FBE084918F01882339F00E94E53F0F5F5A
:100E10001F4FF8018491F7CFECEDF7E084918F013B
:100E2000882339F00E94E53F0F5F1F4FF80184913E
:100E3000F7CF4AE050E0B7018CE197E00E942D3EE9
:100E40008AE00E94E53FE2E1F7E405911491F801A0
:100E50008491882311F40C9453620E94E53F0F5F44
:100E60001F4FF5CF86E40E94AE3F8823D9F00E9441
:100E7000DC3F6B017C016093390870933A088093E2
:100E80003B0890933C0820E030E0A9010F9435A680
:100E9000181644F4C0920E02D0920F02E092100293
:100EA000F0921102E3EFFBE084918F01882339F087
:100EB0000E94E53F0F5F1F4FF8018491F7CFE6E7EF
:100EC000F8E405911491F8018491882329F00E9497
:100ED000E53F0F5F1F4FF7CF60916A0870E04AE06F
:100EE00050E08CE197E00E942D3E8AE00E94E53FB1
:100EF0006BC0E3EFFBE084918F01882339F00E94FF
:100F0000E53F0F5F1F4FF8018491F7CFE4E0F5E470
:100F100005911491F8018491882329F00E94E53FFE
:100F20000F5F1F4FF7CF0091520E1091530E095AC9
:100F3000114FD8018D918D01882319F00E94E53F52
:100F4000F8CFE7EDF7E084918F01882311F40C943A
:100F500053620E94E53F0F5F1F4FF8018491F5CF68
:100F6000711028C0662031F181E0809391100F94B8
:100F7000A00D6B017C0180E00F94A00DAB01BC01C2
:100F80009701860181E990E10E94FD3F9B01AC0140
:100F900060918608709187088091880890918908EF
:100FA0000F9458A3609386087093870880938808ED
:100FB000909389088091DD18882321F084E190E0E6
:100FC0000F94AE3B1092FA0881E090E090931802E3
:100FD000809317020E947F4E86C5C0905508D0901E
:100FE0005608E0905708F090580820918A083091F0
:100FF0008B0840918C0850918D08C701B6010F9461
:1010000058A32DEC3CEC4CEC5DE30F9435A6181680
:1010100014F00C94CD63C0928A08D0928B08E092B1
:101020008C08F0928D088AE898E00F94CD0360E078
:1010300080E00E94735257C50E94DC3F20917208E5
:101040003091730840917408509175080F9459A31A
:1010500060937E0870937F08809380089093810846
:101060000C94C4640E94DC3F20917608309177088C
:1010700040917808509179080F9459A360938208A1
:101080007093830880938408909385080C94D164AE
:101090000E94DC3F20917A0830917B0840917C08C7
:1010A00050917D080F9459A3609386087093870828
:1010B00080938808909389080C94D26520E030E0F2
:1010C00040E85FE360918A0870918B0880918C08FA
:1010D00090918D080F9459A360938A0870938B08A0
:1010E00080938C0890938D08E0908608F090870894
:1010F0000091880810918908209182083091830816
:10110000409184085091850860917E0870917F0815
:101110008091800890918108EAE6F8E0FF93EF93D0
:10112000812C912CE8ECAE2EE3E4BE2EFAE8CF2E13
:10113000F8E0DF2E0E9488F70F900F900C94447017
:1011400082E090E0909318028093170280E00F9461
:10115000FB2F0C9463750F94A21881E00E946F58C6
:1011600080E00F94186B0C9434750E94D13FAB0152
:10117000BC014093170C5093180C6093190C70939A
:101180001A0C82E69BE00E94229B1ECF0E94DC3F4D
:101190000F94A1A48B010C945F770F94350D88E513
:1011A0000E94AE3F882319F0179A10926F0889E5C4
:1011B0000E94AE3F882319F0169A109270088AE5B3
:1011C0000E94AE3F85E40E94AE3F882311F40C9448
:1011D000947B149A0C94947B809101018460809399
:1011E00001010115110509F04FC09FB7F8948091D6
:1011F00002018460809302019FBF0F5F1F4FB1E027
:101200004B1609F44FC04B1608F048C084E090E03C
:101210000E9409570F945B9B75016401F0ECCF0E9F
:10122000F7E2DF1EF9E0EF1EF11CC616D706E8064E
:10123000F90608F095CCE091CC08F0E0EE0FFF1F26
:10124000EA5BF94B859194910E94CC431092FA1776
:101250001092F9171092FC171092FB171092FE17BC
:101260001092FD170F94350D149A442443940F9453
:10127000A21881E00E946F58043FF1E01F0709F0B7
:10128000ABCF00E010E0A8CF0431110509F0B5CFD5
:101290009FB7F894809102018B7FACCFE2E04E16AD
:1012A000B9F05ECC84E090E00E9409570F94B3310E
:1012B0008823E9F2E0916A08F0E0EE0FFF1FE750A3
:1012C000F84E718260820F94DE6E42E0442ECFCFE2
:1012D000E0906A08F12CF701EE0FFF1FE750F84E7F
:1012E00060817181882777FD8095982F0F94D4A411
:1012F000F701EE0FFF1FEE0FFF1FEF50F84E20819A
:101300003181428153810F9458A36B017C0120E00D
:1013100030E0A9010F9435A618165CF420E030E007
:1013200040E85FE3C701B6010F9432A487FF1CC0F9
:101330000AC020E030E040E85FEBC701B6010F943F
:1013400035A618168CF4E091CC08F0E0EE0FFF1FE4
:10135000EE5BF94B859194910E94CC430F945B9B7B
:101360004B015C01412CFECB44E061E08CE598E14F
:101370000E945B39E0916A0824E0E29FF0011124A9
:10138000EF50F84E80819181A281B3818FA798ABF5
:10139000A9ABBAABCE018F960F947A40BC018CE515
:1013A00098E10F941A9E04E110E061CF9FB7F89482
:1013B000809102018B7F809302019FBF1092F208FF
:1013C0001092F108E091CC08F0E0EE0FFF1FE05022
:1013D000FB4B859194910E94CC4382E090E09093E6
:1013E00018028093170281E08093C008E091CC0836
:1013F000F0E0EE0FFF1FE050FB4B859194910F94AE
:1014000028308CE40E94AE3F882359F00E94DC3FD4
:101410009B01AC016BA57CA58DA59EA50F9459A33E
:101420000AC020E030E040EA52E46BA57CA58DA51F
:101430009EA50F9458A36BA77CA78DA79EA720E01D
:1014400030E040EA52E46BA57CA58DA59EA50F94E3
:1014500059A320E030E044E352E40F9458A36BA773
:101460007CA78DA79EA7EFA0F8A409A51AA52BA17C
:101470003CA14DA15EA16F8D78A189A19AA1BAE688
:101480006B2EB8E07B2E7F926F92812C912CECEA30
:10149000AE2EE2E4BE2EDE019B966D010E9488F71F
:1014A0000F94350D20E030E040E751E46BA57CA5BA
:1014B0008DA59EA50F9458A36BA77CA78DA79EA76B
:1014C000EFA0F8A409A51AA52BA13CA14DA15EA1EE
:1014D0006F8D78A189A19AA17F926F92812C912C16
:1014E000F0E8AF2EF1E4BF2E0E9488F70F94350D7F
:1014F00020E030E040EA51E46BA57CA58DA59EA5D7
:101500000F9458A36BA77CA78DA79EA7EFA0F8A464
:1015100009A51AA52BA13CA14DA15EA16F8D78A1B3
:1015200089A19AA17F926F920E9488F70F94350D3E
:101530000F94350DE091CC08F0E0EE0FFF1FE85D51
:10154000F94B859194910E94CC43149A64E670E023
:1015500080E090E00F948A9B9FB7F89480910201FD
:101560008460809302019FBF0F900F900F900F90A7
:101570000F900F9000E010E00F94B331811104C080
:101580000233110509F073C29FB7F89480910201EC
:101590008B7F809302019FBF84E090E090931802BC
:1015A00080931702E091CC08F0E0EE0FFF1FE850A7
:1015B000FB4B8591949141E060E00F94377099273F
:1015C00087FD90959093F2088093F108892B59F448
:1015D000E091CC08F0E0EE0FFF1FE851F84B859149
:1015E00094910F945D7A81E00F94E66D0F94DC4A3C
:1015F00084E090E090931802809317028091060295
:10160000882391F0511004C080914E10882361F01E
:101610000E94DFBC09C00F94A21881E00E946F589D
:1016200080910602811105C00F94B331882399F38C
:1016300019C0511004C080914E108823A9F30E9454
:1016400004BD882389F320E030E0A90168EE73E04F
:1016500084E50F94B39F82E390E00E94095784E5EC
:101660000F94D7A280910602882339F0511003C04D
:1016700080914E1081110E94FDBC82E090E0909319
:1016800018028093170220E030E04CE852E46BA58A
:101690007CA58DA59EA50F9459A36BA77CA78DA7AC
:1016A0009EA7EFA0F8A409A51AA52BA13CA14DA1C6
:1016B0005EA16F8D78A189A19AA1AAE66A2EA8E001
:1016C0007A2E7F926F92812C912CB0EAAB2EB1E4EE
:1016D000BB2EFE01BB966F010E9488F720E030E030
:1016E00048E452E46BA57CA58DA59EA50F9459A353
:1016F0006BA77CA78DA79EA7EFA0F8A409A51AA5A4
:101700002BA13CA14DA15EA16F8D78A189A19AA1C9
:101710007F926F92812C912CA12CE0E4BE2E0E942E
:1017200088F71092F2081092F1080F945D4B20E0B8
:1017300030E0A90164EF71E084E50F94B39F82E388
:1017400090E00E94095784E50F94D7A20F900F9064
:101750000F900F908091F1089091F208019709F491
:101760009AC01092F2081092F108E4E0F0E0F093D1
:101770001802E09317020F94A74B22E030E0309359
:101780001802209317028091F1089091F20882309C
:10179000910571F1039709F078C020E030E048E44A
:1017A00052E46BA57CA58DA59EA50F9459A36BA7AC
:1017B0007CA78DA79EA7EFA0F8A409A51AA52BA129
:1017C0003CA14DA15EA16F8D78A189A19AA17F92C4
:1017D0006F92812C912CA12CB0E4BB2EDE019B9644
:1017E0006D010E9488F70F94134B0F900F90B2CFAA
:1017F00020E030E04CE852E46BA57CA58DA59EA5C9
:101800000F9459A36BA77CA78DA79EA7EFA0F8A460
:1018100009A51AA52BA13CA14DA15EA16F8D78A1B0
:1018200089A19AA17F926F92812C912CE0EAAE2E31
:10183000E1E4BE2EDE019B966D010E9488F720E058
:1018400030E048E452E46BA57CA58DA59EA50F94DD
:1018500059A36BA77CA78DA79EA7EFA0F8A409A505
:101860001AA52BA13CA14DA15EA16F8D78A189A1E4
:101870009AA17F926F92812C912CA12CF0E4BF2E23
:101880000E9488F70F945D4B61CF0F94004B81E06D
:101890000F94E66D5FCF309269082092680820E0CF
:1018A00030E040EA50E46BA57CA58DA59EA50F9481
:1018B00059A36BA77CA78DA79EA7EFA0F8A409A5A5
:1018C0001AA52BA13CA14DA15EA16F8D78A189A184
:1018D0009AA1EAE66E2EE8E07E2E7F926F92812C2E
:1018E000912CA12CF0E4BF2EFE01BB966F010E944B
:1018F00088F7A50194016BA57CA58DA59EA50F94E5
:1019000058A36BA77CA78DA79EA7EFA0F8A409A555
:101910001AA52BA13CA14DA15EA16F8D78A189A133
:101920009AA17F926F92812C912CA8EEAA2EA2E40C
:10193000BA2E0E9488F7EFA0F8A409A51AA52D8158
:101940003E814F81588569817A818B819C817F920C
:101950006F92812C912CB8E4AB2EB2E4BB2E0E9486
:1019600088F7E984FA840B851C852D813E814F819F
:10197000588569817A818B819C817F926F92812CBD
:10198000912CE0E7AE2EE1E4BE2E0E9488F720E025
:1019900030E040E050E46BA57CA58DA59EA50F949A
:1019A00059A36BA77CA78DA79EA7E984FA840B8512
:1019B0001C852D813E814F81588569817A818B817B
:1019C0009C817F926F92812C912CF8EEAF2EF2E4E5
:1019D000BF2E0E9488F7CE010D960F94CD03809103
:1019E0004A0290914B0280935802909359029F9320
:1019F0008F9383E098E09F938F938E01015D1F4F3B
:101A00001F930F930F9441AE60E0C8010E94C9B5C7
:101A1000E091CC08F0E0EE0FFF1FE458FB4B8591FE
:101A200094910F9428301092C0081092BE08109222
:101A3000BD0850926A020FB6F894DEBF0FBECDBF4C
:101A400080914E10882309F4BFCA0E94F3B40F940A
:101A5000350D0E942CB7811105C00E94E1600E94E3
:101A6000F3B4F7CF0E9454BC0E9441BCADCA06300B
:101A7000110544F09FB7F894809102018B7F809309
:101A800002019FBF84E690E00E9409570F5F1F4F3D
:101A900073CD9FB7F894809102018B7F80930201F0
:101AA0009FBF0F94350D0F94B331882329F084E63E
:101AB00090E00E940957F7CF81E00F94E66DE09126
:101AC000CC08F0E0EE0FFF1FE458FB4B859194919A
:101AD0000F9428301092C0081092BE081092BD08D2
:101AE00050926A0271CAC95ADF4F0FB6F894DEBF2E
:101AF0000FBECDBFDF91CF911F910F91FF90EF905F
:101B0000DF90CF90BF90AF909F908F907F906F901D
:101B10005F904F903F902F9008950F931F9381E017
:101B200090E090931802809317028091F3089091AF
:101B3000F408892BA1F00F945B9B00912008109171
:101B400021082091220830912308601B710B820B21
:101B5000930B693E73408105910508F092C0809116
:101B6000F3089091F408892B11F41092FB088091EE
:101B7000CB08882319F00E943E4B6FC00E9435B7F6
:101B800060E086E099E00E94F6B080914E0E909160
:101B90004F0E892B09F461C010924D0E80910609F9
:101BA0008823B1F00091520E1091530E095A114F33
:101BB0006BE67AE0C8010F94A4AC892BE9F4B80174
:101BC00086E099E00E9462A980910709882319F0B4
:101BD0000E94E16023C0E2E8F6E405911491F80167
:101BE0008491882329F00E94E53F0F5F1F4FF7CFB4
:101BF0008AE00E94E53F12C060E086E099E00E9422
:101C000005AAE8E7F7E405911491F8018491882387
